:100000000C9464110C945D140C9488140C94B31427
:100010000C94DE140C9409150C9434150C945F1593
:100020000C948A150C9494110C9494110C949411C2
:100030000C9494110C9494110C9494110C949411AC
:100040000C9494110C94DD340C9494110C94941130
:100050000C9494110C9494110C9422290C949611E4
:100060000C9494110C94871A0C94331B0C949411D7
:100070000C9494110C9494110C9494110C9494116C
:100080000C9494110C9494110C9494110C9494115C
:100090000C9494110C9494110C9494110C9494114C
:1000A0000C9494110C9494110C9494110C9494113C
:1000B0000C9494110C9494110C9494110C9494112C
:1000C0000C9494110C9494110C9494110C9494111C
:1000D0000C9494110C9494110C9494110C9494110C
:1000E0000C949411D312D812DD12E712F1126A1394
:1000F000FB1203130B1315131F1329133813421389
:100100006A134C13561360138E13911380138413C8
:100110008A13C813951399139F13A313A713AD1331
:10012000B113B513C813BB13BF13C313C317C11740
:10013000E517E217E01717181418121870183E1870
:100140003B183918BA1AC01AD11ADC1AE41AF91A6B
:10015000E81AF91AEC1AF01AF91AF61A084AD73BF3
:100160003BCE016E84BCBFFDC12F3D6C74319ABD86
:1001700056833DDA3D00C77F11BED9E4BB4C3E91AA
:100180006BAAAABE000000803F05A84CCDB2D44E99
:10019000B93836A9020C50B9918688083CA6AAAA9B
:1001A0002ABE000000803F004E414E494E4954593E
:1001B000494E46CDCCCC3D0AD7233C17B7D1387732
:1001C000CC2B329595E6241FB14F0A000020410048
:1001D00000C84200401C4620BCBE4CCA1B0E5AAE92
:1001E000C59D7400000A0B02090C0D0E08070304DC
:1001F00001000000000000000000000000000000FE
:1002000000000000000000000000000000000012DC
:1002100011100000000000000000000000000000BD
:10022000000000000000000000010210202008086B
:100230001020401020408002010201080402010148
:100240000204081020408080402010080402018031
:100250000402018040201008040201080402010188
:10026000020408102040800102040810204080058C
:10027000050505070508080808020202020A0A081F
:100280000804040404010101010101010103030345
:100290000303030303040707070C0C0C0C0C0C0CE2
:1002A0000C0202020206060606060606060B0B0BE9
:1002B0000B0B0B0B0B000020002300260029002C49
:1002C000002F0032000001000003010601090100B7
:1002D000002200250028002B002E003100340002EF
:1002E000010000050108010B010000210024002786
:1002F000002A002D00300033000101000004010736
:10030000010A014F4646004F4E006563686F3A0090
:100310004572726F723A004572726F72207772691D
:1003200074696E6720746F20454550524F4D210A05
:100330000063616E63656C00706F7765726F6666EF
:10034000002F2F616374696F6E3A0020573A0020C6
:10035000573A00202F002042403A0020403A0054F3
:100360006865726D616C2052756E617761790048C5
:100370006F7420456E6420544845524D414C2052C4
:10038000554E415741590042454420544845524D2D
:10039000414C2052554E4157415900202D20496E65
:1003A00076616C6964206578747275646572206E1C
:1003B000756D62657220210A0048656174696E6717
:1003C000206661696C6564004265642068656174DB
:1003D000696E67206661696C656400546865726D5A
:1003E000616C2052756E61776179004245442054FA
:1003F0004845524D414C2052554E415741590048B5
:10040000656174696E67206661696C656400486F38
:100410007420456E642048656174696E672066616A
:10042000696C656400546865726D616C2052756E0C
:100430006177617900486F7420456E6420544845A7
:10044000524D414C2052554E41574159004D494E55
:1004500054454D5020747269676765726564004841
:100460006F7420456E64204572723A204D494E5497
:10047000454D50004572723A204D494E54454D50FD
:1004800020424544004D415854454D5020747269F6
:1004900067676572656400486F7420456E64204527
:1004A00072723A204D415854454D50004572723A8F
:1004B000204D415854454D502042454400626564EA
:1004C000002C2073797374656D2073746F70706580
:1004D0006421204865617465725F49443A200023B5
:1004E000646566696E652044454641554C545F001D
:1004F0004B6420004B6920004B7020000062656453
:1005000000504944204175746F74756E65206669AA
:100510006E69736865642120507574207468652065
:100520006C617374204B702C204B6920616E6420C9
:100530004B6420636F6E7374616E74732066726FA8
:100540006D2062656C6F7720696E746F20436F6EEB
:1005500066696775726174696F6E2E680A0050492A
:1005600044204175746F74756E65206661696C65B1
:1005700064212074696D656F75740A005468657232
:100580006D616C2052756E6177617900486F7420DF
:10059000456E6420544845524D414C2052554E41C1
:1005A0005741590042454420544845524D414C2042
:1005B00052554E415741590048656174696E672034
:1005C0006661696C656400486F7420456E642048FC
:1005D000656174696E67206661696C656400426577
:1005E000642068656174696E67206661696C656422
:1005F00000504944204175746F74756E65206661C2
:10060000696C6564212054656D70657261747572E2
:100610006520746F6F20686967680A00204B643A30
:100620002000204B693A2000204B703A20000A201D
:10063000436C617373696320504944200A0020545D
:10064000753A2000204B753A2000206D61783A20E1
:1006500000206D696E3A200020643A200020626913
:1006600061733A2000504944204175746F74756E6F
:10067000652073746172740A005049442041757496
:100680006F74756E65206661696C656421205465C0
:100690006D706572617475726520746F6F20686922
:1006A00067680A001000AD0330016A0150022B0197
:1006B00070030A019004F500B005E500D006D800EB
:1006C000F007CE001009C500300ABE00500BB7007D
:1006D000700CB100900DAB00B00EA600D00FA200C0
:1006E000F0109D00101299003013950050149200E4
:1006F00070158E0090168B00B0178700D0188400FC
:10070000F0198100101B7E00301C7B00501D790009
:10071000701E7600901F7300B0207000D0216E0014
:10072000F0226B001024690030256600502663001B
:100730007027610090285E00B0295C00D02A590023
:10074000F02B5600102D5400302E5100502F4E002B
:1007500070304B0090314800B0324500D033420039
:10076000F0343E0010363B0030373700503833004D
:1007700070392E00903A2900B03B2300D03C1B007A
:10078000F03D1100103F0100F03F00001000C902D1
:1007900010012C014001220170011801B0010E016D
:1007A000F00104015002FA00B002F0003003E6004C
:1007B000D003DC009004D2007005C800A006BE0083
:1007C0000008B400B009AA00D00BA000600E96008B
:1007D00060118C000015820020197800C01D6E0089
:1007E000A0226400B0275A00902C5000003146002F
:1007F000E0343C0010383200903A2800603C1E0083
:10080000A03D1400803E0A00203F00006F70656E1E
:1008100000545249474745524544003A20007A5F08
:100820006D6178007A5F6D696E00795F6D61780047
:10083000795F6D696E00785F6D617800785F6D69D2
:100840006E005265706F7274696E6720656E6473B6
:10085000746F70207374617475730A00205A3A00C3
:1008600020593A0020583A00656E6473746F7073B3
:10087000206869743A2000486F6D696E6720666170
:10088000696C656400496E76616C69642065787492
:1008900072756465720A0045303A20005A3A2000A9
:1008A000593A20004D53312C4D53322C4D533320A7
:1008B00050696E730A583A20004D6963726F737401
:1008C00065707320756E617661696C61626C650A32
:1008D00000205A3A0020593A0020436F756E742068
:1008E000583A00C23100001C260000F4190000D85C
:1008F0000F0000EB080000C004000075020000407B
:1009000001000024F4D43050C38E20C2A2401782CC
:100910008B7011127A910D816CD90AA861E108C718
:10092000586607615143061E4B5D05C145A7041A71
:10093000411104093D9803713931034036DB0265EA
:10094000339102D4305402802E1D02632CEE0175C7
:100950002AC501B028A001102781018F2564012B31
:10096000244B01E0223401AC211F018D200D0180B8
:100970001FFC00841EED00971DDF00B81CD200E6AE
:100980001BC600201BBC00641AB200B219A8000AE2
:1009900019A0006A189900D117910040178B00B573
:1009A00016840031167E00B31579003A157300C71E
:1009B000146F0058146A00EE136600881363002554
:1009C000135E00C7125B006C12570015125400C171
:1009D00011510070114F0021114B00D61049008DAC
:1009E0001047004610440002104200C00F40008033
:1009F0000F3E00420F3C00060F3B00CB0E38009329
:100A00000E37005C0E3500270E3400F30D3200C1A6
:100A10000D3100900D3000600D2E00320D2D0005BF
:100A20000D2C00D90C2B00AE0C2900850C29005C84
:100A30000C2700350C27000E0C2600E80B2400C400
:100A40000B2400A00B23007D0B23005A0B2100393F
:100A50000B2100180B2000F80A1F00D90A1E00BB4A
:100A60000A1E009D0A1D00800A1D00630A1C004723
:100A70000A1B002C0A1B00110A1A00F7091A00DDD4
:100A8000091900C4091900AB091900920917007B64
:100A9000091800630917004C0916003609160020D2
:100AA0000916000A091500F5081500E0081400CC25
:100AB000081400B8081400A4081400900813007D5E
:100AC0000812006B08130058081200460812003480
:100AD000081100230811001208110001081100F08C
:100AE000071000E0071000D0071000C0071000B08A
:100AF000070F00A107100091070E0083070F007475
:100B0000070F0065070E0057070E0049070E003B50
:100B1000070D002E070E0020070D0013070D00061D
:100B2000070D00F9060C00ED060D00E0060C00D4E0
:100B3000060C00C8060C00BC060C00B0060C00A495
:100B4000060B0099060C008D060B0082060B007741
:100B5000060B006C060B0061060A0057060B004CE2
:100B6000060A0042060A0038060A002E060A002479
:100B7000060A001A060A001006090007060A00FD08
:100B8000050900F4050900EB050900E2050900D993
:100B9000050900D0050900C7050900BE050900B513
:100BA000050800AD050800A50509009C050800948E
:100BB0000508008C050800840508007C0508007401
:100BC0000508006C050700650508005D050700566F
:100BD0000508004E050700470507004005080038D6
:100BE000050700310507002A050700230507001C3B
:100BF000050600160507000F050700080506000298
:100C0000050700FB040600F5040700EE040600E8F3
:100C1000040600E2040700DB040600D5040600CF4A
:100C2000040600C9040600C3040600BD040600B79C
:100C3000040600B1040500AC040600A6040600A0EA
:100C40000405009B04060095040500900406008A34
:100C500004050085040500800406007A040500757B
:100C6000040500700405006B0405006604050061BE
:100C70000405005C04050057040500520405004DFE
:100C800004050048040500430405003E0404003A3E
:100C900004050035040500300404002C0405002779
:100CA000040400230405001E0404001A04040016B2
:100CB000040500110404000D0404000904050004E7
:100CC00004040000040400FC030400F8030400F41E
:100CD000030400F0030400EC030400E8030400E450
:100CE000030400E0030400DC030400D8030400D480
:100CF000030400D0030400CC030400C8030300C5B0
:100D000003030024F404D9201BC40C5C0E9804C413
:100D1000095F0265077101F405F900FB04B300489F
:100D2000048700C10369005803550003034500BE52
:100D3000023A008402310053022A002902250004ED
:100D4000022000E4011C00C8011900AF011700983F
:100D500001140084011300710110006101100051A1
:100D6000010E0043010D0036010B002B010B00208A
:100D7000010B00150109000C01090003010800FB2B
:100D8000000800F3000800EB000700E4000600DEA6
:100D9000000600D8000600D2000600CC000500C7FF
:100DA000000500C2000500BD000400B9000400B544
:100DB000000400B1000400AD000400A9000400A577
:100DC000000300A20003009F0004009B00030098A2
:100DD0000003009500020093000300900003008DC3
:100DE0000002008B000300880002008600020084DD
:100DF000000300810002007F0002007D0002007BF2
:100E00000002007900020077000100760002007401
:100E100000020072000100710002006F0002006D0C
:100E20000001006C0002006A000100690002006716
:100E3000000100660001006500010064000200621C
:100E400000010061000100600001005F0002005D20
:100E50000001005C0001005B0001005A0001005924
:100E60000001005800010057000100560001005524
:100E70000001005400010053000000530001005223
:100E800000010051000100500001004F0001004E20
:100E90000000004E0001004D0001004C0001004B1D
:100EA0000000004B0001004A000100490001004819
:100EB0000000004800010047000100460000004615
:100EC000000100450000004500010044000100430E
:100ED0000000004300010042000000420001004108
:100EE00000000041000100400001003F0000003F01
:100EF0000001003E0000003E0001003D0000003DFA
:100F00000001003C0000003C0000003C0001003BF0
:100F10000000003B0001003A0000003A00010039E7
:100F200000000039000100380000003800000038DF
:100F300000010037000000370001003600000036D5
:100F400000000036000100350000003500000035CB
:100F500000010034000000340000003400010033C0
:100F600000000033000000330001003200000032B6
:100F700000000032000100310000003100000031AB
:100F80000001003000000030000000300001002FA0
:100F90000000002F0000002F0000002F0001002E95
:100FA0000000002E0000002E0001002D0000002D8A
:100FB0000000002D0000002D0001002C0000002C7E
:100FC0000000002C0000002C0001002B0000002B72
:100FD0000000002B0000002B0001002A0000002A66
:100FE0000000002A0000002A00010029000000295A
:100FF000000000290000002900000029000100284D
:101000000000002800000028000000280000002840
:101010000001002700000027000000270000002733
:101020000000002700010026000000260000002626
:101030000000002600000026000100250000002519
:10104000000000250000002500000025000000250C
:1010500000010024000000240000002400000024FF
:1010600000000024000100230000002300000023F2
:1010700000000023000000230000002300000023E4
:1010800000010022000000220000002200000022D7
:1010900000000022000000220001002100000021C9
:1010A00000000021000000210000002100000021BC
:1010B00000000021000100200000002000000020AE
:1010C00000000020000000200000002000000020A0
:1010D000000000200001001F0000001F0000001F92
:1010E0000000001F0000001F0000001F0000001F84
:1010F0000001001E0000001E0000001E0000001E77
:101100000000003A0A0020286D6D290020530020BD
:101110005A0020590020580020204D3432352046F6
:10112000004261636B6C61736820636F6D70656E04
:10113000736174696F6E3A0A00204500205A0020DE
:10114000204D393037205800537465707065722017
:101150006D6F746F722063757272656E74733A0A84
:101160000020204D393030204B004C696E65617293
:1011700020416476616E63653A0A0020204D38355F
:1011800031205A005A2D50726F6265204F66667387
:1011900065740020440020490020204D3330342065
:1011A000500020440020490020204D333031205091
:1011B000005049442073657474696E67733A0A007D
:1011C00020204D3432302053004175746F20426529
:1011D00064204C6576656C696E673A0A00204500AC
:1011E000205A00205900205800205400205300208D
:1011F000204D32303520420020453C6D61785F65DE
:101200005F6A65726B3E0020583C6D61785F785F65
:101210006A65726B3E20593C6D61785F795F6A65E3
:10122000726B3E205A3C6D61785F7A5F6A65726BC3
:101230003E00416476616E6365643A20423C6D69AC
:101240006E5F7365676D656E745F74696D655F75FC
:10125000733E20533C6D696E5F66656564726174B0
:10126000653E20543C6D696E5F74726176656C5F9B
:1012700066656564726174653E002054002052000A
:1012800020204D323034205000416363656C65721C
:101290006174696F6E2028756E6974732F733229BB
:1012A0003A20503C7072696E745F616363656C3E96
:1012B00020523C726574726163745F616363656C34
:1012C0003E20543C74726176656C5F616363656C4B
:1012D0003E0A00204500205A0020590020204D32AF
:1012E00030312058004D6178696D756D2041636320
:1012F000656C65726174696F6E2028756E697473B0
:101300002F7332293A0A00204500205A0020590044
:1013100020204D3230332058004D6178696D756D55
:10132000206665656472617465732028756E6974E2
:10133000732F73293A0A00537465707320706572B5
:1013400020756E69743A0A0020204732312020202F
:10135000203B20556E69747320696E206D6D0048C6
:10136000617264636F6465642044656661756C7462
:101370002053657474696E6773204C6F6164656493
:101380000A00282300002823000064000000E8036E
:10139000000000009643000096430000004100005A
:1013A00020420000C9420000C9420000C844004079
:1013B0005044290A002062797465733B206372638C
:1013C00020002073746F7265642073657474696E95
:1013D00067732072657472696576656420280020E1
:1013E0002863616C63756C6174656429210A00204F
:1013F000213D2000454550524F4D20435243206D22
:1014000069736D61746368202D202873746F726531
:10141000642920002053697A653A2000496E64658A
:10142000783A2000204D61726C696E3D5636352940
:101430000A00454550524F4D2076657273696F6EB4
:10144000206D69736D617463682028454550524F63
:101450004D3D00290A002062797465733B20637258
:1014600063200053657474696E67732053746F72E0
:101470006564202800454550524F4D2064617461D9
:1014800073697A65206572726F722E0A0050726FEE
:1014900062696E67206661696C65640A00576172F3
:1014A0006E696E673A20486F6D696E672042756D90
:1014B000702044697669736F72203C20310A000203
:1014C00002042066697273740A00486F6D6520001B
:1014D00020746F6F206C6F6E6720657874727573FF
:1014E000696F6E2070726576656E7465640A00209F
:1014F000636F6C6420657874727573696F6E2070A9
:10150000726576656E7465640A0020453A00205A5B
:101510003A0020593A00583A000000F0410000F02B
:101520004100000041FF01010000A0400000A04078
:101530000000004000002543000045430000214317
:10154000000040C000003E4300001F430000224353
:1015500000003E4300001F43000040C00000E0C008
:10156000000000C020746F6F206C6F6E672065787C
:1015700074727573696F6E2070726576656E7465CE
:10158000640A0020636F6C642065787472757369F7
:101590006F6E2070726576656E7465640A006275A0
:1015A00073793A2070617573656420666F72206983
:1015B0006E7075740A00627573793A207061757384
:1015C000656420666F7220757365720A00627573B8
:1015D000793A2070726F63657373696E670A004DA4
:1015E0003131372050726F626520737563636573A4
:1015F0007366756C0A0020496E76616C69642065BB
:10160000787472756465722000205A3A200020595F
:101610003A200042656420583A200050726F62659B
:10162000205A204F66667365743A20003F5A206F37
:101630007574206F662072616E676520282D3220D8
:10164000746F2035290A00220A00556E6B6E6F7781
:101650006E20636F6D6D616E643A202200454550C7
:10166000524F4D204F4B0A004543484F00494E46CC
:101670004F004552524F52530044525952554E005A
:10168000434F4D4D554E49434154494F4E006F66AF
:10169000660068166D167216791680164445425516
:1016A000473A00205A00205900580020204D617808
:1016B0003A2000205A00205900580020204D696E21
:1016C0003A2000536F667420656E6473746F707394
:1016D0003A20002569730025696D2025697300256E
:1016E00069682025696D20256973002569642025B6
:1016F00069682025696D2025697300256979202591
:101700006964202569682025696D2025697300506A
:1017100072696E742074696D653A20004D31313301
:101720002053002F2F20004361703A004348414D61
:101730004245525F54454D50455241545552450023
:101740004D4F54494F4E5F4D4F444553005448450B
:10175000524D414C5F50524F54454354494F4E00F7
:101760004155544F5245504F52545F53445F535468
:10177000415455530050524F4D50545F53555050A3
:101780004F525400454D455247454E43595F5041D5
:101790005253455200434153455F4C494748545FBB
:1017A0004252494748544E45535300544F47474CC3
:1017B000455F4C494748545300534F465457415294
:1017C000455F504F574552004255494C445F504584
:1017D0005243454E54004C4556454C494E475F4494
:1017E000415441005A5F50524F4245004155544FB9
:1017F0004C4556454C005052494E545F4A4F4200AA
:1018000050524F4752455353004155544F52455043
:101810004F52545F54454D5000564F4C554D455412
:1018200052494300454550524F4D0042494E4152A6
:10183000595F46494C455F5452414E53464552000C
:1018400053455249414C5F584F4E5F584F464600F2
:101850004649524D574152455F4E414D453A4D61C3
:10186000726C696E20204649524D574152455F5671
:10187000455253494F4E3A322E302E302E313132AE
:101880002045585452554445525F545950453A5397
:10189000696E676C65457874727564657220534F24
:1018A000555243455F434F44455F55524C3A687427
:1018B0007470733A2F2F636F64652E616C65706866
:1018C0006F626A656374732E636F6D2F64696666F9
:1018D0007573696F6E2F4D41524C494E2050524FD7
:1018E000544F434F4C5F56455253494F4E3A312E59
:1018F00030204D414348494E455F545950453A4C7C
:10190000756C7A426F74204D696E69204558545247
:10191000554445525F434F554E543A312055554931
:10192000443A33353134383762362D636139612DAD
:10193000346331612D383736352D643636386231AF
:101940006461363538350A0020284E6F7420796579
:1019500074206D656173757265642900202041767D
:101960006572616765206D6561737572656420627B
:1019700061636B6C61736820286D6D293A002020CB
:10198000536D6F6F7468696E6720286D6D293A20FA
:101990002020202020202020202020202020202047
:1019A000530020204261636B6C617368204469734B
:1019B00074616E636520286D6D293A2020202020F7
:1019C00020202000202846312E30203D2066756CD6
:1019D0006C2C2046302E30203D206E6F6E65290A1B
:1019E000002020436F7272656374696F6E20416DD1
:1019F0006F756E742F466164652D6F75743A202083
:101A000020202046006163746976653A0A00696E99
:101A1000004261636B6C61736820436F727265632F
:101A200074696F6E2000205A0020506F73697469CA
:101A30006F6E616C204572726F723A0A004E6F7A57
:101A40007A6C6520546970204F7574657220446902
:101A50006D656E73696F6E733A0A002020546F7063
:101A60003A2000202046726F6E743A200020204CED
:101A70006566743A20004261636B6C6173683A0A70
:101A800000205A0043656E7465723A0A00202046B1
:101A9000726F6E743A200020204C6566743A200004
:101AA0002020546F703A200053696465733A0A002D
:101AB000426564204C6576656C696E6720004661FE
:101AC000696C656420746F20656E61626C6520428C
:101AD0006564204C6576656C696E670A00426564D2
:101AE000204C6576656C20436F7272656374696F14
:101AF0006E204D61747269783A000A0A426564206A
:101B00004C6576656C20436F7272656374696F6EA5
:101B1000204D61747269783A00202B000A436F727D
:101B2000726563746564204265642048656967680E
:101B3000742076732E2042656420546F706F6C6F32
:101B400067793A0A00202B000A42656420486569DB
:101B500067687420546F706F6772617068793A0AB1
:101B60002020202B2D2D2D204241434B202D2D2B8D
:101B70000A2020207C20202020202020202020201F
:101B80007C0A204C207C20202020282B292020206B
:101B9000207C20520A2045207C202020202020204C
:101BA000202020207C20490A2046207C20282D2926
:101BB000204E20282B29207C20470A2054207C20DE
:101BC000202020202020202020207C20480A2020A7
:101BD000207C20202020282D29202020207C2054FB
:101BE0000A2020207C2020202020202020202020AF
:101BF0007C0A2020204F2D2D2046524F4E54202D60
:101C00002D2B0A2028302C30290A003474682070CB
:101C1000726F626520706F696E742C2064697374D2
:101C2000616E63652066726F6D20706C616E653ADF
:101C30002000202844525952554E2900473239205D
:101C40004175746F20426564204C6576656C696EE1
:101C500067003F20284C2C522C462C4229206F75BF
:101C600074206F6620626F756E64732E0A003F5099
:101C7000726F626520706F696E7473202859292015
:101C8000697320696D706C61757369626C65202879
:101C9000322D32292E0A003F50726F626520706F1C
:101CA000696E74732028582920697320696D706CDF
:101CB00061757369626C652028322D32292E0A0005
:101CC0003F2856296572626F7365206C6576656C76
:101CD00020697320696D706C61757369626C652031
:101CE00028302D34292E0A00416476616E63652008
:101CF0004B3D003F4B2076616C7565206F757420FD
:101D00006F662072616E67652028302D3130292E74
:101D10000A004D31313720486F7420456E642048E9
:101D2000656174696E672E2E2E0A4D313034205352
:101D30003137302054300A473238204F310A47318A
:101D400020593235205A31302046353030300A4D56
:101D5000313137205265776970696E67206E6F7A0E
:101D60007A6C650A54300A4731205834352059318D
:101D700037322046353030300A4D3130392052313B
:101D800037302054300A4731205A310A4731205821
:101D9000343520593137322046343030300A47311B
:101DA0002058343520593137322046343030300A0B
:101DB00047312058343520593137322046343030BD
:101DC000300A4731205834352059313732204634D3
:101DD0003030300A473120583435205931373220DD
:101DE00046343030300A47312058343520593137A5
:101DF000322046343030300A4731205834352059AB
:101E00003137322046343030300A473120583435AB
:101E100020593137322046343030300A473120588B
:101E2000343520593137322046343030300A47318A
:101E30002058343520593137322046343030300A7A
:101E4000473120583435205931373220463430302C
:101E5000300A473120583435205931373220463442
:101E60003030300A4731205A31350A4D3130362072
:101E700053323535200A47302058302059300A4D2A
:101E800031303920523136302054300A4D3130371C
:101E90000A0020466C6F773A200020643A002069DF
:101EA0003A0020703A00204500205A0020590020B6
:101EB0004D393220580043290A0061626C65642064
:101EC000286D696E2074656D70200064697300650B
:101ED0006E00436F6C64206578747275646573205E
:101EE0006172652000205400205200416363656CDC
:101EF00065726174696F6E3A205000496E76616C4C
:101F000069642065787472756465720A0020643AA9
:101F10000020693A0020703A0047322F4733206290
:101F2000616420706172616D65746572730A00503E
:101F300072696E7465722073746F7070656420646A
:101F4000756520746F206572726F72732E204669FA
:101F50007820746865206572726F7220616E6420EB
:101F6000757365204D39393920746F20726573742B
:101F70006172742E202854656D706572617475727B
:101F8000652069732072657365742E205365742013
:101F9000697420616674657220726573746172740D
:101FA000696E67290A004E6F20436865636B73751D
:101FB0006D2077697468206C696E65206E756D623E
:101FC00065722C204C617374204C696E653A200058
:101FD000636865636B73756D206D69736D617463A0
:101FE000682C204C617374204C696E653A20004C5B
:101FF000696E65204E756D626572206973206E6F23
:1020000074204C617374204C696E65204E756D624E
:1020100065722B312C204C617374204C696E653ACB
:1020200020004D31313000526573656E643A2000F6
:102030002042002050006F6B00220A00656E71750F
:10204000657565696E6720220050494420417574AA
:102050006F74756E65206661696C656421204261EC
:1020600064206578747275646572206E756D626542
:10207000720A006F6B002020506C616E6E657242B8
:10208000756666657242797465733A2000204672FF
:102090006565204D656D6F72793A2000436F6D70F4
:1020A000696C65643A2041707220323520323031DB
:1020B000390A00207C20417574686F723A202841EB
:1020C0006C657068204F626A6563747320496E6343
:1020D0002E2C204C756C7A426F7420476974205204
:1020E00065706F7369746F7279290A0000204C6102
:1020F000737420557064617465643A2000322E3028
:102100002E302E3131320A004D61726C696E002022
:10211000536F6674776172652052657365740A0047
:10212000205761746368646F672052657365740A31
:10213000002042726F776E206F7574205265736550
:10214000740A002045787465726E616C2052657364
:1021500065740A00506F77657255700A0073746178
:1021600072740A005072696E7465722068616C74D2
:1021700065642E206B696C6C28292063616C6C652A
:1021800064210A004B494C4C2063617573656420DF
:10219000627920746F6F206D75636820696E61636A
:1021A000746976652074696D65202D20637572727F
:1021B000656E7420636F6D6D616E643A20004D3101
:1021C00032310A4730205A31300A473238205830ED
:1021D0002059300A4731320A4D31303920523136D8
:1021E000300A4D3131372050726F62696E6720625C
:1021F00065640070726F62655F7265776970650013
:1022000050726F62696E67206661696C6564004D2B
:1022100031313720426564206C6576656C696E6784
:10222000206661696C65642E0A4730205A31300A95
:1022300047302045300A4D3330302050323520535E
:102240003838300A4D333030205035302053300A82
:102250004D3330302050323520533838300A4D332A
:102260003030205035302053300A4D33303020503C
:10227000323520533838300A4734205331007072D9
:102280006F62655F6661696C65640050726F74654A
:10229000637465642050696E0A0025301D0C1E2889
:1022A0002924311C0B184527232F1B0A17444322CE
:1022B0002B1A4142043803FF3604080606000100C9
:1022C000B71D9132E26D7E9311241FBECFEFD1E294
:1022D000DEBFCDBF00E00CBF13E0A0E0B2E0EEE156
:1022E000F2E701E00BBF02C007900D92AE39B107D3
:1022F000D9F72EE0AEE9B3E001C01D92A93EB207C6
:10230000E1F711E1C4E6D1E100E006C0219701093F
:10231000802FFE010E94A4B1C036D10780E00807DB
:10232000A9F766D40C940DB90C9400001F920F927B
:102330000FB60F9211242F933F938F939F93AF93D8
:10234000BF9380919F039091A003A091A103B091AE
:10235000A20330919E0323E0230F2D3720F4019632
:10236000A11DB11D05C026E8230F0296A11DB11DB8
:1023700020939E0380939F039093A003A093A103B7
:10238000B093A2038091A3039091A403A091A5030D
:10239000B091A6030196A11DB11D8093A303909354
:1023A000A403A093A503B093A603BF91AF919F91FF
:1023B0008F913F912F910F900FBE0F901F90189506
:1023C0002FB7F89460919F037091A0038091A103AF
:1023D0009091A2032FBF08953FB7F8948091A30373
:1023E0009091A403A091A503B091A60326B5A89B44
:1023F00005C02F3F19F00196A11DB11D3FBFBA2F97
:10240000A92F982F8827820F911DA11DB11DBC01F6
:10241000CD0142E0660F771F881F991F4A95D1F7BB
:1024200008958F929F92AF92BF92CF92DF92EF92D8
:10243000FF926B017C01D0DF4B015C01C114D10420
:10244000E104F104F1F091D3C7DFDC01CB0188197D
:102450009909AA09BB09883E9340A105B10570F30B
:1024600021E0C21AD108E108F10888EE880E83E065
:10247000981EA11CB11CC114D104E104F10421F780
:10248000DDCFFF90EF90DF90CF90BF90AF909F9007
:102490008F900895789484B5826084BD84B58160FE
:1024A00084BD85B5826085BD85B5816085BDEEE65C
:1024B000F0E0808181608083E1E8F0E0108280813B
:1024C00082608083808181608083E0E8F0E08081A9
:1024D00081608083E1EBF0E0808184608083E0EBC9
:1024E000F0E0808181608083E1E9F0E080818260BA
:1024F0008083808181608083E0E9F0E08081816079
:102500008083E1EAF0E08081826080838081816065
:102510008083E0EAF0E0808181608083E1E2F1E0A5
:10252000808182608083808181608083E0E2F1E04D
:10253000808181608083EAE7F0E08081846080832D
:1025400080818260808380818160808380818068D7
:1025500080831092C10008951F93CF93DF93182FAB
:10256000EB0161E016D1209711F460E004C0CF3F89
:10257000D10531F461E0812FDF91CF911F9145C1E9
:10258000E12FF0E0ED51FE4FE4914E2F50E0FA01C3
:102590003197E231F10508F09DC08827EE58FF4FD2
:1025A0008F4F0C94A4B184B5806884BDC7BD97C01B
:1025B00084B5806284BDC8BD92C08091800080686F
:1025C00080938000D0938900C093880088C0809158
:1025D0008000806280938000D0938B00C0938A003B
:1025E0007EC080918000886080938000D0938D00B1
:1025F000C0938C0074C08091B00080688093B0005C
:10260000C093B3006CC08091B00080628093B00032
:10261000C093B40064C08091900080688093900063
:10262000D0939900C09398005AC080919000806226
:1026300080939000D0939B00C0939A0050C08091EB
:102640009000886080939000D0939D00C0939C0080
:1026500046C08091A00080688093A0008091A00077
:102660008F7B8093A000D093A900C093A80037C0AF
:102670008091A00080628093A000D093AB00C093B3
:10268000AA002DC08091A00088608093A000D09304
:10269000AD00C093AC0023C080912001806880937E
:1026A0002001D0932901C093280119C080912001F5
:1026B000806280932001D0932B01C0932A010FC028
:1026C00080912001886080932001D0932D01C093D8
:1026D0002C0105C0C038D1050CF04CCF46CFDF919E
:1026E000CF911F91089590E0FC013197E231F105FF
:1026F00008F04EC08827EC57FF4F8F4F0C94A4B1C1
:10270000809180008F7703C0809180008F7D8093BF
:102710008000089580918000877FF9CF84B58F77FE
:1027200002C084B58F7D84BD08958091B0008F77FD
:1027300003C08091B0008F7D8093B0000895809198
:1027400090008F7707C0809190008F7D03C08091AB
:102750009000877F8093900008958091A0008F77EC
:1027600007C08091A0008F7D03C08091A000877F6B
:102770008093A0000895809120018F7707C08091F9
:1027800020018F7D03C080912001877F80932001ED
:102790000895CF93DF9390E0FC01E75DFD4F249116
:1027A000FC01E159FD4F8491882361F190E0880F8D
:1027B000991FFC01E751FD4FC591D491FC01E153F4
:1027C000FD4FA591B491611109C09FB7F89488811C
:1027D000209582238883EC912E230BC0623061F414
:1027E0009FB7F8943881822F809583238883EC915A
:1027F0002E2B2C939FBF06C08FB7F894E8812E2B09
:1028000028838FBFDF91CF9108951F93CF93DF93DC
:10281000282F30E0F901ED51FE4F8491F901E75D79
:10282000FD4FD491F901E159FD4FC491CC23C1F082
:10283000162F811158DFEC2FF0E0EE0FFF1FE15350
:10284000FD4FA591B4918FB7F894111105C09C91DB
:10285000ED2FE095E92302C0EC91ED2BEC938FBFB7
:10286000DF91CF911F910895CF93DF93282F30E010
:10287000F901ED51FE4F8491F901E75DFD4FD491CF
:10288000F901E159FD4FC491CC2389F081112BDF6F
:10289000EC2FF0E0EE0FFF1FEB54FD4FA591B4912C
:1028A000EC91ED2381E090E021F480E002C080E033
:1028B00090E0DF91CF91089508951F920F920FB687
:1028C0000F9211240BB60F922F933F934F935F9368
:1028D0006F937F938F939F93AF93BF93EF93FF93E8
:1028E000E0910402F09105021995FF91EF91BF91DB
:1028F000AF919F918F917F916F915F914F913F9198
:102900002F910F900BBE0F900FBE0F901F90189538
:102910001F920F920FB60F9211240BB60F922F93A6
:102920003F934F935F936F937F938F939F93AF9357
:10293000BF93EF93FF93E0910602F0910702199580
:10294000FF91EF91BF91AF919F918F917F916F9187
:102950005F914F913F912F910F900BBE0F900FBE43
:102960000F901F9018951F920F920FB60F9211247F
:102970000BB60F922F933F934F935F936F937F9379
:102980008F939F93AF93BF93EF93FF93E0910802D0
:10299000F09109021995FF91EF91BF91AF919F912D
:1029A0008F917F916F915F914F913F912F910F90F8
:1029B0000BBE0F900FBE0F901F9018951F920F9295
:1029C0000FB60F9211240BB60F922F933F934F9394
:1029D0005F936F937F938F939F93AF93BF93EF9387
:1029E000FF93E0910A02F0910B021995FF91EF918C
:1029F000BF91AF919F918F917F916F915F914F9117
:102A00003F912F910F900BBE0F900FBE0F901F9014
:102A100018951F920F920FB60F9211240BB60F92BA
:102A20002F933F934F935F936F937F938F939F93D6
:102A3000AF93BF93EF93FF93E0910002F0910102F7
:102A40001995FF91EF91BF91AF919F918F917F91D8
:102A50006F915F914F913F912F910F900BBE0F900F
:102A60000FBE0F901F9018951F920F920FB60F92E6
:102A700011240BB60F922F933F934F935F936F9355
:102A80007F938F939F93AF93BF93EF93FF93E091C7
:102A90000202F09103021995FF91EF91BF91AF915E
:102AA0009F918F917F916F915F914F913F912F9166
:102AB0000F900BBE0F900FBE0F901F9018951F9296
:102AC0000F920FB60F9211240BB60F922F933F93D4
:102AD0004F935F936F937F938F939F93AF93BF9326
:102AE000EF93FF93E0910C02F0910D021995FF9185
:102AF000EF91BF91AF919F918F917F916F915F9176
:102B00004F913F912F910F900BBE0F900FBE0F90E2
:102B10001F9018951F920F920FB60F9211240BB6AB
:102B20000F922F933F934F935F936F937F938F9366
:102B30009F93AF93BF93EF93FF93E0910E02F091B9
:102B40000F021995FF91EF91BF91AF919F918F91D6
:102B50007F916F915F914F913F912F910F900BBE9D
:102B60000F900FBE0F901F90189508954F925F928F
:102B70006F927F92AF92BF92CF92DF92EF92FF92CD
:102B80000F931F93CF93DF93CDB7DEB729013A019F
:102B90009B01AC0124193509460957098A899B898B
:102BA000AC89BD89BC01CD016A197B098C099D09DD
:102BB0000E9430B1A8019701241935094609570927
:102BC0000E9488B1CA01B9016A0D7B1D8C1D9D1D33
:102BD000DF91CF911F910F91FF90EF90DF90CF90F9
:102BE000BF90AF907F906F905F904F900895089541
:102BF00051DCFDDF0E94C3ACC0E0D0E00E9442ADDA
:102C00002097E1F30E940000F9CFCF93C82F0E94D4
:102C1000F332CC2349F024982C9A65E070E080E0F0
:102C200090E0FFDB149A03C0249A2C981498CF915B
:102C3000089580E0EACFCF92DF92EF92FF926B018E
:102C40007C0183E3C816D104E104F10468F082E357
:102C5000C81AD108E108F10862E370E080E090E072
:102C6000E0DB0E944727EDCFC701B601DADBFF901A
:102C7000EF90DF90CF900C944727DC01FB01460FCB
:102C8000571FE417F507C1F081912D913C911197E1
:102C9000382798E0B901660F771F37FF06C09B0100
:102CA00081E2282780E1382701C09B01915091F7EC
:102CB00011963C932E93E5CF0895CF93DF93FC01BB
:102CC0008491EF012196882319F061D5FE01F8CF98
:102CD000DF91CF9108958AE093E0EFCF80E193E018
:102CE000ECCF0F931F93CF93DF931F921F92CDB71B
:102CF000DEB769837A83E1DF6981062F7A81172F36
:102D0000F80181918F01882311F041D5F9CF0F90FF
:102D10000F90DF91CF911F910F910895CF93DF9383
:102D2000EB01CBDF6AE070E0CE01DF91CF9122C6EC
:102D3000CF92DF92EF92FF926A017B01BEDF4AE001
:102D400050E0C701B601FF90EF90DF90CF9001C631
:102D5000CF92DF92EF92FF926A017B01AEDF42E0F9
:102D600050E0C701B601FF90EF90DF90CF908DC685
:102D7000CF92DF92EF92FF926A017B019EDF42E0E9
:102D800050E0C701B601FF90EF90DF90CF907DC675
:102D9000CF93DF93EB0191DF6AE070E0CE01DF912A
:102DA000CF91FDC5CF92DF92EF92FF926A017B0136
:102DB00084DF4AE050E0C701B601FF90EF90DF905A
:102DC000CF90E7C5811103C083E093E002C087E0A4
:102DD00093E073CFF7DF8AE0DAC4CF93DF931F92DB
:102DE0001F92CDB7DEB72091E30E3091E40ECE01F5
:102DF00001962115310519F4895E9E4002C0821B9F
:102E0000930B9A83898389819A810F900F90DF9128
:102E1000CF91089581E0089581E008958F929F9267
:102E2000AF92BF92CF92DF92EF92FF920F931F93D8
:102E3000CF93DF931F921F92CDB7DEB76C0159017C
:102E40008B017B01E40EF51E0E151F0561F1F601E5
:102E500080809180F80161918F016983C4016A8348
:102E60000E94F7B86A81681779F0C4010E94FFB820
:102E7000C4010E94F7B89981891731F02CDF87E1EE
:102E800093E01BDF81E010C041E050E0BE016F5FC6
:102E90007F4FC501F2DEF601408151814F5F5F4FE8
:102EA00051834083D1CF80E00F900F90DF91CF917D
:102EB0001F910F91FF90EF90DF90CF90BF90AF9058
:102EC0009F908F9008958F929F92AF92BF92CF92D2
:102ED000DF92EF92FF920F93CF93DF931F92CDB7C4
:102EE000DEB75C016B017A014901F50180819181B6
:102EF0000E94F7B88983002311F0F601808341E036
:102F000050E0BE016F5F7F4FC401B7DEF501408125
:102F100051814F5F5F4F51834083FFEFCF1ADF0A2C
:102F200081E0E81AF10809F780E00F90DF91CF9176
:102F30000F91FF90EF90DF90CF90BF90AF909F9058
:102F40008F900895CF93DF93CDB7DEB760970FB61C
:102F5000F894DEBF0FBECDBF9C01E62F660FFF0BBE
:102F6000ED51FE4FE4918E2F90E0FC013797EC304D
:102F7000F10508F0B5C08827EA56FF4F8F4F0C9433
:102F8000A4B191E001C090E080E1FE013196DF0143
:102F9000482F1D924A95E9F740EB50E05A83498348
:102FA00041EB50E05C834B8343EB50E058874F8309
:102FB00044EB50E05A87498742E04F87988B98C08E
:102FC00081E001C080E08F5F01C080E040E950E017
:102FD000D90111965C934E9341E950E013965C93AE
:102FE0004E93129742E950E015965C934E931497D6
:102FF00048E950E017965C934E9316974AE950E0E3
:1030000019965C934E9318974CE950E01B965C938D
:103010004E931A9746E950E01D965C934E931C9789
:1030200093E058C081E001C080E08F5F01C080E084
:1030300040EA50E0F9015183408341EA50E0538374
:10304000428342EA50E05583448348EA50E0578384
:1030500046834AEA50E0518740874CEA50E0538764
:10306000428746EA50E05587448794E096878787F1
:1030700044C081E001C080E08F5F01C080E040E299
:1030800051E0D90111965C934E9341E251E01396C1
:103090005C934E93129742E251E015965C934E93E7
:1030A000149748E251E017965C934E9316974AE2C4
:1030B00051E019965C934E9318974CE251E01B96A1
:1030C0005C934E931A9746E251E01D965C934E93A3
:1030D0001C9795E01E969C931E971F968C930DC08F
:1030E00080E1FE013196DF01482F1D924A95E9F7F4
:1030F000D90101900D928A95E1F7C90160960FB64A
:10310000F894DEBF0FBECDBFDF91CF9108952F920F
:103110003F924F925F926F927F928F929F92AF9267
:10312000BF92CF92DF92EF92FF920F931F93CF93B4
:10313000DF93CDB7DEB7AE970FB6F894DEBF0FBE04
:10314000CDBF1B01682FCE014196FCDE4B895C8907
:103150005EA34DA35F8D5AA3552309F413C15230CA
:1031600021F0CC24CA94DC2C03C0CC24CA94D12CEA
:103170002114310409F4DBC09601322F2227330FCA
:10318000330F330F40E050E060E074E284EF90E0F2
:103190000E9488B1C90101969CA38BA380E1EFE650
:1031A000F2E0DE01119601900D928A95E1F7FE01A1
:1031B0003196F8A7EFA301E011E019A2AA24AA947E
:1031C000B12C412C84E2582E84EF682E712CFAA188
:1031D000F230F1F0033009F49FC0053009F49CC0CF
:1031E000EFA1F8A582819381289E9001299E300D40
:1031F000389E300D112440E050E0C301B2010E941E
:1032000088B1C901019736952795009729F40AC01E
:103210002FEF30E08FEF90E07C01C816D90628F43C
:10322000760103C0EE24E394F12C2115310531F031
:103230004901C216D30628F4460103C088248394AA
:10324000912CEFA1F8A50280F381E02DFEA7EDA758
:10325000C70101968E9F90018F9F300D9E9F300D6C
:10326000112440E050E0C301B2010E9488B129A7B7
:103270003AA74BA75CA78DA59EA5880F991F889D8F
:103280009001899D300D989D300D112440E050E053
:10329000C301B2010E9488B18BA19CA1821993093C
:1032A00097FF03C091958195910969A57AA5621947
:1032B000730977FF03C0719561957109F901E219EE
:1032C000F309F7FF03C0F195E195F1096817790754
:1032D00074F4E617F7075CF0FAA1F230A1F449A5FF
:1032E0005AA55CA34BA309A3570113E015C0E81727
:1032F000F90794F48AA13CA32BA309A354018230BB
:1033000051F411E009C0E9A5FAA5FCA3EBA309A3B8
:1033100057011EE001C01AE00F5F4FA158A54E5F94
:103320005F4F58A74FA3083009F051CF05C011E0F7
:1033300019A2AA24AA94B12CE989FA898081912F33
:1033400093708C7F892B8083EDA1FEA12081812F3A
:1033500090E0959587959595879543E0880F991FFF
:103360004A95E1F7122F177E812B80838081887F19
:10337000C9A0C82AC082FAA1F23021F0ED8DFE8DDD
:10338000B182A082AE960FB6F894DEBF0FBECDBF5D
:10339000DF91CF911F910F91FF90EF90DF90CF9031
:1033A000BF90AF909F908F907F906F905F904F9065
:1033B0003F902F9008954F925F926F927F92AF92BD
:1033C000BF92CF92DF92EF92FF920F931F93CF9312
:1033D000DF93CDB7DEB760970FB6F894DEBF0FBEB0
:1033E000CDBF6115710511F4622F05C06417750713
:1033F000B9F461E0622760960FB6F894DEBF0FBEA5
:10340000CDBFDF91CF911F910F91FF90EF90DF9093
:10341000CF90BF90AF907F906F905F904F90F5C925
:10342000D22E8A017B01682FCE0101968BDD5F854C
:10343000E889552309F44BC0A981BA814C91F0E089
:1034400083E090E0BC016E1B7F0B660F771F2D2D74
:1034500030E02E5F3F4F062E01C0220F0A94EAF79C
:1034600001C0880F6A95EAF780958423282B2C9356
:10347000523029F0AD85BE85CD90DC9003C0CC24C0
:10348000CA94D12C3396EE0FFF1F81E090E08C0F91
:103490009D1FE80FF91FA080B180B70180E090E088
:1034A0000E94C8AE2B013C01C601B8010E943FB189
:1034B00080E090E00E94C8AE9B01AC01C301B20164
:1034C0000E9466B00E9497AEF5017183608360969A
:1034D0000FB6F894DEBF0FBECDBFDF91CF911F9125
:1034E0000F91FF90EF90DF90CF90BF90AF907F90C3
:1034F0006F905F904F90089598E288E10FB6F8942E
:10350000A895809360000FBE9093600008951F926D
:103510000F920FB60F9211240BB60F920F931F93B9
:103520002F933F934F935F936F937F938F939F93CB
:10353000AF93BF93CF93DF93EF93FF930091CD03AE
:10354000D091CC0311E01D0F1F77C091C600909160
:10355000A803492F092E000C550B660B770B4C3036
:10356000510508F046C0FA018827EE55FF4F8F4FEE
:103570000C94A4B1CD3441F0CE34B9F481E005C04F
:10358000CA3330F0CD3471F582E08093A8034AC08D
:10359000C03308F047C0C03209F444C0CD3211F541
:1035A00041C0C13329F0C43329F0C032D9F43AC044
:1035B00083E0EBCF88E0E9CFC03321F0C13391F451
:1035C00086E0E3CF84E0E1CFC83361F485E0DDCF6E
:1035D000C23341F487E0D9CFC13321F489E0D5CF9C
:1035E000C03311F08BE0D1CF8AE0CFCFCA30D1F415
:1035F00017C0CA30B9F480915704882389F09730F6
:1036000049F09A3059F0953059F410926D021092A9
:10361000E20E06C081E08093580402C00E949AAB7B
:103620001092A803101731F0ED2FF0E0E453FC4F97
:10363000C283D12FD093CC03FF91EF91DF91CF9133
:10364000BF91AF919F918F917F916F915F914F91BA
:103650003F912F911F910F910F900BBE0F900FBEB6
:103660000F901F9018951F920F920FB60F92112472
:103670000BB60F922F938F939F93EF93FF938091AD
:10368000AB032091AA03281791F0E82FF0E0E6554C
:10369000FC4F92818F5F8F719093C6008093AB0334
:1036A0009091C00090649093C000281305C0809151
:1036B000C1008F7D8093C100FF91EF919F918F9109
:1036C0002F910F900BBE0F900FBE0F901F9018956B
:1036D0009B01AC011092C000211581EE3807410515
:1036E0005105C1F08091C00082608093C00060E00D
:1036F00079E08DE390E00E9488B1CA01B901615080
:1037000071098109910922E030E040E050E00E9417
:1037100088B102C020E130E03093C5002093C4009E
:103720008091C10080618093C1008091C100886058
:103730008093C1008091C10080688093C100809116
:10374000C1008F7D8093C1001092A90308958091DC
:10375000CC039091CD03891759F0E92FF0E0E453A1
:10376000FC4F82819F5F9F779093CD0390E00895F7
:103770008FEF9FEF0895ECECF3E080818183089553
:10378000ECECF3E080819181891B8F77089591E0C3
:103790009093A9039091C10095FD04C09091C00041
:1037A00095FD40C02091AA032F5F2F710FB607FC33
:1037B00034C09091AB03291322C09091C00095FFB3
:1037C0001DC09091AB034091AA03491791F0E92FD6
:1037D000F0E0E655FC4F32819F5F9F713093C60049
:1037E0009093AB033091C00030643093C000491314
:1037F00005C09091C1009F7D9093C100DACFE09108
:10380000AA03F0E0E655FC4F82832093AA0380913F
:10381000C10080628093C10008959091AB03291389
:10382000EECFFBCF8093C6008091C0008064809370
:10383000C00008958DE0ABDF8AE0A9CFCF93DF937E
:10384000EC018991882311F0A2DFFBCFDF91CF91AA
:10385000F1CF8F929F92AF92BF92EF92FF921F9300
:10386000CF93DF93CDB7DEB7A0970FB6F894DEBF46
:103870000FBECDBF611571058105910579F110E08D
:10388000842E912CA12CB12CEE24E394F12CEC0E7F
:10389000FD1EE10EF11C17FDFA94A50194010E9492
:1038A00066B1F7016083B901CA011F5F6115710537
:1038B0008105910549F7115010F1E1E0F0E0EC0FBE
:1038C000FD1FE10FF11D17FDFA9580818A3010F080
:1038D00097E301C090E3890F5ADFEDCF80E3A09614
:1038E0000FB6F894DEBF0FBECDBFDF91CF911F9111
:1038F000FF90EF90BF90AF909F908F9048CFA09691
:103900000FB6F894DEBF0FBECDBFDF91CF911F91F0
:10391000FF90EF90BF90AF909F908F900895CF92BF
:10392000DF92EF92FF926B017C0197FF0AC08DE25C
:103930002EDFF094E094D094C094C11CD11CE11C03
:10394000F11C4AE0C701B601FF90EF90DF90CF90E5
:1039500080CF4115510511F4862F19CF4A305105FA
:1039600009F4DDCF76CFAB01682F880F770B880B7A
:10397000990BEFCFAB01BC01990F880B990BE9CFE5
:10398000AB01BC01990F880B990BE3DF53CFE1DF4B
:1039900051CF4115510511F4862FF9CE5ACFAB0105
:1039A000BC0180E090E0F5CF8F929F92AF92BF92E2
:1039B000CF92DF92EF92FF92CF936B017C01B42EF6
:1039C00020E030E0A9010E9428AE87FF06C08DE20A
:1039D000DEDEF7FAF094F7F8F094C0E060E070E013
:1039E00080E09FE3CB1541F02DEC3CEC4CEC5DE32B
:1039F0000E9466B0CF5FF6CF9B01AC01C701B60154
:103A00000E944FAD6B017C010E949CAE4B015C019A
:103A10004AE01FDFCC2379F1C501B4010E94C8AE92
:103A20009B01AC01C701B6010E944EAD6B017C0148
:103A30008EE2ADDE20E030E040E251E4C701B601A5
:103A40000E9466B04B015C010E9497AE6B01770F3C
:103A5000EE08FF08C701B60162DFC701B6010E9488
:103A6000CAAE9B01AC01C501B4010E944EAD6B0111
:103A70007C01C150F9F6CF91FF90EF90DF90CF908D
:103A8000BF90AF909F908F9008958ECFCF92DF928E
:103A9000EF92FF920F931F930E94E0110091520446
:103AA0001091530420915404309155046B017C0112
:103AB000C01AD10AE20AF30AF7FC52C08B019C013A
:103AC0000C53164F2F4F3F4F009352041093530443
:103AD0002093540430935504079B39C0069B37C08C
:103AE000059B35C02091DC04211131C0049B2FC0FF
:103AF00000914E0410914F042091500430915104D4
:103B0000011511052105310571F0DC01CB01801B88
:103B1000910BA20BB30B80569A4EA109B109B7FFC6
:103B200002C068E701C060E0609356048091020122
:103B30006111809588708093000170E086E01F918C
:103B40000F91FF90EF90DF90CF900C94AC126093A8
:103B50004E0470934F048093500490935104C8CF47
:103B60001F910F91FF90EF90DF90CF90089581E02B
:103B7000809357040895909130068917D1F00E94E0
:103B80004D5E80913006882359F04AE552E066E5A3
:103B900072E082E592E00E94105D1092300607C04C
:103BA00081E08093300682E592E00E947E5D0C9475
:103BB0002652089580E0DFDF8CE096E00C9406A7A3
:103BC0002F923F924F925F926F927F928F929F922D
:103BD000AF92BF92CF92DF92EF92FF920F931F931B
:103BE000CF93DF93CDB7DEB76B970FB6F894DEBFF8
:103BF0000FBECDBF80916504102F1827DB018D907B
:103C00009D90AD90BC9089288A288B2809F41E7F4E
:103C1000FA014081518162817381452B462B472BEC
:103C200009F41D7FD9014D915D916D917C91452BDA
:103C3000462B472B09F41B7F8127809365046091F5
:103C40008204662309F439C1FC8AEB8A70E080E0C3
:103C500090E00E94C8AE20E030E04FE753E40E94BD
:103C60002FAE69837A838B839C838091100290911D
:103C70001102A0911202B09113028D879E87AF8727
:103C8000B88BA6E7B4E0BA8BA98BFE82ED82E9E59A
:103C9000F4E0FA8FE98F81E696E09C878B87212CF0
:103CA000312CC12CD12C7601A02FB0E0BE8BAD8B76
:103CB000E12FF0E0F88FEF8B89819A81AB81BC8195
:103CC000B0588F839887A987BA87A989BA898D90B8
:103CD0009D90AD90BD90BA8BA98B20E030E0A901FA
:103CE000C501B4010E9428AE882309F4CFC00D8914
:103CF0001E89022C02C0159507950A94E2F70170FF
:103D000011278F89988D022C02C0959587950A946A
:103D1000E2F780FF35C0E98DFA8D60817181828183
:103D200093810E94CAAE2B013C010115110529F0B7
:103D3000BF81A885E985FA8504C0B981AA81EB8194
:103D4000FC81A50194016B2F7A2FCF010E9466B0F0
:103D5000AB85BC8554962D913D914D915C915797C3
:103D60000E9466B09B01AC01C301B2010E944FAD3D
:103D70000E9497AEE98DFA8D60837183828393836D
:103D8000A98DBA8D8D909D90AD90BC9081149104B9
:103D9000A104B10409F47AC020E030E0A9016D85E6
:103DA0007E858F8598890E9428AE882309F445C0B6
:103DB000D501C4018827B7FD83959927AA27BB277A
:103DC0000817190709F062C020E030E0A901C70117
:103DD000B6010E9428AE81111CC02D853E854F85FD
:103DE0005889EB89FC8965857685878590890E944D
:103DF0002FAE6B017C0120E030E040E85FE30E94E1
:103E00002BB0181634F4C12CD12C80E8E82E8FE3A7
:103E1000F82EC501B4010E94CAAE9B01AC01C701D6
:103E2000B6010E9466B00E9415AE0E9497AE611561
:103E300071058105910519F429C0C501B4018B01F3
:103E40009C0197FF07C0002711279801061B170B3D
:103E5000280B390BAD81BE8155964D905D906D90CC
:103E60007C905897040D151D261D371DFD01058BEF
:103E7000168B278B308F861A970AA80AB90AA98D44
:103E8000BA8D8D929D92AD92BC921397BFEF2B1A73
:103E90003B0AED81FE813496FE83ED83898D9A8DF8
:103EA00004969A8F898FAB85BC851496BC87AB87A7
:103EB000B3E02B16310409F008CF6B960FB6F894D7
:103EC000DEBF0FBECDBFDF91CF911F910F91FF904D
:103ED000EF90DF90CF90BF90AF909F908F907F90AA
:103EE0006F905F904F903F902F9008954F925F9208
:103EF0006F927F928F929F92AF92BF92CF92DF92FA
:103F0000EF92FF92CF93DF93CDB7DEB728970FB62E
:103F1000F894DEBF0FBECDBF809169048F3F09F4D6
:103F20005FC080905A0290905B02A0905C02B090BB
:103F30005D02412C512C80E8682E8FE3782EC090D2
:103F40005A02D0905B02E0905C02F0905D0220E0AB
:103F500030E040E05FE3C501B4010E944FAD9B013A
:103F6000AC01C701B6010E9428AE87FF1AC01C9998
:103F700018C049825A826B827C822AE037ED43EA7C
:103F80005BE3C701B6010E944FAD6D837E838F83D3
:103F90009887BE016F5F7F4FCE0105960E94BF5389
:103FA000CECFA5019401C701B6010E944EAD9B0181
:103FB000AC016091720470917304809174049091CB
:103FC00075040E944FAD60937204709373048093E4
:103FD000740490937504809169048F5F80936904E1
:103FE00028960FB6F894DEBF0FBECDBFDF91CF91FC
:103FF000FF90EF90DF90CF90BF90AF909F908F9009
:104000007F906F905F904F9008950F931F93CF9381
:10401000DF931F92CDB7DEB78C0181E493E0698313
:104020000E945D16C8010E945D166981662339F001
:104030008AE00F90DF91CF911F910F91A8CB0F9045
:10404000DF91CF911F910F91089561E088E393E094
:10405000DCCF61E081E393E0D8CFEF92FF920F9342
:104060001F93CF93DF931F92CDB7DEB78C017B01F7
:1040700080E249838CDB49814F3F11F084E501C028
:1040800082E485DB8AE383DBF801608171818281D0
:10409000938142E050E0F9DCF70140815181628177
:1040A000738183E593E00E94A81662E070E080E0EF
:1040B00090E00F90DF91CF911F910F91FF90EF90C3
:1040C0000C941112FB01DC0112964D915D916D91E2
:1040D0007C911597411551056105710599F0808115
:1040E0009181A281B381841B950BA60BB70B8095A0
:1040F0009095A095B0958827B7FD83959927AA2715
:10410000BB27089580E00895811109C0CB016F3F5E
:10411000710519F010F08FEF90E08093EF0408958F
:1041200087FF03C08091DC0407C097E18902F0019A
:104130001124E051FB4F828590E008954F925F92E9
:104140006F927F928F929F92AF92BF92CF92DF92A7
:10415000EF92FF92CF93DF9300D01F92CDB7DEB7DF
:10416000E090F804F090F9048090F4049090F50445
:10417000A090F604B090F70420ED3CEC4CE45DE335
:1041800060910305709104058091050590910605E5
:104190000E9466B02B013C012091B4043091B5041B
:1041A0004091B6045091B704C501B4010E944EADD0
:1041B0009B01AC01C301B2010E9466B02B013C011E
:1041C00023E333E343E75FE36091B0047091B1040C
:1041D0008091B2049091B3040E9466B09B01AC013F
:1041E000C301B2010E944FAD69837A838B839C83A4
:1041F0006093B0047093B1048093B2049093B304BD
:104200008092B4049092B504A092B604B092B70420
:10421000E114F104A1F0B701FF0C880B990B0E9487
:10422000CAAEA50194010E944EAD6B017C0120E055
:1042300030E040E251EC0E9428AE87FF07C081E0E9
:104240008093A704412C512C3201C1C020E030E002
:1042500040E251E4C701B6010E942BB0181654F495
:1042600081E08093A704412C512C2FE7622E23E498
:10427000722EADC08091A704882351F01092A30440
:104280001092A4041092A5041092A6041092A70400
:104290002091A3043091A4044091A5045091A60458
:1042A000C701B6010E944FAD4B015C016093A304AE
:1042B0007093A4048093A5049093A6042091FB041A
:1042C0003091FC044091FD045091FE04C701B601F9
:1042D0000E9466B02B013C016093A8047093A9046E
:1042E0008093AA049093AB042091FF0430910005C1
:1042F0004091010550910205C501B4010E9466B0CC
:104300009B01AC016093AC047093AD048093AE0448
:104310009093AF04C301B2010E944FAD29813A814D
:104320004B815C810E944EAD2B013C0120E030E0CE
:104330004FE753E40E942BB020E030E0A9011816AB
:10434000DCF4C701B6010E942BB01816B4F5A70122
:104350009601C501B4010E944EAD6093A304709311
:10436000A4048093A5049093A604412C512C9FE7AC
:10437000692E93E4792E2BC0C301B2010E9428AEAE
:1043800087FF25C020E030E0A901C701B6010E94E7
:1043900028AE87FF19C0A7019601C501B4010E948C
:1043A0004EAD6093A3047093A4048093A5049093EE
:1043B000A604412C512C32010AC0412C512C8FE70C
:1043C000682E83E4782E03C0412C512C3201C301A6
:1043D000B2010F900F900F900F90DF91CF91FF904F
:1043E000EF90DF90CF90BF90AF909F908F907F9095
:1043F0006F905F904F9008954F925F926F927F926F
:104400008F929F92AF92BF92CF92DF92EF92FF92E4
:10441000CF93DF93CDB7DEB72C970FB6F894DEBFFE
:104420000FBECDBF8091D6049091D704A091D8043F
:10443000B091D90489839A83AB83BC836091DA04F9
:104440007091DB04072E000C880B990B0E94CAAEFA
:1044500029813A814B815C810E944EAD6B017C01C8
:1044600020919F043091A0044091A1045091A20496
:104470000E944FAD4B015C0160939F047093A004B8
:104480008093A1049093A2042091DD043091DE0476
:104490004091DF045091E004C701B6010E9466B06C
:1044A0006D837E838F8398876093930470939404C5
:1044B00080939504909396042091E1043091E20456
:1044C0004091E3045091E404C501B4010E9466B038
:1044D00069877A878B879C87609397047093980489
:1044E0008093990490939A0420ED3CEC4CE45DE3B6
:1044F0006091E5047091E6048091E7049091E804EE
:104500000E9466B02B013C0120918F0430919004F1
:10451000409191045091920469817A818B819C81B0
:104520000E944EAD9B01AC01C301B2010E9466B076
:104530002B013C0123E333E343E75FE360919B04FA
:1045400070919C0480919D0490919E040E9466B09D
:104550009B01AC01C301B2010E944FAD2B013C0194
:1045600060939B0470939C0480939D0490939E049D
:1045700089819A81AB81BC8180938F049093900450
:10458000A0939104B093920429853A854B855C856C
:104590006D817E818F8198850E944FADA30192012C
:1045A0000E944EAD2B013C0120E030E04FE753E488
:1045B0000E942BB020E030E0A9011816DCF4C701FE
:1045C000B6010E942BB01816B4F5A7019601C501DB
:1045D000B4010E944EAD60939F047093A004809339
:1045E000A1049093A204412C512C9FE7692E93E4DF
:1045F000792E2BC0C301B2010E9428AE87FF25C0CF
:1046000020E030E0A901C701B6010E9428AE87FF73
:1046100019C0A7019601C501B4010E944EAD609377
:104620009F047093A0048093A1049093A204412C52
:10463000512C32010AC0412C512C8FE7682E83E4A3
:10464000782E03C0412C512C3201C301B2012C96AB
:104650000FB6F894DEBF0FBECDBFDF91CF91FF90B4
:10466000EF90DF90CF90BF90AF909F908F907F9012
:104670006F905F904F9008954F925F926F927F92EC
:104680008F929F92AF92BF92CF92DF92EF92FF9262
:104690000F931F93CF93DF933C01C62F662399F0AE
:1046A0000E946E166AE070E08C2F90E063D98BE96F
:1046B00093E00E945D1680E090E00E94DFAB60E036
:1046C00070E0CB017AC0B0E2A0E06A2F70E0AB01ED
:1046D0004B0F511D559547954A1711F04B130BC0C1
:1046E000EAE0F8E065917491072E000C880B990BB5
:1046F0000E94CAAE62C0CA010197880F991F880F35
:10470000991FFC01E457F84F059114919A01220F6B
:10471000331F220F331FF901E457F84FC591D4918D
:104720006016710614F4B42FD2CFA42FC615D70586
:104730000CF4CBCF8257984FFC01E590F490F9012F
:10474000E257F84FC590D490B7010F2C000C880B9E
:10475000990B0E94CAAE4B015C01B301601B710B47
:10476000072E000C880B990B0E94CAAE2B013C014E
:10477000B6016E197F09072E000C880B990B0E9459
:10478000CAAE9B01AC01C301B2010E9466B06B01CD
:104790007C01C01BD10BBE01DD0F880B990B0E9461
:1047A000CAAE9B01AC01C701B6010E942FAE9B01AE
:1047B000AC01C501B4010E944FADDF91CF911F91B3
:1047C0000F91FF90EF90DF90CF90BF90AF909F90B0
:1047D0008F907F906F905F904F9008954F925F926F
:1047E0006F927F928F929F92AF92BF92CF92DF9201
:1047F000EF92FF920F931F93CF93DF933C01BAE3A5
:10480000A0E06A2F70E0AB014B0F511D5595479505
:104810004A1711F04B130BC0EAE8F7E06591749169
:10482000072E000C880B990B0E94CAAE62C0CA0109
:104830000197880F991F880F991FFC01EC55F94FBC
:10484000059114919A01220F331F220F331FF90192
:10485000EC55F94FC591D4916016710614F4B42F3C
:10486000D2CFA42FC615D7050CF4CBCF8A55994FBC
:10487000FC01E590F490F901EA55F94FC590D49008
:10488000B7010F2C000C880B990B0E94CAAE4B018C
:104890005C01B301601B710B072E000C880B990B98
:1048A0000E94CAAE2B013C01B6016E197F09072E8A
:1048B000000C880B990B0E94CAAE9B01AC01C3018E
:1048C000B2010E9466B06B017C01C01BD10BBE011E
:1048D000DD0F880B990B0E94CAAE9B01AC01C7018A
:1048E000B6010E942FAE9B01AC01C501B4010E942C
:1048F0004FADDF91CF911F910F91FF90EF90DF901F
:10490000CF90BF90AF909F908F907F906F905F906F
:104910004F900895CF93DF93C0EFD4E060E08A8199
:104920009B81AADE6C837D838E839F83C2EDD4E05E
:104930008A819B8153DF6C837D838E839F83A895BF
:104940001092C804DF91CF9108956D9A7598809167
:104950000101806180930101809102018071809347
:104960000001809101018860809301018091020122
:104970008870809300019D9AA598809101018062C2
:10498000809301016AE770E088E00E9487188091B7
:1049900001018860809301016AE770E086E00E946F
:1049A000871887ED80937A0010927E0010927D0028
:1049B00080917E00816080937E0080917E00846083
:1049C00080937E0080E888BD80916E008460809333
:1049D0006E006AEF70E080E090E00E94111285E0C6
:1049E00090E090931C0280931B0260E0809117027C
:1049F0009091180241DE20E030E040EA50E40E944D
:104A000028AE87FF0AC08091170290911802409744
:104A10009093180280931702E8CF81E391E090937E
:104A20001E0280931D0260E080911702909118028F
:104A300023DE20E030E848E953E40E942BB018164A
:104A400054F48091190290911A02409690931A02A0
:104A500080931902E8CF8091210290912202BEDE5C
:104A600020E030E040EA50E40E9428AE87FF0AC010
:104A7000809121029091220240979093220280938C
:104A80002102E9CF8091D0049091D104A7DE20E0EB
:104A900030E046E153E40E942BB0181654F48091A4
:104AA000210290912202409690932202809321024B
:104AB000E9CF0895CF92DF92EF92FF928091F804B0
:104AC0009091F9040097B9F0C090F404D090F504E7
:104AD000E090F604F090F7040D97BC01990F880B55
:104AE000990B0E94CAAE9B01AC01C701B6010E949E
:104AF00028AE87FD09C01092EB041092EC041092CE
:104B0000ED041092EE041EC020E030E040E050E4DE
:104B1000C701B6010E944FAD0E949CAE7093EA049B
:104B20006093E9040E94E011DC01CB01805E914BAF
:104B3000AF4FBF4F8093EB049093EC04A093ED0430
:104B4000B093EE04FF90EF90DF90CF900895CF9256
:104B5000DF92EF92FF928091DA049091DB0400974C
:104B6000B9F0C090D604D090D704E090D804F0906B
:104B7000D9040897BC01990F880B990B0E94CAAE03
:104B80009B01AC01C701B6010E9428AE87FD09C098
:104B90001092CC041092CD041092CE041092CF0447
:104BA0001EC020E030E040E050E4C701B6010E94A2
:104BB0004FAD0E949CAE7093CB046093CA040E94D8
:104BC000E011DC01CB01805A9541AF4FBF4F80937C
:104BD000CC049093CD04A093CE04B093CF04FF9067
:104BE000EF90DF90CF90089580911D0290911E026A
:104BF0000F971816190614F480E090E09093F904CA
:104C00008093F80480E056DF1092DB041092DA04FF
:104C10009EDF80911D0290911E020F9718161906B3
:104C200014F480E090E09093F9048093F80480E01D
:104C300041DF1092FA0475981092DB041092DA04A6
:104C40001092DC04A5980895EF92FF920F931F93A2
:104C5000CF93C82F7B018A0180916E028823D1F007
:104C60000E946E16C7010E945D1681EC94E00E94BE
:104C70005D16C7FD08C06AE070E08C2FCC0F990B61
:104C80000E94BA1C04C08DEB94E00E945D168AE07D
:104C90000E94C71B8091B80481110DC010926E0252
:104CA00081E08093B804C801CF911F910F91FF90CC
:104CB000EF900C94DFABCF911F910F91FF90EF908D
:104CC00093CF8F3F19F047E954E002C04CEA54E01B
:104CD00065E874E0B9CF8F3F19F04FE554E002C0AA
:104CE00044E754E06DE474E0AFCF2F923F924F92CF
:104CF0005F926F927F928F929F92BF92CF92DF923C
:104D0000EF92FF920F931F93CF93DF936C014B01B0
:104D1000B22E180127FD04C0C22F220FDD0B02C0E6
:104D2000C1E0D0E0FA014080518062807380CC0FF6
:104D3000DD1FCC0FDD1F8E0109571B4FA301920110
:104D4000F80160817181828193810E9428AE88235D
:104D500091F0F801408251826282738211E020E07A
:104D600030E0A901C301B2010E942BB018160CF06B
:104D700010E0F6011483F60184818230C9F083309B
:104D800009F456C0813009F070C0FE01E957FB4FAD
:104D90002081318142815381F4016081718182815E
:104DA00093810E9428AE87FD60C082E0F601848373
:104DB000C957DB4FB70180E090E00E94C8AE9B016D
:104DC000AC01688179818A819B810E944EAD9B01F3
:104DD000AC01F40160817181828193810E942BB0CA
:104DE00087FD15C00E94E0112B013C019101A8EE46
:104DF000B3E00E94ACB1DC01CB01840D951DA61D72
:104E0000B71DF60180839183A283B3832EC00E94D5
:104E1000E011F6010081118122813381DC01CB0197
:104E2000801B910BA20BB30BB7FD1FC083E08483E3
:104E3000FFEFBF1619F04FE653E002C047E853E01A
:104E40006FE573E08B2DDF91CF911F910F91FF9054
:104E5000EF90DF90CF90BF909F908F907F906F905A
:104E60005F904F903F902F90EFCEDF91CF911F91A9
:104E70000F91FF90EF90DF90CF90BF909F908F9019
:104E80007F906F905F904F903F902F9008958F92FA
:104E90009F92AF92BF92CF92DF92EF92FF920F93C9
:104EA0001F93CF93DF93CDB7DEB728970FB6F89453
:104EB000DEBF0FBECDBF80915804811117C0809115
:104EC000C804811118C028960FB6F894DEBF0FBE33
:104ED000CDBFDF91CF911F910F91FF90EF90DF90A9
:104EE000CF90BF90AF909F908F90089580E090E01A
:104EF0000E94DFABE4CF0EDD0E94E0114B015C01AC
:104F00006D837E838F83988760911D0270911E024E
:104F1000072E000C880B990B0E94CAAE9B01AC01B6
:104F20006091F4047091F5048091F6049091F70477
:104F30000E942BB0181634F445E354E065E274E0A7
:104F400080E082DE6091F8047091F904072E000C75
:104F5000880B990B0E94CAAE69837A838B839C83EA
:104F60003EE1E32EF12C0FE010E020E0AE014F5FB8
:104F70005F4F64EF74E083EC94E0B7DEC090F4041C
:104F8000D090F504E090F604F090F70480911B02B5
:104F900090911C02BC01990F880B990B0E94CAAE1C
:104FA0009B01AC01C701B6010E942BB01816CCF4CE
:104FB00060911D0270911E02072E000C880B990B48
:104FC0000E94CAAE9B01AC01C701B6010E9428AE87
:104FD00087FF07C080E0B2D80E9497AE75956795AD
:104FE00001C060E06093FA048091EB049091EC04BE
:104FF000A091ED04B091EE040097A105B10511F167
:10500000881A990AAA0ABB0AB7FC1CC06091E90475
:105010007091EA0480E090E00E94C8AE9B01AC0170
:105020006091F4047091F5048091F6049091F70476
:105030000E9428AE87FF85C04EE054E06FEF73E01A
:1050400080E002DE20E030E046E153E46091D604E7
:105050007091D7048091D8049091D9040E942BB00C
:1050600018160CF465C0BE016B5F7F4F8AEC94E0AC
:1050700029D88823D9F06091CA047091CB0480E0CC
:1050800090E00E94C8AE2091D6043091D7044091A0
:10509000D8045091D9040E942BB018160CF04FC0C0
:1050A00048EC53E069EB73E08FEFCEDD6091DA04FA
:1050B0007091DB04072E000C880B990B0E94CAAE7E
:1050C00069837A838B839C839AE0E92EF12C0FE02D
:1050D00010E02FEFAE014F5F5F4F66ED74E08EEB97
:1050E00094E003DE8090D6049090D704A090D8047A
:1050F000B090D90420E030E040EA50E4C501B401AA
:105100000E942BB087FD0AC020E030E046E153E466
:10511000C501B4010E9428AE181624F460E0609323
:10512000DC04D1CE69D90E9497AE75956795F7CF0B
:105130004BEE53E06BED73E08FEF86DD94CF07DD30
:10514000B5CF80E0B7DC7ECFE0EFF4E080819181E5
:1051500093838283E2EDF4E0808191819383828363
:1051600081E08093C80408951F93CF93DF938091CB
:10517000C804811101C0E8DF1092F1041092F0041C
:105180001092D3041092D204C091F204D091F3048F
:10519000D195C195D1098091F8049091F90411E05D
:1051A000181619062CF08091FA04811101C010E044
:1051B0008091190290911A029195819591098C170D
:1051C0009D0714F480E07DDD112361F080911702CA
:1051D00090911802919581959109C817D90714F4F7
:1051E00080E079DD8091DA049091DB04C1E018164B
:1051F00019062CF08091DC04811101C0C0E02091DF
:10520000D4043091D5048091D0049091D1048217B8
:10521000930714F08FEF55DDCC2381F0209121020C
:10522000309122028091D4049091D5048217930783
:105230002CF08FEFDF91CF911F914DCDDF91CF916A
:105240001F9108950F930FB70F9300916E000B7F7E
:1052500000936E0078940F930BB70F930CB70F92D7
:105260001F922F933F934F935F936F937F938F93EF
:105270009F93AF93BF93EF93FF931124C7D0FF91F8
:10528000EF91BF91AF919F918F917F916F915F91BE
:105290004F913F912F911F900F900CBF0F910BBF1B
:1052A0000F910460F89400936E000F910FBF0F915F
:1052B0001895CF93809116028F3790F08F57909169
:1052C000FA0490938604992311F0759A01C0759899
:1052D0009091DC0490938504992359F0A59A0AC013
:1052E00090918604891708F0759890918504891724
:1052F00008F0A598805F809316029091840481E065
:105300008927809384048091150285301CF4C1E0C4
:10531000C80F01C0C0E08230A1F184F4882329F1D4
:10532000813009F062C010927B0080E480937C00A1
:1053300080917A00806480937A0057C0843009F4A9
:105340003EC094F1853009F050C0909183049111D2
:1053500002C08093830480918304815080938304EE
:10536000882309F442C0C5E040C0809114028F5FD9
:1053700080311CF48093140238C010921402F4DEC1
:1053800034C080917A0086FD2DC080917800909184
:1053900079002091F0043091F104820F931F9093D3
:1053A000F1048093F00421C010927B0082E480938A
:1053B0007C0080917A00806480937A0016C080918E
:1053C0007A0086FD11C0809178009091790020913B
:1053D000D2043091D304820F931F9093D30480930F
:1053E000D20403C0C2E001C0C4E0C09315020E9411
:1053F0003F348091AA069091AB06009729F001975F
:105400009093AB068093AA06CF91089552CFFF9256
:105410000F931F93CF93DF93CDB7DEB728970FB6C7
:10542000F894DEBF0FBECDBFF82E00EF14E0F801F8
:1054300060857185072E000C880B990B0E94CAAEFF
:1054400069837A838B839C83F80184819581A6810B
:10545000B7818D839E83AF83B8874DEFBE016F5FA9
:105460007F4FCE0105960E942D2002ED14E0F80139
:1054700060857185072E000C880B990B0E94CAAEBF
:1054800069837A838B839C83F80184819581A681CB
:10549000B7818D839E83AF83B8874FEFBE016F5F67
:1054A0007F4FCE0105960E942D208F2D0E949020C7
:1054B000BC018BE593E00E948E16F801628570E0D6
:1054C00086E593E00E948E1628960FB6F894DEBF0C
:1054D0000FBECDBFDF91CF911F910F91FF90089527
:1054E0002F923F924F925F926F927F928F929F92F4
:1054F000AF92BF92CF92DF92EF92FF920F931F93E2
:10550000CF93DF93CDB7DEB7CD54D1090FB6F89462
:10551000DEBF0FBECDBF2E969FAF8EAF2E97162F3C
:10552000742E26962FAF26970E94E011688B798BF8
:105530008A8B9B8B17FD04C0A4E1EA2EF12C03C0DB
:10554000FCE3EF2EF12C2E96AEADBFAD2E972D9134
:105550003D914D915C912FA738AB49AB5AAB17FDEC
:105560008FC4C12E012E000CDD08F60183E0EE0F82
:10557000FF1F8A95E1F7E95EFD4F668177816F50E5
:105580007109072E000C880B990B0E94CAAE9B0173
:10559000AC016FA578A989A99AA90E942BB0181609
:1055A000ECF489E796E0C35BDF4F0FB6F894DEBFFB
:1055B0000FBECDBFDF91CF911F910F91FF90EF9064
:1055C000DF90CF90BF90AF909F908F907F906F9023
:1055D0005F904F903F902F900C945D1685E696E07B
:1055E0000E945D1601DB27E12C9DC0012D9D900DD1
:1055F0001124FC01E051FB4F2FE7228780E090E06F
:10560000A0E5B1E423968CAF9DAFAEAFBFAF2397BB
:105610009701A8EEB3E00E94ACB16BAF7CAF8DAF49
:105620009EAF9B01AC0188899989AA89BB89280F03
:10563000391F4A1F5B1F2BAB3CAB4DAB5EAB81E010
:1056400080936D0288889988AA88BB888EA29FA2C1
:10565000A8A6B9A6188E198E1A8E1B8E1C8A1D8AB2
:105660001E8A1F8A1A821B821C821D821A8690E45F
:105670009C8FACE1AD8FB6E4BE8F1F8E18A219A22D
:105680001AA21EA61FAA18AE19AE1AAE2FE730E056
:1056900040E050E02E833F8348875987EFE7CE2EC6
:1056A000D12CE12CF12C1AA61BA61CA61DA631E0BC
:1056B0003BA31F861E86212C312C00E0198247E176
:1056C0001402C001112480519B4FDC011A962596CB
:1056D000BFAFAEAF2597FC013496FDA3ECA3272DF9
:1056E000770C330B28963FAF2EAF289780916D0231
:1056F000882309F48EC20E94E0112B013C018091A5
:10570000C804882309F4F9C005D917FF0AC02090FE
:10571000D6043090D7040091D8043091D90439834D
:105720000CC0ACA1BDA12C9011963C901197129683
:105730000C9112971396BC91B9839101402F598116
:105740006F8D78A189A19AA10E9428AE87FF05C01C
:105750002F8E38A209A3E981EAA39101402F598134
:105760006A857C8D8D8D9E8D0E942BB018162CF431
:105770002A863C8E0D8FF981FE8F2BA1222309F4FE
:1057800063C02E96AEADBFAD2E972D913D914D913C
:105790005C91B101802F99810E942BB018160CF0FA
:1057A000ACC0A3019201281939094A095B092C965A
:1057B0002CAF3DAF4EAF5FAF2C97DA01C9018858CF
:1057C0009341A109B109B7FD98C0D701C6012E8147
:1057D0003F8148855985821B930BA40BB50BB5956A
:1057E000A7959795879517FF03C08093DC0405C0A4
:1057F0002596EEADFFAD259780832C962CAD3DAD63
:105800004EAD5FAD2C972AA73BA74CA75DA72E9660
:10581000AEADBFAD2E97BC91BF8F2E96EEADFFAD56
:105820002E97F181F8A32E96AEADBFAD2E971296AE
:10583000BC91B9A32E96EEADFFAD2E97F381FAA3DE
:105840004EA25FA268A679A62E96AEADBFAD2E97EA
:105850002D913D914D915C91B101802F99810E94D4
:1058600028AE87FF0BC3D301C2012EA13FA148A5DB
:1058700059A5821B930BA40BB50BAC01BD01485875
:1058800053416109710977FDF9C24E855F85452B4A
:1058900009F0DAC18E819F81A885B9858C0D9D1D87
:1058A000AE1DBF1DB595A7959795879517FFE0C2CB
:1058B0008093DC042E853F852F5F3F4F3F872E87E7
:1058C0002E96AEADBFAD2E97BC91BA872E96EEAD9B
:1058D000FFAD2E97F181FC8F2E96AEADBFAD2E970A
:1058E0001296BC91BD8F2E96EEADFFAD2E97F38133
:1058F000FE8F5301420121E02BA320E030E040EA7B
:1059000051E42E96AEADBFAD2E976D917D918D91E8
:105910009C910E944FAD9B01AC01B101802F9981F8
:105920000E942BB018162CF481EF95E00E945D16B2
:1059300070C1D301C201288939894A895B89821BD8
:10594000930BA40BB50BB7FD8BC0812F17FD80E027
:105950005EDD8AE00E94C71BD301C2018053984FCD
:10596000AF4FBF4F888B998BAA8BBB8B9EA5911194
:1059700055C02FA938AD49AD5AADB101802F9981DD
:105980000E942BB0181694F520E030E040E050E47F
:10599000B101802F99810E944FAD6FAB78AF89AF75
:1059A0009AAF2BAD3CAD4DAD5EAD240D351D461D02
:1059B000571D2BAB3CAB4DAB5EAB23962CAD3DAD39
:1059C0004EAD5FAD23976FA578A989A99AA90E94CA
:1059D0004EAD9B01AC0181E08EA7B101802F998172
:1059E0000E942BB01816E4F11EA63AC0D301C201E2
:1059F0002BA93CA94DA95EA9821B930BA40BB50B47
:105A0000B7FD2EC01F3F19F047EC55E002C04EED28
:105A100055E068EB75E0812F17D922C020E030E017
:105A200040EA51E42E96AEADBFAD2E976D917D91BB
:105A30008D919C910E944EAD9B01AC01B101802FD4
:105A400099810E9428AE87FF0BC01F3F19F04CE8D8
:105A500055E002C044EA55E06CE775E0812FF4D8C8
:105A6000D301C201880F991FAA1FBB1F2EA13FA1FE
:105A700048A559A5821B930BA40BB50B881999094E
:105A8000AA09BB0981389F44A241B10528F08EE5DF
:105A900095E00E945D16BDC04E855F8528968EAD4F
:105AA0009FAD2897841795070CF020CE4330510501
:105AB0000CF41CCE81E095E00E945D1617FD05C038
:105AC0002CEFE22E24E0F22E04C09DEFE92E94E0AC
:105AD000F92E8FED94E00E945D16C7010E945D16BD
:105AE0004A815B816C817D8188EF94E00E94A816D9
:105AF0008AE00E94C71B8FED94E00E945D16C701EB
:105B00000E945D164C895D896E897F8984EF94E0DF
:105B10000E94A8168AE00E94C71B8FED94E00E94A5
:105B20005D16C7010E945D16488D598D6A8D7B8D6B
:105B300080EF94E00E94A8168AE00E94C71B269678
:105B40009FAD2697992309F4BCC117FF31C02A8164
:105B50003B814C815D812093DD043093DE044093D2
:105B6000DF045093E0042CEA35EC47E25EE36C89F5
:105B70007D898E899F890E9466B06093E10470934D
:105B8000E2048093E3049093E4042CEA35EC47E2CA
:105B90005EE3688D798D8A8D9B8D0E942FAE609318
:105BA000E5047093E6048093E7049093E80489C1C8
:105BB00047E1140290011124890100511B4F8A8191
:105BC0009B81AC81BD81F80183879487A587B687C7
:105BD0002CEA35EC47E25EE36C897D898E899F89EA
:105BE0000E9466B0D8011F966D937D938D939C9310
:105BF00052972CEA35EC47E25EE3688D798D8A8D09
:105C00009B8D0E942FAEF801638B748B858B968BD6
:105C100058C1C35BDF4F0FB6F894DEBF0FBECDBFD8
:105C2000DF91CF911F910F91FF90EF90DF90CF9078
:105C3000BF90AF909F908F907F906F905F904F90AC
:105C40003F902F900C94F4258AA49BA4ACA4BDA4EF
:105C5000880E991EAA1EBB1E2AA53BA54CA55DA5B4
:105C6000281B390B4A0B5B0BCA01B9012E813F81FE
:105C7000488559850E9430B1A50194010E9488B1E0
:105C8000D701C601820F931FA41FB51F8431910550
:105C9000A105B105FCF06C017D018C3E9105A105CB
:105CA000B1052CF06BEEC62ED12CE12CF12C40E886
:105CB000C416D104E104F104DCF08EEF90E0A0E022
:105CC000B0E08C199D09AE09BF098E839F83A88718
:105CD000B98712C054E1C52ED12CE12CF12C24E15E
:105CE00030E040E050E02E833F834887598704C06E
:105CF000CE82DF82E886F986B701A6018DE596E0BF
:105D00000E9498164E815F816885798588E596E0C6
:105D10000E9498164A855C8D6D8D7E8D81E596E09A
:105D20000E94A8164F8D58A169A17AA18AE496E035
:105D30000E94A8164E855F85433051050CF4AACD0C
:105D40006E817F81888599850E94CAAE20E030E00F
:105D500040E850E40E9466B06A837B838C839D8315
:105D60002A853C8D4D8D5E8D6F8D78A189A19AA17C
:105D70000E944EAD2BED3FE049E450E40E9466B036
:105D800020E030E040E05FE30E9466B09B01AC01A0
:105D90006A817B818C819D810E942FAE6A877B877F
:105DA0008C879D87C501B4010E94CAAE2FE632E1FF
:105DB00043E85AE30E9466B04B015C012AE939E9E5
:105DC00049E15FE36A857B858C859D850E9466B08D
:105DD0006A837B838C839D839B01AC010E944FADC2
:105DE000A50194010E942FAE6C8B7D8B8E8B9F8BB7
:105DF000A50194016A817B818C819D810E9466B09E
:105E000020E030E040E05EE30E9466B0688F798F6A
:105E10008A8F9B8F4A855B856C857D8584E496E0BF
:105E20000E94A816B501A4018EE396E00E94A81670
:105E30008EE296E00E945D164A815B816C817D81D5
:105E400088E296E00E94A8164C895D896E897F8958
:105E500082E296E00E94A816488D598D6A8D7B8D4E
:105E60008CE196E00E94A8168AE00E94C71B12CD22
:105E70002596EEADFFAD259780831CCD1BA23DCDB1
:105E800020E030E047E053E46FA578A989A99AA9FA
:105E90000E942BB018160CF484CB85E696E00E9485
:105EA0005D160E94F4258FE78093DC0420E030E04B
:105EB00040E051E423962CAF3DAF4EAF5FAF239748
:105EC000A7CBC35BDF4F0FB6F894DEBF0FBECDBFCD
:105ED000DF91CF911F910F91FF90EF90DF90CF90C6
:105EE000BF90AF909F908F907F906F905F904F90FA
:105EF0003F902F900895CF92DF92EF92FF92809182
:105F0000BD048823A1F10E94E011C090B904D09093
:105F1000BA04E090BB04F090BC04DC01CB018C1906
:105F20009D09AE09BF09B7FD22C00E94E0116B01B7
:105F30007C012091BD0430E0A8EEB3E00E94ACB13A
:105F4000DC01CB018C0D9D1DAE1DBF1D8093B904DE
:105F50009093BA04A093BB04B093BC0480E057DADA
:105F60008AE0FF90EF90DF90CF900C94C71BFF90DA
:105F7000EF90DF90CF9008952F923F924F925F92D3
:105F80006F927F928F929F92AF92BF92CF92DF9249
:105F9000EF92FF920F931F93CF93DF93CDB7DEB7AE
:105FA00064970FB6F894DEBF0FBECDBF898B6A8BA6
:105FB00081E080936D021A821B821C821D821986E9
:105FC0001A861B861C8621E0288719821D863CE3E1
:105FD0003E874CE14F8756E4588BC12CD12C80E88A
:105FE000E82E9FEBF92E812C912C54016091F8043E
:105FF0007091F904072E000C880B990B0E94CAAE11
:106000006B8B7C8B182F092F9B01482F592FB601C2
:10601000C7010E9428AE882399F12091F4043091A1
:10602000F5044091F6045091F7046B897C89812F27
:10603000902F0E9428AE881F8827881F89838A890D
:10604000882311F199819923F9F080916D0264966A
:106050000FB6F894DEBF0FBECDBFDF91CF911F9179
:106060000F91FF90EF90DF90CF90BF90AF909F90F7
:106070008F907F906F905F904F903F902F900895FA
:10608000CB8ADC8A1E2D0F2D0E94E0116B017C0152
:10609000DC01CB0129853A854B855C85821B930BFE
:1060A000A40BB50BB7FD34C0D701C60188519C4F76
:1060B000AF4FBF4F89879A87AB87BC878989A7D99C
:1060C0008FE493E00E945D1681149104A104B10451
:1060D000C9F0D501C40188519C4FAF4FBF4FBC01DF
:1060E000CD016C197D098E099F0928EE33E040E04F
:1060F00050E00E9466B1CA01B9014AE050E00E9436
:10610000A91C03C08FE30E94C71B8AE00E94C71B23
:106110000E94B6AC0E94E01160931A0C70931B0CA5
:1061200080931C0C90931D0C2090F4043090F50487
:106130009091F6049E83A091F704AF839101492FBB
:106140005A2F6B897C89812F902F0E944EAD2B0195
:106150003C0120E030E0A9010E942BB087FF04C081
:10616000C301B201905802C0C301B20120E030E087
:1061700040E251E481149104A104B10481F40E942D
:1061800028AE87FF12C0B88546015701BB2369F0CE
:10619000E8EE8E0EE3E09E1EA11CB11C06C00E941C
:1061A0002BB0181614F446015701F981FF2391F121
:1061B0002A813B814C815D812115310541055105C5
:1061C00041F0D701C601821B930BA40BB50BB7FDA1
:1061D00021C091014E815F816D857E858F85988973
:1061E0000E944EAD20E030E040EC5FE30E9428AE1C
:1061F00087FD2BCFD701C601805A9541AF4FBF4FC6
:106200008A839B83AC83BD832D863E869E819F8738
:10621000AF81A88B80916D02882309F416CF811479
:106220009104A104B10431F41886CB88DC88E12EF6
:10623000F02EDCCEB8EECB1AB3E0DB0AE108F108B1
:10624000C818D908EA08FB08F7FCEECFFECE2F925B
:106250003F924F925F926F927F928F929F92AF92F6
:10626000BF92CF92DF92EF92FF920F931F93CF9343
:10627000DF93CDB7DEB763970FB6F894DEBF0FBEDE
:10628000CDBF898B81E080936D021A821B821C82B4
:106290001D8219861A861B861C8621E02887198292
:1062A0001D863CE33E874CE14F8756E4588BC12C5A
:1062B000D12C80E8E82E9FEBF92E812C912C5401F3
:1062C0006091DA047091DB04072E000C880B990BA7
:1062D0000E94CAAE6A8B7B8B182F092F9B01482F17
:1062E000592FB601C7010E9428AE882399F1209149
:1062F000D6043091D7044091D8045091D9046A89CA
:106300007B89812F902F0E9428AE881F8827881FA5
:1063100089838989882311F199819923F9F08091E2
:106320006D0263960FB6F894DEBF0FBECDBFDF914E
:10633000CF911F910F91FF90EF90DF90CF90BF9082
:10634000AF909F908F907F906F905F904F903F9015
:106350002F900895CA8ADB8A1E2D0F2D0E94E0110E
:106360006B017C01DC01CB0129853A854B855C857D
:10637000821B930BA40BB50BB7FD34C0D701C6012C
:1063800088519C4FAF4FBF4F89879A87AB87BC8797
:1063900080E03DD88BE493E00E945D168114910467
:1063A000A104B104C9F0D501C40188519C4FAF4F7D
:1063B000BF4FBC01CD016C197D098E099F0928EEE4
:1063C00033E040E050E00E9466B1CA01B9014AE002
:1063D00050E00E94A91C03C08FE30E94C71B8AE003
:1063E0000E94C71B0E94B6AC0E94E01160931A0C79
:1063F00070931B0C80931C0C90931D0C9091D604F1
:106400009E83A091D704AF832090D8043090D90404
:10641000292F3A2FA1016A897B89812F902F0E9411
:106420004EAD2B013C0120E030E0A9010E942BB0D1
:1064300087FF04C0C301B201905802C0C301B2017A
:1064400020E030E040EA50E481149104A104B1045A
:1064500081F40E9428AE87FF12C0B885460157011B
:10646000BB2369F0E8EE8E0EE3E09E1EA11CB11C7A
:1064700006C00E942BB0181614F446015701F9818A
:10648000FF2391F12A813B814C815D8121153105EA
:106490004105510541F0D701C601821B930BA40BA6
:1064A000B50BB7FD21C02E813F81A1016D857E8591
:1064B0008F8598890E944EAD20E030E040EC5FE38C
:1064C0000E9428AE87FD2BCFD701C601805A954187
:1064D000AF4FBF4F8A839B83AC83BD839E819D87D3
:1064E000AF81AE872F86388A80916D02882309F4A8
:1064F00016CF81149104A104B10431F41886CA881E
:10650000DB88E12EF02EDCCEB8EECB1AB3E0DB0A4E
:10651000E108F108C818D908EA08FB08F7FCEECF33
:10652000FECEE3ECF4E01082118212821382148218
:106530000895CF93C82F6115710519F0CB010E9402
:106540005D168BE198E00E945D16C11103C08CE0DE
:1065500098E002C081E198E00E945D168AE0CF9148
:106560000C94C71B80910F058093100508958091AE
:106570000E05882319F010920E05089587E798E01C
:106580000C94DFAB80911005811105C080910A0544
:10659000811101C0089562E070E080E090E00E9407
:1065A0001B1680910B05882339F061E070E080E0D4
:1065B00090E00E941B16F5CF0895809310058093FC
:1065C0000F05E0CF26982E9A25982D9A24982C9A7C
:1065D0003F98479A0A98129A0998119A81E0EDCF4C
:1065E00080931005CFCF80930A05CCCF80910E0504
:1065F000882339F190910E0580910905981709F1CA
:106600000E946B1688E698E00E945D1680910E0548
:1066100080FD1CC080910E0584FD18C080910E0580
:1066200081FD1EC080910E0585FD1AC080910E056A
:1066300082FD20C080910E0586FD1CC08AE00E946C
:10664000C71B80910E0580930905089580E00E9484
:10665000145EAB01BC0184E698E00E94A816DECF70
:1066600081E00E94145EAB01BC0180E698E00E94CC
:10667000A816DCCF82E00E94145EAB01BC018CE561
:1066800098E00E94A816DACFCF9382E498E00E94A7
:106690005D1683B1C1E086FB882780F96CE378E062
:1066A0008C2747DF86B1809566E378E0881F8827CE
:1066B000881F3FDF83B185FB882780F960E378E09E
:1066C0008C2737DF80B182FB882780F96AE278E087
:1066D0008C272FDF83B18295817064E278E08C276C
:1066E00028DF80B1869581706EE178E08C27CF91AC
:1066F00020CF80910D051E9904C0816080930D0507
:1067000003C08E7F80930D0580910D05379904C0DD
:10671000806180930D0503C08F7E80930D0580916D
:106720000D051D9904C0826080930D0503C08D7F07
:1067300080930D0580910D05029904C080628093BD
:106740000D0503C08F7D80930D0580910D051C996B
:1067500004C0846080930D0503C08B7F80930D057A
:1067600080910D05019904C0806480930D0503C0DC
:106770008F7B80930D059091080580910D059817EA
:1067800031F092E090930B058093080509C0809149
:106790000B05882329F0815080930B05882349F04D
:1067A00080911005811108C080910A05811104C0F3
:1067B000089590930C05F4CF80917F0580FF1BC056
:1067C0009091800580910C0590FF0BC080FF13C055
:1067D00080910E05816080930E0580E00E94125E1C
:1067E0000AC084FF08C080910E05806180930E0569
:1067F00080E00E94125E80917F0581FF1BC0909116
:10680000800580910C0591FF0BC081FF13C0809122
:106810000E05826080930E0581E00E94125E0AC020
:1068200085FF08C080910E05806280930E0581E08F
:106830000E94125E80917F0582FF20C080918005BA
:1068400082FF10C080910A058823C1F080910C0559
:1068500082FF14C080910E05846080930E0582E053
:106860000C94125E80910C0586FF08C080910E0585
:10687000806480930E0582E00C94125E089539CFF7
:10688000CF938823A1F0C82F0E946B1684E50E9445
:10689000C71B6AE070E08C2F90E00E94BA1C80E277
:1068A0000E94C71B85E898E0CF910C945D16CF91AC
:1068B000089508958091AF069091AC06891B8F7062
:1068C00019F480E090E008959091A906992351F081
:1068D000833030F48FEF890F19F08093A906F1CF40
:1068E0001092A906E091AC0686E5E89FF00111241C
:1068F000E055F94F808180FDE4CF8091AC068F5F39
:106900008F708093AE069091AC068091AD0698137F
:1069100006C08091AE068093AD06CF010895CF01E9
:106920000895EFE6F0E08081826080830895809191
:10693000800580FF09C080910B018270809309015E
:106940008FEF8093110509C080910B0180958270B3
:106950008093090181E0809311058091800581FF7A
:106960000AC080910B0180958170809309018FEF9F
:106970008093120508C080910B01817080930901FA
:1069800081E0809312058091800582FF09C080918B
:106990000B018470809309018FEF8093130509C068
:1069A00080910B01809584708093090181E0809330
:1069B000130500000000000008950F930FB70F9318
:1069C00000916E000F930B7F00936E0000916F009B
:1069D0000D7F00936F000F930BB70F930CB70F92BF
:1069E0001F922F933F934F935F936F937F938F9358
:1069F0009F93AF93BF93EF93FF9311240E94BD3DEC
:106A0000FF91EF91BF91AF919F918F917F916F9186
:106A10005F914F913F912F911F900F900CBF0F915D
:106A20000BBF0F910260F89400936F000F910093D9
:106A30006E000F910FBF0F911895CF92DF92EF92DA
:106A4000FF920F931F9380917E058823D1F01092BF
:106A50007E058091810590918205892B91F010929D
:106A60007F0510928205109281059091AF0680916A
:106A7000AC06981731F08091AC068F5F8F708093D1
:106A8000AC068091810590918205892B09F4AAC1F9
:106A900040914D0550914E0560914F057091500504
:106AA0009091750500914105109142052091430593
:106AB00030914405041B150B260B370B892F90E0F2
:106AC000A0E0B0E0081719072A073B0710F4D90126
:106AD000C801E82F840F951FA61FB71F80934D058F
:106AE00090934E05A0934F05B093500520918400DC
:106AF00030918500225E3F4F4091650550916605BB
:106B000060916705709168058091550590915605D3
:106B1000A0915705B0915805840F951FA61FB71F68
:106B20008093650590936605A0936705B09368050B
:106B3000B7FD1CC0409A4091150550911605609113
:106B400017057091180580911105082E000C990BFE
:106B5000AA0BBB0B840F951FA61FB71F80931505AB
:106B600090931605A0931705B093180540916905F9
:106B700050916A0560916B0570916C058091590583
:106B800090915A05A0915B05B0915C05840F951F0B
:106B9000A61FB71F8093690590936A05A0936B05A4
:106BA000B0936C05B7FD1CC0419A409119055091F6
:106BB0001A0560911B0570911C0580911205082E25
:106BC000000C990BAA0BBB0B840F951FA61FB71FB8
:106BD0008093190590931A05A0931B05B0931C058B
:106BE00040916D0550916E0560916F057091700533
:106BF00080915D0590915E05A0915F05B091600563
:106C0000840F951FA61FB71F80936D0590936E0587
:106C1000A0936F05B0937005B7FD1CC0429A4091D8
:106C20001D0550911E0560911F05709120058091F2
:106C30001305082E000C990BAA0BBB0B840F951F94
:106C4000A61FB71F80931D0590931E05A0931F05D7
:106C5000B0932005409171055091720560917305C4
:106C6000709174058091610590916205A091630512
:106C7000B0916405840F951FA61FB71F80937105FF
:106C800090937205A0937305B0937405B7FD3CC053
:106C9000C0902105D0902205E0902305F0902405B6
:106CA00040911405042E000C550B660B770B4C0D10
:106CB0005D1D6E1D7F1D409321055093220560933D
:106CC0002305709324054091510550915205609120
:106CD000530570915405841B950BA60BB70B80933D
:106CE000710590937205A0937305B093740590910C
:106CF00080058091360593FF04C08150809336054E
:106D000003C08F5F80933605809184009091850049
:106D100082179307C8F38091650590916605A0914D
:106D20006705B0916805B7FD15C0409151055091B8
:106D300052056091530570915405841B950BA60B69
:106D4000B70B8093650590936605A0936705B09394
:106D5000680540988091690590916A05A0916B053E
:106D6000B0916C05B7FD15C0409151055091520589
:106D70006091530570915405841B950BA60BB70BBE
:106D80008093690590936A05A0936B05B0936C0599
:106D9000419880916D0590916E05A0916F05B0911D
:106DA0007005B7FD15C04091510550915205609195
:106DB000530570915405841B950BA60BB70B80935C
:106DC0006D0590936E05A0936F05B0937005429882
:106DD000E15041F0809184009091850082179307E3
:106DE000C8F388CE1F910F91FF90EF90DF90CF9066
:106DF0000895CF92DF92EF92FF928091350588231C
:106E000009F465C0C0904D05D0904E05E0904F0547
:106E1000F090500540914505509146056091470519
:106E200070914805809136054C155D056E057F050E
:106E3000E8F420913B0530913C05E0913905F09153
:106E40003A05E217F30790F48150809336052150FC
:106E5000310930933C0520933B0540912702509126
:106E600028026091290270912A0234C0C416D50606
:106E7000E606F706E8F420913B0530913C05409189
:106E80003705509138052417350790F48F5F8093AC
:106E900036052F5F3F4F30933C0520933B054091D3
:106EA0002702509128026091290270912A0212C093
:106EB0008FEF9FEFDC018093270290932802A0932D
:106EC0002902B0932A024FEF5FEFBA0103C04FEFE0
:106ED0005FEFBA018091360587FD06C080910B01F6
:106EE00080748093090106C080910B0180958074A5
:106EF000809309012091840030918500225E3F4FEC
:106F000080913605882311F1439A809184009091F5
:106F1000850082179307C8F38091360587FF04C068
:106F20008F5F8093360503C0815080933605439868
:106F300080913605882321F380918400909185000B
:106F400082179307C8F3225E3F4FDACFCB01BA0115
:106F5000FF90EF90DF90CF900895BC0120918105C4
:106F600030918205409181055091820524173507A3
:106F700011F09A01F7CF81E06217730709F080E002
:106F80000895CF93DF93EC0188819981AA81BB8119
:106F9000E5E1F5E080839183A283B383EB018881EF
:106FA0009981AA81BB8184839583A683B783EA01F3
:106FB00088819981AA81BB8180879187A287B387C5
:106FC000E90188819981AA81BB8184879587A687F9
:106FD000B787DF91CF9108953F924F925F926F9262
:106FE0007F928F929F92AF92BF92CF92DF92EF9259
:106FF000FF920F931F93CF93DF93CDB7DEB7289700
:107000000FB6F894DEBF0FBECDBFA0918105B09141
:107010008205109739F180904D0590904E05A09013
:107020004F05B09050054091410550914205609147
:1070300043057091440584169506A606B706C8F068
:1070400010927F0510928205109281059091AF06F3
:107050008091AC06981731F08091AC068F5F8F70ED
:107060008093AC0670EDC72E77E0D72EE12CF12C83
:1070700097C14091490550914A0560914B05709127
:107080004C05481559056A057B0508F46EC000914A
:107090007A0510917B0520917C0530917D05D19674
:1070A0004D915D916D917C91D497EE27059FF12DC7
:1070B000169FC001269F900D259F800D911D069F54
:1070C000F00D811D9E1F159FF00D811D9E1F249F99
:1070D000F00D811D9E1F149FF10D8E1F9E1FF695B2
:1070E0008E1F9E1F709F800D911D719F900D11240A
:1070F000FD01EB5BFF4F4081518162817381480F3D
:10710000591F611D711D40933105509332056093E5
:107110003305709334053497C080D180E280F380CA
:10712000C416D506E606F70640F4C0923105D092A3
:107130003205E0923305F0923405409131055091CB
:107140003205609133057091340583EE98E0BB24DD
:10715000B394FC01C590D590E590F490C416D50683
:10716000E606F70608F475C27FC2409045055090C8
:1071700046056090470570904805481459046A0414
:107180007B0408F080C0209176053091770540910E
:107190007805509179052D833E834F835887D1968A
:1071A0000D911D912D913C91D4974D815E816F8100
:1071B0007885EE27419FF12D529FC001629F900D6F
:1071C000619F800D911D429FF00D811D9E1F519F5B
:1071D000F00D811D9E1F609FF00D811D9E1F509F11
:1071E000F10D8E1F9E1FF6958E1F9E1F349F800DE2
:1071F000911D359F900D11248C0120E030E0C0904E
:107200003105D0903205E0903305F0903405CD0182
:10721000875B9F4FFC010C151D052E053F05C0F433
:10722000408151816281738149835A836B837C835E
:10723000C01AD10AE20AF30AC416D506E606F70612
:1072400010F46A017B0183EE98E03324339410C07C
:10725000C080D180E280F380F6CFF694E794D79493
:10726000C794330C049628E08F3F920709F480C23C
:10727000FC0105911591259134910C151D052E05E4
:107280003F0558F375C2809136058823D9F0D7960B
:107290004D915C91D89760E070E0009127021091C9
:1072A00028022091290230912A0204171507260787
:1072B000370741F010922B0210922C0210922D02EF
:1072C00010922E02409123025091240260912502D7
:1072D0007091260277FF5CC0AF5BBF4F8D919D918F
:1072E0000D90BC91A02D23EE38E041E0F901C5904E
:1072F000D590E590F490C816D906EA06FB0658F436
:10730000B695A79597958795440F2C5F3F4F58E00A
:107310002F3F350759F74093750580329105A10538
:10732000B10520F480E290E0A0E0B0E08097A109F0
:10733000B109811578E09707A105B10508F4CEC21F
:1073400024E0929FF00111249F012D5F324FF9013B
:10735000329665917491EE27879FA001869F410D1B
:107360005E1F06944E1F5E1F112460E070E0F9015D
:1073700085919491A0E0B0E0841B950BA60BB70B10
:107380008093230290932402A0932502B0932602B7
:10739000C0902302D0902402E0902502F0902602B3
:1073A0008091810590918205892B09F01DC382DAB5
:1073B0009093820580938105892B09F415C3E09190
:1073C0008105F0918205808183FF19C09F012F5DA7
:1073D0003F4FAF01435E5F4FBF01675E7F4FCF01FD
:1073E0004596CFDD9091AF068091AC069817F9F2E3
:1073F0008091AC068F5F8F708093AC06D8CFC58824
:10740000D688E788F08C81E0C114D104E104F1044E
:1074100009F480E0018D128D238D348D0115110545
:107420002105310509F08260458D568D678D70A16B
:10743000411551056105710509F0846080937F0550
:1074400010927605109277051092780510927905C2
:1074500010927A0510927B0510927C0510927D05A2
:1074600085A196A1A7A1B0A580934105909342055F
:10747000A0934305B0934405882499245401881AA5
:10748000990AAA0ABB0A8092710590927205A0928D
:107490007305B092740580926D0590926E05A0926E
:1074A0006F05B09270058092690590926A05A0926E
:1074B0006B05B0926C058092650590926605A0926E
:1074C0006705B0926805CC0CDD1CEE1CFF1CC09259
:1074D0005505D0925605E0925705F0925805000FD9
:1074E000111F221F331F0093590510935A05209333
:1074F0005B0530935C05440F551F661F771F409353
:107500005D0550935E0560935F057093600541A132
:1075100052A163A174A1440F551F661F771F4093AA
:107520006105509362056093630570936405880F4D
:10753000991FAA1FBB1F8093510590935205A093DA
:107540005305B093540510924D0510924E051092BC
:107550004F051092500581A592A5A3A5B4A58093CF
:10756000490590934A05A0934B05B0934C0585A51A
:1075700096A5A7A5B0A98093450590934605A0932D
:107580004705B093480586A980933505882309F1FE
:1075900083AD94AD90933A058093390581AD92AD5A
:1075A000909338058093370510922B0210922C028D
:1075B00010922D0210922E0287A990ADA0E0B0E0AB
:1075C0008093270290932802A0932902B0932A0265
:1075D0000BC08FEF9FEFDC0180932702909328026E
:1075E000A0932902B0932A0285A99091800589175A
:1075F00019F0809380059BD97CD88FEF9FEFDC0139
:107600008093230290932402A0932502B093260234
:10761000E0918105F0918205EB5BFF4F80819181C4
:10762000A281B3818093310590933205A0933305F5
:10763000B093340523EE38E041E0F901C590D590D0
:10764000E590F490C816D906EA06FB0608F46BC16B
:1076500076C17695679557954795BB0C0496E8E0FB
:107660008F3F9E0709F075CDB092750540325105E8
:107670006105710520F440E250E060E070E04052A6
:10768000510961097109411588E0580761057105C3
:1076900000F194E0599FF0011124CF018D5F924FCA
:1076A000FC013296E590F490F701DD244F9F5001E4
:1076B0004E9FA10CBD1C0694AD1CBD1C1124FC01E9
:1076C000C590D490E12CF12CCA18DB08E108F10830
:1076D00024C06A017B01F694E794D794C794F6011D
:1076E000EC7FCF018D5F964F7C01FC0185919491D9
:1076F000F7013296E590F49047704E9DB0014F9D92
:10770000700D1124AB0163E0569547956A95E1F73A
:107710006C01C41AD50AE12CF12C0C0D1D1D2E1D77
:107720003F1D00937A0510937B0520937C053093D1
:107730007D059091350580913605992309F465C042
:10774000882309F42DCED7968D919C91D897A0E0EF
:10775000B0E0409127025091280260912902709177
:107760002A02481759076A077B0709F051C018CE4B
:1077700030927505F0E2CF16D104E104F10428F44B
:1077800030E2C32ED12CE12CF12CF0E2CF1AD1083B
:10779000E108F108C11428E0D206E104F10408F47C
:1077A00040C034E0D39EC00111248D5F924FFC0194
:1077B0003296059114916C2D3327619FA001609F33
:1077C000410D531F0694431F531F1124FC01C59004
:1077D000D490E12CF12CC41AD50AE108F1084D81AE
:1077E0005E816F8178854C0D5D1D6E1D7F1D409300
:1077F00076055093770560937805709379058091AD
:107800003505811132C080913605882309F4C8CD31
:1078100010922B0210922C0210922D0210922E0226
:10782000BFCD970186013695279517950795F801E5
:10783000EC7FCF018D5F964FFC0105911491FC0107
:107840003296459154913C2D3770349FC001359F3D
:10785000900D112423E0969587952A95E1F768010C
:10786000C81AD90AE12CF12CBACF430C511C611C67
:10787000711C481459046A047B04C8F480913605CD
:10788000882309F48DCDD7964D915C91D89760E00F
:1078900070E0009127021091280220912902309176
:1078A0002A02041715072607370709F479CD109225
:1078B0002B0210922C0210922D0210922E02D796BB
:1078C0008D919C91D897A0E0B0E08093270290938F
:1078D0002802A0932902B0932A0262CDAC01BD0117
:1078E0007695679557954795FA01EC7FAF014D5F07
:1078F000564FFA0125913491FA01329665917491AF
:107900008770869FA001879F500D1124CA01F3E064
:1079100096958795FA95E1F7A901481B590BCA017D
:10792000A0E0B0E02DCDB695A79597958795440F2B
:107930002C5F3F4F68E02F3F360709F07ECE409323
:10794000750580329105A105B10520F480E290E033
:10795000A0E0B0E08097A109B109811558E0950732
:10796000A105B105F8F064E0969FF00111249F0194
:107970002D5F324FF901329665917491EE27879F02
:10798000A001869F410D5E1F06944E1F5E1F1124AD
:10799000F901C590D490E12CF12CC41AD50AE10864
:1079A000F10822C0AC01BD017695679557954795C2
:1079B000FA01EC7FAF014D5F564FFA01C590D490AC
:1079C000FA013296459154918770849F9001859F6A
:1079D000300D1124C901A3E096958795AA95E1F78A
:1079E000C81AD90AE12CF12CC701B60128960FB6A6
:1079F000F894DEBF0FBECDBFDF91CF911F910F91E5
:107A0000FF90EF90DF90CF90BF90AF909F908F90BE
:107A10007F906F905F904F903F900895CF92DF924C
:107A2000EF92FF921F93CF93DF938FEF9FEF90938F
:107A30008900809388001AE0C0E0D0E078948091BB
:107A40003D0590913E05A0913F05B0914005892BE1
:107A50008A2B8B2B11F40E941D3580912B02909163
:107A60002C02A0912D02B0912E02892B8A2B8B2BF8
:107A700049F4BFD960932B0270932C0280932D029E
:107A800090932E0280913D0590913E05A0913F0577
:107A9000B0914005892B8A2B8B2B49F49DDA60939A
:107AA0003D0570933E0580933F0590934005C0903F
:107AB0003D05D0903E05E0903F05F0904005409197
:107AC0002B0250912C0260912D0270912E02FC2D00
:107AD000ED2D3E2D2F2D4C155D056E057F0520F4F7
:107AE000F42FE52F362F272F8F2F9E2FA32FB22F66
:107AF000009721E0A207B10520F08FEF9FEFA0E0F3
:107B0000B0E0C81AD90AEA0AFB0AC0923D05D09231
:107B10003E05E0923F05F09240054F3F2FEF5207A0
:107B20006207720761F0481B590B6A0B7B0B40938D
:107B30002B0250932C0260932D0270932E02F89426
:107B40002091840030918500205F3F4F115039F023
:107B5000C80FD91FC217D30708F470CF01C0E901BD
:107B6000D0938900C09388007894DF91CF911F91C2
:107B7000FF90EF90DF90CF90089550CF90916F00DD
:107B800091FB222720F991FF05C090916F009D7F06
:107B900090936F0094E0899FF0011124EB5EFA4FFF
:107BA0006081718182819381222329F020916F006D
:107BB000226020936F00089590916F0091FB22271F
:107BC00020F991FF05C090916F009D7F90936F0009
:107BD00034E0839FC0011124FC01EB5EFA4F408129
:107BE000518162817381FC01EB5DFA4F40835183C7
:107BF0006283738381E080937E05222329F0809144
:107C00006F00826080936F00089590916F0091FBE8
:107C1000222720F991FF05C090916F009D7F9093DE
:107C20006F0094E0899FF0011124EB5DFA4F6081B1
:107C3000718182819381222329F020916F0022603B
:107C400020936F0008954F925F926F927F928F9270
:107C50009F92AF92BF92CF92DF92EF92FF9280916C
:107C60006F0081FB992790F981FF05C080916F001B
:107C70008D7F80936F0040901505509016056090A1
:107C80001705709018058090190590901A05A0901E
:107C90001B05B0901C05C0901D05D0901E05E090FE
:107CA0001F05F0902005992329F080916F008260D4
:107CB00080936F0089ED98E00E945D164AE050E0E5
:107CC000C301B2010E94A91C85ED98E00E945D16D7
:107CD0004AE050E0C501B4010E94A91C81ED98E082
:107CE0000E945D164AE050E0C701B6010E94A91C3F
:107CF0008AE0FF90EF90DF90CF90BF90AF909F9081
:107D00008F907F906F905F904F900C94C71BDB011A
:107D100090918F05992309F440C0833070F494E06A
:107D2000899FF0011124ED57FA4FAB01770F660BD5
:107D3000770B4083518362837383813091F018F015
:107D40008230E9F008952FEF30E00E94BBB120EDC2
:107D500037E040E050E00E9488B1B9018EE20C9417
:107D6000AC122FEF30E00E94BBB120ED37E040E0D5
:107D700050E00E9488B1B9018DE20C94AC122FEF53
:107D800030E00E94BBB120ED37E040E050E00E94BF
:107D900088B1B9018CE20C94AC12089580918F05E2
:107DA000882391F0609183057091840580E0AFDFB6
:107DB000609187057091880581E0A9DF60918B054E
:107DC00070918C0582E0A3CF0895EAE0F1E0808114
:107DD00088608083808180618083808180628083ED
:107DE000DDDFE1E2F1E08081887F816080830895BA
:107DF00067FD2CC0813061F028F0823099F083302B
:107E0000D9F024C0662311F0A19A2AC0A19828C0F5
:107E1000809108016111809580788093060147FF69
:107E200027C0089580910801611180958074809326
:107E3000060147FF23C008958091080161118095D4
:107E400088708093060147FF21C0089547FD26C032
:107E5000813071F038F0823089F08330B9F00895C4
:107E600047FD1CC0442311F0A09A0895A0980895DE
:107E7000442311F0A29A0895A298089580910801D0
:107E800041118095807280930601089580910801C8
:107E900041118095807180930601089508956430A2
:107EA00091F040F4613059F06230A9F420E040E0F4
:107EB00061E09ECF683059F0603149F00CC020E09D
:107EC00040E060E095CF20E041E060E091CF20E02D
:107ED00041E061E08DCF0E946E1689EB98E00C9432
:107EE0005D160F931F93CF93999A989A80910701EB
:107EF0008068809307019A9A80910701806480933B
:107F0000070180910701806280930701809107013A
:107F10008860809307018091070180618093070149
:107F20000FE213E0C0E0F80161918F018C2FB7DF01
:107F3000CF5FC630C1F7CF911F910F910895D1DF68
:107F4000EAE0F1E0808182608083808181608083CB
:107F50008081846080838081806480830F9A179AF7
:107F60000E9A169A0D9A159A0C9A149A389A409865
:107F7000179A8091B9058E7F8093B905399A4198F7
:107F8000169A8091B9058D7F8093B9053A9A4298E7
:107F9000159A8091B9058B7F8093B9053B9A4398D8
:107FA000149AA0E8B0E08C918C7F8C93E1E8F0E02B
:107FB0008081877E886080838C918F738C93808191
:107FC000887F8260808380E090E490938900809332
:107FD00088001092850010928400EFE6F0E0808126
:107FE00082608083789482E0809380050E94973439
:107FF00081E080938F05E9CE84EA98E00E945D16C7
:10800000919902C080E301C081E30E94C71B90994F
:1080100002C080E301C081E30E94C71B80EA98E0B0
:108020000E945D1680910601881F8827881F805D49
:108030000E94C71B929902C080E301C081E30E94A5
:10804000C71B8CE998E00E945D168091060186FDB1
:1080500002C080E301C081E30E94C71B809106013A
:1080600085FD02C080E301C081E30E94C71B87E950
:1080700098E00E945D168091060183FD02C080E3B6
:1080800001C081E30E94C71B8091060184FD02C0EC
:1080900080E301C081E30C94C71BCF93DF93CDB77E
:1080A000DEB760970FB6F894DEBF0FBECDBF8091EC
:1080B000520290915302A0915402B09155028983CB
:1080C0009A83AB83BC838091560290915702A09112
:1080D0005802B09159028D839E83AF83B8878091F7
:1080E0005A0290915B02A0915C02B0915D02898777
:1080F0009A87AB87BC8780915E0290915F02A091C6
:108100006002B09161028D879E87AF87B88B0E9415
:10811000716D6091660270916702072E000C880BEA
:10812000990B0E94CAAE2AE037ED43E25CE30E945D
:1081300066B06093620270936302809364029093CE
:10814000650280E00E94365481E00E94365482E04D
:108150000E94365423DE0E94B86D40E150E062E593
:1081600072E0CE0101960E94F3B5892B51F0609622
:108170000FB6F894DEBF0FBECDBFDF91CF910C9448
:10818000FE5160960FB6F894DEBF0FBECDBFDF91F3
:10819000CF9108958D35924041F00E946E1685E78B
:1081A00094E10E945D1681E0089580E00895EF92C9
:1081B000FF920F931F93CF93DF93CDB7DEB7C458D1
:1081C000D1090FB6F894DEBF0FBECDBFED961CAE41
:1081D0001DAE1EAE1FAEED9785E492E5A2E5B0E0C0
:1081E000E9968CAF9DAFAEAFBFAFE997CF57DF4FEA
:1081F00019821882C158D04084E690E0C158DF4F00
:1082000099838883CF57D0400E940A171092910516
:108210009E012F573F4F44E050E0BE016B587F4F07
:10822000CE0181589F4F0E940E17C158DF4F8881A1
:108230009981CF57D0400296C158DF4F99838883E8
:10824000CF57D040CF57DF4F19821882C158D04046
:1082500081E0CC57DF4F8883C458D0409E012F5710
:108260003F4F41E050E0BE016C577F4FCE01815837
:108270009F4F0E940E179E012F573F4F48E450E03A
:1082800061E676E0CE0181589F4F0E940E179E0155
:108290002F573F4F40E150E061E376E0CE01815837
:1082A0009F4F0E940E178AE097EDA3EABCE3ED967C
:1082B0008CAF9DAFAEAFBFAFED979E012F573F4F35
:1082C00044E050E0BE0167587F4FCE0181589F4F78
:1082D0000E940E178E010F5F1F4F8CE0F801119264
:1082E0008A95E9F79E012F573F4F4CE050E0B801C7
:1082F000CE0181589F4F0E940E1780E090E0A0E2CF
:10830000B1E489839A83AB83BC839E012F573F4F8F
:1083100044E050E0B801CE0181589F4F0E940E17F3
:10832000ED961CAE1DAE1EAE1FAEED9783E0AE9671
:108330008FAFAE9789839E012F573F4F44E050E0A7
:10834000BE0167587F4FCE0181589F4F0E940E1784
:108350009E012F573F4F41E050E0BE0163597F4FD0
:10836000CE0181589F4F0E940E179E012F573F4FFD
:1083700041E050E0B801CE0181589F4F0E940E1796
:108380002AE0F22EFA949E012F573F4F44E050E02E
:10839000FF2049F0BE0167587F4FCE0181589F4FA3
:1083A0000E940E17EFCF62E975E0CE0181589F4F12
:1083B0000E940E179E012F573F4F44E250E06CE0A1
:1083C00076E0CE0181589F4F0E940E1783E0CD5773
:1083D000DF4F8883C358D040EE968FAFEE97E1967B
:1083E0001CAE1DAE1EAE1FAEE19719821A821B8213
:1083F0001C82ED961CAE1DAE1EAE1FAEED979E010B
:108400002F573F4F41E050E0BE016D577F4FCE01E7
:1084100081589F4F0E940E179E012F573F4F41E0FA
:1084200050E0BE0163587F4FCE0181589F4F0E949C
:108430000E179E012F573F4F44E050E0B801CE0188
:1084400081589F4F0E940E179E012F573F4F44E0C7
:1084500050E0BE0163597F4FCE0181589F4F0E946B
:108460000E179AE0E92EF12CF1E0EF1AF10871F005
:108470009E012F573F4F44E050E0BE0167587F4FA9
:10848000CE0181589F4F0E940E17EECFAE961FAEC1
:10849000AE978FEF89839E012F573F4F41E050E009
:1084A000BE0163597F4FCE0181589F4F0E940E1726
:1084B0009E012F573F4F41E050E0B801CE01815857
:1084C0009F4F0E940E1780E1F82EF8018F2D119218
:1084D0008A95E9F79E012F573F4F40E150E0B801E0
:1084E000CE0181589F4F0E940E1788EC90E0AF9606
:1084F0009FAF8EAFAF9780EF90E0E1969FAF8EAFCA
:10850000E19786E490E09A8389838EE690E09C83ED
:108510008B83EE961FAEEE97EF961FAEEF979E0100
:108520002F573F4F44E050E0BE0163597F4FCE01CB
:1085300081589F4F0E940E179E012F573F4F44E0D6
:1085400050E0B801CE0181589F4F0E940E179E0146
:108550002F573F4F42E050E0BE0163587F4FCE019E
:1085600081589F4F0E940E17F8011192FA94E9F773
:1085700080E090E0A0E8BFE38D879E87AF87B88B4F
:108580008091FB049091FC04A091FD04B091FE0445
:1085900089839A83AB83BC838091FF04909100050B
:1085A000A0910105B09102058D839E83AF83B887AA
:1085B0008091030590910405A0910505B0910605F1
:1085C00089879A87AB87BC879E012F573F4F40E131
:1085D00050E0B801CE0181589F4F0E940E1784E1F0
:1085E00090E09A8389839E012F573F4F42E050E0ED
:1085F000B801CE0181589F4F0E940E179E012F5740
:108600003F4F4CE050E06DED74E0CE0181589F4F3C
:108610000E940E1780E290E09A8389839E012F5773
:108620003F4F42E050E0B801CE0181589F4F0E9479
:108630000E1781E089839E012F573F4F41E050E0A4
:10864000B801CE0181589F4F0E940E1780E2EFE7DC
:10865000F2E0D80101900D928A95E1F79E012F5723
:108660003F4F40E250E0B801CE0181589F4F0E9439
:108670000E17AE961FAEAE979E012F573F4F41E0AB
:1086800050E0BE0163597F4FCE0181589F4F0E9439
:108690000E17198280E090E0A0E4B0E4ED968CAF74
:1086A0009DAFAEAFBFAFED979E012F573F4F41E05B
:1086B00050E0B801CE0181589F4F0E940E179E01D5
:1086C0002F573F4F44E050E0BE0167587F4FCE0127
:1086D00081589F4F0E940E178AE1F80111928A95E6
:1086E000E9F79E012F573F4F4AE150E0B801CE0114
:1086F00081589F4F0E940E1784E3EFE9F2E0D80102
:1087000001900D928A95E1F79E012F573F4F44E368
:1087100050E0B801CE0181589F4F0E940E171A8277
:1087200019821C821B821E821D829E012F573F4F81
:1087300046E050E0B801CE0181589F4F0E940E17CD
:108740008DE0F80111928A95E9F79E012F573F4F6E
:108750004DE050E0B801CE0181589F4F0E940E17A6
:108760009E012F573F4F44E050E063ED75E0CE018E
:1087700081589F4F0E940E179E012F573F4F4CE08C
:1087800050E063E875E0CE0181589F4F0E940E17BC
:108790008CE6F80111928A95E9F79E012F573F4F19
:1087A0004CE650E0B801CE0181589F4F0E940E1751
:1087B0009E012F573F4F4CE050E060E076E0CE0145
:1087C00081589F4F0E940E17E1961CAE1DAE1EAE43
:1087D0001FAEE197E5961CAE1DAE1EAE1FAEE5972F
:1087E0009E012F573F4F48E050E0BE0163597F4F35
:1087F000CE0181589F4F0E940E179E012F573F4F69
:1088000044E050E066E774E0CE0181589F4F0E943B
:108810000E179E012F573F4F44E050E06AE774E087
:10882000CE0181589F4F0E940E179E012F573F4F38
:1088300044E050E06EE774E0CE0181589F4F0E9403
:108840000E179E012F573F4F41E050E062E874E061
:10885000CE0181589F4F0E940E179E012F573F4F08
:1088600044E050E060E172E0CE0181589F4F0E94E9
:108870000E17EE961FAEEE9780E090E0A8ECB1E404
:10888000E1968CAF9DAFAEAFBFAFE1979E012F5782
:108890003F4F41E050E0BE0163587F4FCE01815809
:1088A0009F4F0E940E179E012F573F4F44E050E00C
:1088B000BE0163597F4FCE0181589F4F0E940E1712
:1088C0008091910581114FC0C158DF4F08811981F6
:1088D000CF57D04004561109CF57DF4F8881998177
:1088E000C158D040AF969FAF8EAFAF9784E690E06F
:1088F000C158DF4F99838883CF57D0409E012F57AF
:108900003F4F44E050E065E373E0CE0181589F4F54
:108910000E940E179E012F573F4F42E050E0BE01CC
:1089200063597F4FCE0181589F4F0E940E170E94BE
:108930006B16B80183E694E10E94C816AF964EAD5F
:108940005FADAF9760E070E086E594E10E94D216DB
:1089500083E594E10E945D16C8011CDC90919105AD
:10896000892B809391050E940C179091910581E0CD
:108970008927CC57DF4F0FB6F894DEBF0FBECDBFAF
:10898000DF91CF911F910F91FF90EF9008951F936A
:10899000CF93DF93CDB7DEB72C970FB6F894DEBF39
:1089A0000FBECDBFA1E6B6E020E030E0C901243023
:1089B000310510F083E090E0880F991F880F991F10
:1089C000FC01EE55FC4E459155916591749154967C
:1089D0004D935D936D937C935797FC01EE56FC4E3F
:1089E000459155916591749194964D935D936D93D6
:1089F0007C939797FC01EE57FC4E459155916591FC
:108A000074914D935D936D937D932F5F3F4F243011
:108A1000310509F0CBCF80E29EE4A0E0B0E0809386
:108A2000710690937206A0937306B093740680E06B
:108A300090E0AAEFB4E48093950690939606A093F5
:108A40009706B093980640E050E86BE375E44093D6
:108A5000990650939A0660939B0670939C068093A8
:108A60009D0690939E06A0939F06B093A006109239
:108A7000A1061092A2061092A3061092A4061092CC
:108A8000A5061092A6061092A7061092A80680E0EE
:108A900090E0A0E4B1E48093310690933206A09375
:108AA0003306B09334068093350690933606A09330
:108AB0003706B09338068DEC9CECACECBEE38093AB
:108AC000390690933A06A0933B06B0933C0680E0AB
:108AD00090E0A0E2B1E480933D0690933E06A0931F
:108AE0003F06B093400610928204109276041092D2
:108AF0007704109278041092790410927A041092FC
:108B00007B0410927C0410927D0410927E041092DB
:108B10007F04109280041092810480E090E0A0E431
:108B2000B0E48093100290931102A0931202B093CC
:108B300013020E94DA1D80E090E0A0EBBFEB80936F
:108B4000920590939305A0939405B09395058CEEB0
:108B500091E5A6EEB1E48093FB049093FC04A0930E
:108B6000FD04B093FE0480EF98E3A0EABEE3809397
:108B7000FF0490930005A0930105B093020588EBD4
:108B800092E9A5E2B4E48093030590930405A093D1
:108B90000505B093060580E090E0A3E9B3E4809377
:108BA000DD049093DE04A093DF04B093E00483EC33
:108BB00094E6AAE2B1E48093E1049093E204A093E6
:108BC000E304B093E40480EB98EBA1E1B5E4809377
:108BD000E5049093E604A093E704B093E80481E0F1
:108BE0000E94DD320E9459341092D3051092D405B0
:108BF0001092D5051092D6058CE0E3EDF2E0DE018F
:108C0000119601900D928A95E1F713E01150C0F092
:108C100084E0189F90011124E1E0F0E0EC0FFD1FCB
:108C2000E20FF31F6081718182819381F901ED5719
:108C3000FA4F6083718382839383812F68D8E6CF54
:108C40002CDA0E946B168FE593E12C960FB6F89400
:108C5000DEBF0FBECDBFDF91CF911F910C945D168B
:108C6000CF93C82F811102C00E946B1688E493E154
:108C70000E945D1686E091E10E945D168AE00E94E6
:108C8000C71B8AE00E94C71BC11106C00E946B1659
:108C900087E393E10E945D166FEF81E08C270E94CD
:108CA0005D95C11108C00E946B1689E193E10E9495
:108CB0005D160E946B164091850650918606609164
:108CC00087067091880680E193E10E94A816409182
:108CD000890650918A0660918B0670918C068DE012
:108CE00093E10E94A81640918D0650918E066091E6
:108CF0008F06709190068AE093E10E94A816409139
:108D0000910650919206609193067091940687E0C7
:108D100093E10E94A8168AE00E94C71BC11108C0F7
:108D20000E946B1685EE92E10E945D160E946B1602
:108D3000609161067091620680916306909164066D
:108D40000E94C8AEAB01BC018CED92E10E94A81656
:108D5000609165067091660680916706909168063D
:108D60000E94C8AEAB01BC0189ED92E10E94A81639
:108D70006091690670916A0680916B0690916C060D
:108D80000E94C8AEAB01BC0186ED92E10E94A8161C
:108D900060916D0670916E0680916F0690917006DD
:108DA0000E94C8AEAB01BC0183ED92E10E94A816FF
:108DB0008AE00E94C71BC11108C00E946B1689E897
:108DC00092E10E945D160E946B16409195065091AB
:108DD0009606609197067091980680E892E10E944D
:108DE000A8164091990650919A0660919B06709141
:108DF0009C068DE792E10E94A81640919D06509135
:108E00009E0660919F067091A0068AE792E10E94FB
:108E1000A8168AE00E94C71BC11113C00E946B16DE
:108E200082E392E10E945D1687E092E10E945D1666
:108E300088EF91E10E945D168AE00E94C71B0E94A4
:108E40006B16609171067091720680917306909115
:108E500074060E94C8AEAB01BC018FEE91E10E9486
:108E6000A8164091A1065091A2066091A3067091A8
:108E7000A4068CEE91E10E94A8164091A50650919F
:108E8000A6066091A7067091A80689EE91E10E945E
:108E9000A8164091310650913206609133067091C8
:108EA000340686EE91E10E94A81640913506509155
:108EB0003606609137067091380683EE91E10E9484
:108EC000A8164091390650913A0660913B06709180
:108ED0003C0680EE91E10E94A81640913D0650911B
:108EE0003E0660913F06709140068DED91E10E9433
:108EF000A8168AE00E94C71BC11108C00E946B1609
:108F000089EC91E10E945D160E946B16609130061B
:108F100070E080EC91E10E948E168AE00E94C71BEF
:108F2000C11108C00E946B1681EB91E10E945D1691
:108F30000E946B164091FB045091FC046091FD046B
:108F40007091FE0488EA91E10E94A8162CEA35ECA3
:108F500047E25EE36091FF04709100058091010596
:108F6000909102050E942FAEAB01BC0185EA91E110
:108F70000E94B8162CEA35EC47E25EE360910305E7
:108F80007091040580910505909106050E9466B0D8
:108F9000AB01BC0182EA91E10E94B8168AE00E940E
:108FA000C71BC11102C00E946B164091DD04509195
:108FB000DE046091DF047091E00489E991E10E9490
:108FC000A8162CEA35EC47E25EE36091E10470916B
:108FD000E2048091E3049091E4040E942FAEAB017F
:108FE000BC0186E991E10E94B8162CEA35EC47E213
:108FF0005EE36091E5047091E6048091E70490914E
:10900000E8040E9466B0AB01BC0183E991E10E94D3
:10901000B8168AE00E94C71BC11110C00E946B16CF
:1090200084E891E10E945D1686E091E10E945D1660
:1090300083E091E10E945D160E946B1640919205BB
:109040005091930560919405709195058BE791E19E
:109050000E94A8168AE00E94C71BC11108C00E9486
:109060006B168AE691E10E945D160E946B16409194
:10907000D3055091D4056091D5057091D60581E650
:1090800091E10E94A8168AE00E94C71BC11108C086
:109090000E946B1688E491E10E945D160E946B1697
:1090A00040918305509184056091850570918605F6
:1090B0008FE391E10E94D216409187055091880577
:1090C0006091890570918A058CE391E10E94D21626
:1090D00040918B0550918C0560918D0570918E05A6
:1090E00089E391E10E94D2168AE00E94C71BC11158
:1090F00008C00E946B1681E291E10E945D160E94F9
:109100006B168091820424E6829FC001112481584D
:109110009F4F6FEF70E00E9453B170E080E090E0ED
:109120000E94C8AE20E030E048EC52E40E942FAE2E
:10913000AB01BC0188E191E10E94A8164091760440
:1091400050917704609178047091790485E191E100
:109150000E94A81640917A0450917B0460917C048F
:1091600070917D0482E191E10E94A81640917E04F5
:1091700050917F0460918004709181048FE091E1AF
:109180000E94A816409110025091110260911202A3
:10919000709113028CE091E10E94A8168AE0CF91B1
:1091A0000C94C71B2F923F924F925F926F927F92C7
:1091B0008F929F92AF92BF92CF92DF92EF92FF92E7
:1091C0000F931F93CF93DF93CDB7DEB7C45AD10966
:1091D0000FB6F894DEBF0FBECDBF2DB73EB7CD554D
:1091E000DF4F39832883C35AD040C756DF4F1982D7
:1091F0001882C959D04084E690E0C956DF4F998360
:109200008883C759D0400E940A1701E09E01275663
:109210003F4F44E050E0BE016F567F4FCE0189566C
:109220009F4F0E9463179E0127563F4F42E050E038
:10923000BE016B567F4FCE0189569F4F0E94631728
:1092400043E050E0BE016F567F4F85E393E00E94FC
:1092500012B6892B19F1CC56DF4F8881C459D04002
:10926000882359F08FE3CF56DF4F8883C159D04010
:10927000CE56DF4F1882C259D0400E946B16BE01F5
:109280006F567F4F82E394E10E94711684E294E16D
:109290000E945D1681E0809391058DC5C357DF4F15
:1092A000188219821A821B82CD58D040C756DF4FD0
:1092B00019821882C959D04001E09E0127563F4FBC
:1092C00041E050E0BE0164567F4FCE0189569F4F6A
:1092D0000E9463178DB79EB7C156DF4F998388836D
:1092E000CF59D0406E019DE7C90ED11C80E1EFED52
:1092F000F2E0D60101900D928A95E1F77E01EDE64C
:10930000EE0EF11C80E1EFEEF2E0D70101900D923C
:109310008A95E1F780E1EFEFF2E09E012F5F3F4F8A
:109320005901D90101900D928A95E1F7C456DF4F9A
:109330004881CC59D04050E04D5F5F4F440F551FDE
:10934000440F551F8DB79EB7841B950B0FB6F8942D
:109350009EBF0FBE8DBFEDB7FEB731961F010091C6
:10936000900511E0012728563F4FBF01CE018956D5
:109370009F4F0E9463170091900501279E01275679
:109380003F4F44E050E061E776E0CE0189569F4FC1
:109390000E946317C456DF4F8880CC59D040912C6F
:1093A000F3E08F0E911C880C991C880C991C2DB72A
:1093B0003EB7281939090FB6F8943EBF0FBE2DBF2E
:1093C0008DB79EB701962C01EDB7FEB7E819F909E4
:1093D0000FB6F894FEBF0FBEEDBF2DB73EB72F5F9F
:1093E0003F4F39010091900501279E0127563F4FBD
:1093F000A401BC01CE0189569F4F0E9463170091C2
:10940000900501279E0127563F4FA401B301CE01CD
:1094100089569F4F0E94631730919005C256DF4FC7
:109420003883CE59D040332309F4CBC011E0C25663
:10943000DF4F0881CE59D04001279E0127563F4F6C
:1094400044E050E065E976E0CE0189569F4F0E94E6
:1094500063170091900501279E0127563F4F44E076
:1094600050E069E976E0CE0189569F4F0E9463176C
:109470000091900501279E0127563F4F44E050E0A0
:109480006DE976E0CE0189569F4F0E9463170091E7
:10949000900501279E0127563F4F44E050E061EAC6
:1094A00076E0CE0189569F4F0E9463170091900588
:1094B00001279E0127563F4F44E050E065EA76E0E1
:1094C000CE0189569F4F0E94631700919005012796
:1094D0009E0127563F4F40E150E061E376E0CE0128
:1094E00089569F4F0E9463170091900501279E01A6
:1094F00027563F4F44E050E0BE0163577F4FCE01F7
:1095000089569F4F0E946317C156DF4F888199810A
:10951000CF59D0400FB6F8949EBF0FBE8DBF0091BB
:10952000900501279E0127563F4F4CE050E0BE01B9
:109530006F5F7F4FCE0189569F4F0E946317009146
:10954000900501279E0127563F4F44E050E0BE01A1
:1095500063577F4FCE0189569F4F0E94631700913A
:10956000900501279E0127563F4F44E050E0BE0181
:1095700063577F4FCE0189569F4F0E94631701E0CA
:109580009E0127563F4F41E050E0B701CE0189567A
:109590009F4F0E9463179E0127563F4F41E050E0C6
:1095A000BE016F5F7F4FCE0189569F4F0E946317A8
:1095B000F701A0808981A89E50011124812C912C53
:1095C0009DC0C456DF4F8881CC59D04090E09C01AB
:1095D0002E5F3F4FCF55DF4F39832883C15AD0408C
:1095E000A1E6B6E040E050E080E090E04601B7013F
:1095F00031E0C356DF4F3883CD59D040CF55DF4FD0
:10960000E881F981C15AD040E817F90764F4C356DC
:10961000DF4F1882CD59D0409C018430910558F01D
:1096200023E030E008C0F101E40FF51F0081118153
:10963000228133810BC0220F331F220F331FF4010D
:10964000E20FF31F00811181228133810D931D935D
:109650002D933D93C356DF4FF881CD59D040FF2362
:1096600041F0F201E40FF51F008111812281338165
:1096700011C09C018430910510F023E030E0220FEE
:10968000331F220F331FFB01E20FF31F00811181F3
:109690002281338150960D931D932D933C935397C4
:1096A000C356DF4F2881CD59D040222341F0F3012A
:1096B000E40FF51F008111812281338111C09C01CB
:1096C0008430910510F023E030E0220F331F220F89
:1096D000331FF501E20FF31F0081118122813381D5
:1096E00090960D931D932D933C93939701964C5F09
:1096F0005F4F8430910509F07BCF98CE00919005A3
:109700008A149B0491F001279E0127563F4F44E0A5
:1097100050E0BE0163577F4FCE0189569F4F0E9494
:1097200063173FEF831A930AE9CF11E001279E01E7
:1097300027563F4F44E050E062E975E0CE0189567C
:109740009F4F0E9463170091900501279E012756A5
:109750003F4F44E250E06CE076E0CE0189569F4FE7
:109760000E94631701E09E0127563F4F41E050E001
:10977000BE0165567F4FCE0189569F4F0E946317E9
:109780009E0127563F4F41E050E0B601CE01895679
:109790009F4F0E9463170091900501279E01275655
:1097A0003F4F44E050E0B701CE0189569F4F0E94E1
:1097B00063170091900501279E0127563F4F44E013
:1097C00050E0BE016F5F7F4FCE0189569F4F0E94D0
:1097D0006317C556DF4FA880CB59D040F601808172
:1097E000A89E50011124812C912C009190058A147F
:1097F0009B0491F001279E0127563F4F44E050E023
:10980000BE0163577F4FCE0189569F4F0E94631759
:10981000FFEF8F1A9F0AE9CF11E001279E0127561B
:109820003F4F41E050E0B701CE0189569F4F0E9463
:1098300063170091900501279E0127563F4F41E095
:1098400050E0BE016F5F7F4FCE0189569F4F0E944F
:1098500063170091900501279E0127563F4F40E175
:1098600050E0BE016F5F7F4FCE0189569F4F0E942F
:1098700063170091900501279E0127563F4F44E052
:1098800050E0B701CE0189569F4F0E9463170091A7
:10989000900501279E0127563F4F44E050E0BE014E
:1098A0006F5F7F4FCE0189569F4F0E9463170091D3
:1098B000900501279E0127563F4F42E050E0B60138
:1098C000CE0189569F4F0E94631700919005012792
:1098D0009E0127563F4F40E150E0BE016F5F7F4F32
:1098E000CE0189569F4F0E94631700919005011188
:1098F0002EC089809A80AB80BC8020E030E84BE3AA
:1099000055E4C501B4010E9428AE882301F180927C
:10991000FB049092FC04A092FD04B092FE048D81A1
:109920009E81AF81B8858093FF0490930005A0933A
:109930000105B093020589859A85AB85BC85809326
:10994000030590930405A0930505B093060511E067
:1099500001279E0127563F4F42E050E0BE016F5F56
:109960007F4FCE0189569F4F0E946317009190054B
:1099700001279E0127563F4F4CE050E0BE016F5F2C
:109980007F4FCE0189569F4F0E946317009190052B
:10999000011115C020E030E84BE355E469817A817C
:1099A0008B819C810E9428AE882349F08CE0FE01C7
:1099B0003196ADEDB4E001900D928A95E1F711E09A
:1099C00001279E0127563F4F42E050E0BE016F5FE6
:1099D0007F4FCE0189569F4F0E94631700919005DB
:1099E00001279E0127563F4F41E050E0BE016F5FC7
:1099F0007F4FCE0189569F4F0E94631700919005BB
:109A000001279E0127563F4F40E250E0BE016F5FA5
:109A10007F4FCE0189569F4F0E946317009190059A
:109A200001279E0127563F4F41E050E0B701CE018C
:109A300089569F4F0E9463170091900501279E0150
:109A400027563F4F45E050E0BE016F5F7F4FCE018C
:109A500089569F4F0E94631780919005811102C023
:109A60000E9459340091900511E001279E0127566C
:109A70003F4F4AE150E0BE016F5F7F4FCE018956F4
:109A80009F4F0E9463170091900501279E01275662
:109A90003F4F44E350E0BE016F5F7F4FCE018956D8
:109AA0009F4F0E9463170091900501279E01275642
:109AB0003F4F46E050E0BE016F5F7F4FCE018956B9
:109AC0009F4F0E9463170091900501279E01275622
:109AD0003F4F4DE050E0BE016F5F7F4FCE01895692
:109AE0009F4F0E9463170091900501279E01275602
:109AF0003F4F44E050E0BE016F5F7F4FCE0189567B
:109B00009F4F0E9463170091900501110CC089813D
:109B10009A81AB81BC818093D3059093D405A093A7
:109B2000D505B093D60581E008279E0127563F4F03
:109B30004CE050E0BE016F5F7F4FCE0189569F4FD2
:109B40000E94631700919005011109C08CE0FE018D
:109B50003196A3E8B5E001900D928A95E1F711E006
:109B600001279E0127563F4F4CE650E0BE016F5F34
:109B70007F4FCE0189569F4F0E94631719821A8228
:109B80001B821C821D821E821F82188619861A86DD
:109B90001B861C860091900501279E0127563F4F8A
:109BA0004CE050E0BE016F5F7F4FCE0189569F4F62
:109BB0000E9463170091900501279E0127563F4F91
:109BC00048E050E0BE016F5F7F4FCE0189569F4F46
:109BD0000E9463170091900501279E0127563F4F71
:109BE00044E050E066E774E0CE0189569F4F0E9442
:109BF00063170091900501279E0127563F4F44E0CF
:109C000050E06AE774E0CE0189569F4F0E946317C7
:109C10000091900501279E0127563F4F44E050E0F8
:109C20006EE774E0CE0189569F4F0E946317009142
:109C3000900501279E0127563F4F41E050E062E822
:109C400074E0CE0189569F4F0E94631700919005E2
:109C500001279E0127563F4F44E050E060E172E04B
:109C6000CE0189569F4F0E946317009190050127EE
:109C70009E0127563F4F41E050E0B701CE01895683
:109C80009F4F0E9463170091900501279E01275660
:109C90003F4F44E050E0BE016F5F7F4FCE018956D9
:109CA0009F4F0E946317C956DF4F88819981C7591A
:109CB000D040845691090E94CA4080939105882320
:109CC000C1F00E946B16C956DF4F68817981C75970
:109CD000D040645671098CE194E10E948E166DE5C6
:109CE00072E084E194E10E94C8168AE00E94C71BDA
:109CF00058C0C756DF4F28813981C959D040CB564B
:109D0000DF4F88819981C559D04028173907E9F07C
:109D1000109391050E946E16CB56DF4F68817981B2
:109D2000C559D04084EF93E10E94C816C756DF4F53
:109D300068817981C959D0408FEE93E10E94C8169D
:109D40008FED93E10E945D162CC0809190058111EA
:109D500028C00E946B1605E313E0F80181918F0182
:109D6000882319F00E94C71BF8CFC956DF4F6881BE
:109D70007981C759D0406456710982EC93E10E9401
:109D80008E16C756DF4F48815981C959D04060E0CF
:109D900070E085EB93E10E94D21682EB93E10E9482
:109DA0005D1680919005811106C080919105811109
:109DB00002C00E944D4080919005811102C00E9416
:109DC00030460E940C179091910581E08927CD556E
:109DD000DF4F28813981C35AD0400FB6F8943EBF77
:109DE0000FBE2DBFCC55DF4F0FB6F894DEBF0FBEB0
:109DF000CDBFDF91CF911F910F91FF90EF90DF903A
:109E0000CF90BF90AF909F908F907F906F905F901A
:109E10004F903F902F90089581E080939005C2D994
:109E2000109290050895F8DF8111BCC90E94C744C3
:109E300081E00895BF92CF92DF92EF92FF920F934D
:109E40001F93CF93DF93CDB7DEB728970FB6F89463
:109E5000DEBF0FBECDBF90910A05981709F47AC0F6
:109E6000B82E882309F453C080E090E0A0EAB0E463
:109E70008D839E83AF83B887C0909205D090930561
:109E8000E0909405F090950520E030E0A901C7012D
:109E9000B6010E9428AE87FF0CC0A701960160E0C2
:109EA00070E080EA90E40E944EAD6D837E838F83E4
:109EB000988720E030E04FE153E46D817E818F810F
:109EC00098850E942BB0181644F480E090E0AFE132
:109ED000B3E48D839E83AF83B88720915A0230917B
:109EE0005B0240915C0250915D026D817E818F81A9
:109EF00098850E942BB0181654F419821A821B827E
:109F00001C82BE016F5F7F4FCE01059638D46091F1
:109F10005202709153028091540290915502209107
:109F200056023091570240915802509159021982BD
:109F30001A821B821C82E0905A02F0905B02009110
:109F40005C0210915D02FE0131966F0164D38B2D8E
:109F50000E94F33280E028960FB6F894DEBF0FBE61
:109F6000CDBFDF91CF911F910F91FF90EF90DF90C8
:109F7000CF90BF9008952F923F924F925F926F9231
:109F80007F928F929F92AF92BF92CF92DF92EF9289
:109F9000FF920F931F93CF93DF93CDB7DEB7A097B8
:109FA0000FB6F894DEBF0FBECDBF1C017F8F6E8F42
:109FB000498F28A3DC018D909D90AD90BC90FB0152
:109FC000408051806280738022ED30E040EE50ECA2
:109FD000C301B201002309F43BC00E942BB087FDEE
:109FE000D5C127E030E04EE353E4C301B2010E9443
:109FF00028AE18160CF4CAC123EA31E040E450EC54
:10A00000C501B4010E942BB087FDC0C127E030E03C
:10A0100042E253E4C501B4010E9428AE18160CF4C4
:10A02000B5C127E030E041E253E4C501B4010E942C
:10A0300028AE18160CF4AAC127E030E041E253E440
:10A04000C301B2010E9428AE18160CF49FC124C0AF
:10A050000E942BB087FD9AC127E030E04EE353E425
:10A06000C301B2010E9428AE18160CF48FC123EA76
:10A0700031E040E450ECC501B4010E942BB087FDF3
:10A0800085C127E030E042E253E4C501B4010E94FB
:10A0900028AE18160CF47AC1E0905A02F0905B02D8
:10A0A00000915C0210915D0280914E0290914F02EE
:10A0B000A0915002B09151028A8F9B8FAC8FBD8FBF
:10A0C0008091480290914902A0914A02B0914B02BE
:10A0D00080934E0290934F02A0935002B09351028E
:10A0E00019821A821B821C82DE0111966D01A30166
:10A0F0009201C501B4018FD281E09CDE8111DEC0E6
:10A100008091B90582FF11C020919205309193058D
:10A11000409194055091950560E070E080E890ECE6
:10A120000E944EAD2B013C0106C0412C512C40E257
:10A13000642E41EC742E4D865E866F86788AC12C23
:10A14000D12CE12C31E4F32EC986DA86EB86FC862D
:10A15000BE01675F7F4FCE010D9611D310910E05A2
:10A1600010920E0582E09CD171D112FD05C060E015
:10A1700070E080EC9FE75DC080905A0290905B0297
:10A18000A0905C02B0905D02C982DA82EB82FC8210
:10A1900020E030E040EA50E4C501B4010E944FAD38
:10A1A0006D837E838F839887BE016F5F7F4FCE0163
:10A1B0000596E5D24D825E826F82788680E090E0DF
:10A1C000A0E8BFE389839A83AB83BC83BE016F5F42
:10A1D0007F4FCE010596D3D210910E0510920E0539
:10A1E00082E05ED133D112FFC2CF0E94761F20E001
:10A1F00030E040E450E460915A0270915B0280913B
:10A200005C0290915D020E9466B02B013C01A501A9
:10A210009401C501B4010E944FAD9B01AC01C30183
:10A22000B2010E944FAD2DEC3CEC4CE45EE30E9489
:10A2300066B020919205309193054091940550911C
:10A2400095050E944FAD5B018C01898D8250823053
:10A2500048F580E090E0A0E0B1E4898B9A8BAB8B6D
:10A26000BC8B60915A0270915B0280915C0290916C
:10A270005D02B98DB33029F020E030E040EA50E4CF
:10A2800004C020E030E048EC51E40E944FAD6D8BFB
:10A290007E8B8F8B988FBE016F5E7F4FCE01459670
:10A2A0006ED207C0E98DE13021F480E0C3DD811179
:10A2B00005C0F8A1F33008F449C008C098A1933054
:10A2C00008F46DC0A12CB12C00EC1FE729E3822E0D
:10A2D00023E0922ED4018D914D01882319F00E9424
:10A2E000C71BF8CFF101608171818281938143E0C6
:10A2F00050E00E94451D91E4892E93E0992ED401EF
:10A300008D914D01882319F00E94C71BF8CFEE8D67
:10A31000FF8D608171818281938143E050E00E94D2
:10A32000451D86E4882E83E0982ED4018D914D0141
:10A33000882319F00E94C71BF8CF43E050E0B50115
:10A34000C8010E94451D8AE00E94C71B8A8D9B8D13
:10A35000AC8DBD8D80934E0290934F02A09350021E
:10A36000B09351029501A801B501C8010E9414B132
:10A37000882389F080E05EDD0E946E168DE894E10E
:10A380000E945D162A2D7B2DC8011AC020E070E0C6
:10A3900080EC9FE715C02A2D7B2DC80111C08A8D46
:10A3A0009B8DAC8DBD8D80934E0290934F02A093F8
:10A3B0005002B0935102A12CB12C00EC1FE7DACF70
:10A3C000822E972E5C01C501B401A0960FB6F894B9
:10A3D000DEBF0FBECDBFDF91CF911F910F91FF90D8
:10A3E000EF90DF90CF90BF90AF909F908F907F9035
:10A3F0006F905F904F903F902F900895CF93DF9391
:10A40000C2E5D2E0488159816A817B8186E195E18C
:10A410000E94A8164C815D816E817F8182E195E169
:10A420000E94A816488559856A857B858EE095E14E
:10A430000E94A8164C855D856E857F858AE095E132
:10A440000E94A816DF91CF910C94233E2EE532E0B6
:10A450004AE552E066E572E082E592E00C94C86C51
:10A460008EE592E00C94156DCF93DF9380E00E940F
:10A47000395ECCE9D5E0688379838A839B8381E068
:10A480000E94395E6C837D838E839F8382E00E946D
:10A49000395E688779878A879B87DF91CF91089596
:10A4A0001F93CF93DF93CDB7DEB760970FB6F894C5
:10A4B000DEBF0FBECDBF182FD7DF80919C059091D6
:10A4C0009D05A0919E05B0919F0589839A83AB83DA
:10A4D000BC838091A0059091A105A091A205B091A7
:10A4E000A3058D839E83AF83B8878091A405909147
:10A4F000A505A091A605B091A70589879A87AB8786
:10A50000BC8780915E0290915F02A0916002B09141
:10A5100061028D879E87AF87B88BCE0101960E941E
:10A520007E5D1E3F51F480E1FE013196A2E5B2E06E
:10A5300001900D928A95E1F716C024E0129FC001A8
:10A540001124FC01EE5AFD4FA1E0B0E0AC0FBD1F9D
:10A55000A80FB91F8D919D910D90BC91A02D808366
:10A560009183A283B38360960FB6F894DEBF0FBECB
:10A57000CDBFDF91CF911F910895AF92BF92CF923F
:10A58000DF92EF920F931F93A12CB12C6501E12C68
:10A590008C012EE532E04AE552E066E572E082E5A4
:10A5A00092E00E948C6B1F910F91EF90DF90CF9003
:10A5B000BF90AF900895AF92BF92CF92DF92EF928B
:10A5C0000F931F93CF93DF9300D01F92CDB7DEB7C9
:10A5D00069837A838B839C83A12CB12C6501E12C48
:10A5E0008E010F5F1F4F24EB35E040EB55E06CEA26
:10A5F00075E088EA95E00E948C6B0F900F900F90A9
:10A600000F90DF91CF911F910F91EF90DF90CF903E
:10A61000BF90AF9008954F925F926F927F928F920A
:10A620009F92AF92BF92CF92DF92EF92FF920F93E1
:10A630001F93CF93DF93CDB7DEB72C970FB6F89467
:10A64000DEBF0FBECDBF2B013C0129873A874B8768
:10A650005C8747015801F601E080F1800281138197
:10A6600020E030E0A901B701C8010E9428AE8111A5
:10A6700007C0E1E2F5E185919591A591B49102C001
:10A68000C701D8018D839E83AF83B88720E030E077
:10A69000A901B701C8010E9428AE811108C0E0904D
:10A6A0004802F090490200914A0210914B02C70102
:10A6B000D80189839A83AB83BC83A50194016091FF
:10A6C0005A0270915B0280915C0290915D020E943F
:10A6D00028AE87FF0BC080925A0290925B02A09234
:10A6E0005C02B0925D02CE01059647DF40925202B5
:10A6F00050925302609254027092550289859A8555
:10A70000AB85BC858093560290935702A093580264
:10A71000B0935902CE01019630DFA50194016091FA
:10A720005A0270915B0280915C0290915D020E94DE
:10A730002BB018165CF480925A0290925B02A092A1
:10A740005C02B0925D02CE01059617DF0E944D5E5D
:10A750002C960FB6F894DEBF0FBECDBFDF91CF9120
:10A760001F910F91FF90EF90DF90CF90BF90AF902F
:10A770009F908F907F906F905F904F900895CF92B1
:10A78000DF92EF92FF920F931F936B01FC01E08029
:10A79000F18002811381E2E5F2E024813581468176
:10A7A0005781608171818281938135DF1F910F9183
:10A7B000FF90EF90DF90CF900895CF92DF92EF92CD
:10A7C000FF920F931F936A01E0905A02F0905B0290
:10A7D00000915C0210915D02FB0120813181428178
:10A7E0005381FC01608171818281938114DF1F910B
:10A7F0000F91FF90EF90DF90CF90089580914E02DF
:10A8000090914F02A0915002B0915102809398050F
:10A8100090939905A0939A05B0939B0580914C0263
:10A8200090914D02909397058093960584E690E071
:10A8300090934D0280934C020895809198059091D9
:10A840009905A0919A05B0919B0580934E02909333
:10A850004F02A0935002B0935102809196059091BF
:10A86000970590934D0280934C020895A82FB0E075
:10A87000CD01880F991F880F991FFC01E85AFA4EE5
:10A88000459155916591749133E0AA0FBB1F3A959C
:10A89000E1F7A15DBD4F4D935D936D937C9313974D
:10A8A000FC01E45BFA4E45915591659174911496C3
:10A8B0004D935D936D937C9317970895CF92DF929C
:10A8C000EF92FF92CF93DF9320914702222309F466
:10A8D00085C0EC01C0902F02D0903002E090310290
:10A8E000F0903202A7019601688179818A819B816B
:10A8F0000E9428AE87FF04C0C882D982EA82FB8208
:10A90000C0903302D0903402E0903502F0903602CD
:10A91000A7019601688179818A819B810E942BB071
:10A92000181624F4C882D982EA82FB82C0903702CA
:10A93000D0903802E0903902F0903A02A7019601D7
:10A940006C817D818E819F810E9428AE87FF04C02B
:10A95000CC82DD82EE82FF82C0903B02D0903C022E
:10A96000E0903D02F0903E02A70196016C817D814E
:10A970008E819F810E942BB0181624F4CC82DD8238
:10A98000EE82FF82C0903F02D0904002E0904102F0
:10A99000F0904202A7019601688579858A859B859A
:10A9A0000E9428AE87FF04C0C886D986EA86FB8647
:10A9B000C0904302D0904402E0904502F0904602DD
:10A9C000A7019601688579858A859B850E942BB0B1
:10A9D000181624F4C886D986EA86FB86DF91CF91C3
:10A9E000FF90EF90DF90CF9008958F929F92AF925B
:10A9F000BF92CF92DF92EF92FF9288EA95E05EDFFE
:10AA00008091A70383FD7DC0C090B405D090B505AB
:10AA1000E090B605F090B70520915E0230915F029C
:10AA20004091600250916102C701B6010E9428AEB8
:10AA3000882309F466C06091F4047091F504809154
:10AA4000F6049091F7042091C904211117C00E94C7
:10AA500097AE20911F02309120026217730774F4A1
:10AA6000C0925E02D0925F02E0926002F0926102B8
:10AA70000E946B168FEE94E10E945D168090B405E3
:10AA80009090B505A090B605B090B70520915E02F4
:10AA900030915F024091600250916102C501B401A2
:10AAA0000E944EAD6B017C0120E030E0A9010E94C4
:10AAB0002BB087FF04C0C701B601905802C0C70180
:10AAC000B60120916202309163024091640250917C
:10AAD00065020E9466B020E030E048E453E40E9442
:10AAE0002BB0181674F480925E0290925F02A092CE
:10AAF0006002B09261020E946B1680ED94E10E94A8
:10AB00005D1660914C0270914D02072E000C880B6F
:10AB1000990B0E94CAAE20914E0230914F02409193
:10AB20005002509151020E9466B02AE037ED43E294
:10AB30005CE30E9466B03FDD80E1E8EAF5E0A2E573
:10AB4000B2E001900D928A95E1F7FF90EF90DF90CF
:10AB5000CF90BF90AF909F908F9008951F93CF9309
:10AB6000DF93882329F0D091BA05D095D17001C028
:10AB7000D0E0662339F01091BA051695117081E086
:10AB8000182701C010E0442341F0C091BA05C2FB70
:10AB9000CC27C0F981E0C82701C0C0E0D11104C0B2
:10ABA000111102C0CC23D1F00E946B168AEC94E103
:10ABB0000E945D16DD2319F088E50E94C71B112352
:10ABC00019F089E50E94C71BCC2319F08AE50E9481
:10ABD000C71B82EC94E10E945D16C1E08C2FDF91CF
:10ABE000CF911F910895CF92DF92EF92FF92CF9372
:10ABF000DF93C82FD0E0FE01E154FB4E8491811118
:10AC000007C00E946B168DE994E10E945D168AE0F0
:10AC1000FE01EE0FFF1FEE0FFF1FE75EFA4EC5901D
:10AC2000D590E590F490682F70E080E090E00E946D
:10AC3000CAAE9B01AC01C701B6010E942FAEDF91E5
:10AC4000CF91FF90EF90DF90CF9008954F925F9259
:10AC50006F927F928F929F92AF92BF92CF92DF922C
:10AC6000EF92FF920F931F93CF93DF93CDB7DEB791
:10AC700068970FB6F894DEBF0FBECDBF2A013B0127
:10AC80006901E82EF12CF701EB5DFA4EE491AA245C
:10AC9000A3941E160CF4A12CBB24B39420E030E046
:10ACA000A901C301B2010E942BB018160CF0B12CFF
:10ACB00080E0DFD769837A838B839C8381E0D9D757
:10ACC0006D837E838F83988782E0D3D769877A8765
:10ACD0008B879C8783E0CDD76D877E878F87988B06
:10ACE000EE0CFF1CEE0CFF1C88248394912C8C0E20
:10ACF0009D1E8E0C9F1CF401108211821282138201
:10AD00009E01235F3F4FAE01475F5F4FBE016B5F08
:10AD10007F4FCE0101960E94ED6BF401408251827B
:10AD200062827382198A1A8A1B8A1C8A20E030E0A8
:10AD3000A901B801C6010E9428AE811108C0F7011F
:10AD4000E75EFA4E85919591A591B49102C0C80134
:10AD5000D6018D8B9E8BAF8BB88FCE0141966C0147
:10AD6000E12C8E010B5E1F4F9E01235F3F4FAE0112
:10AD7000475F5F4FBE016B5F7F4F40970E94A96A9C
:10AD80008CD7AB100E94B73268960FB6F894DEBF2E
:10AD90000FBECDBFDF91CF911F910F91FF90EF902C
:10ADA000DF90CF90BF90AF909F908F907F906F90EB
:10ADB0005F904F90089521E030E0082E01C0220FEF
:10ADC0000A94EAF79091B905922B9093B905909166
:10ADD000BA05292B2093BA0524E0829FC0011124D3
:10ADE000FC01E05CFA4E4591559165917491FC012E
:10ADF000EE5AFD4F408351836283738308954F92CF
:10AE00005F926F927F928F929F92AF92BF92FF92CA
:10AE10000F931F93CF93DF93833008F06AC0F82E0F
:10AE2000C82FD0E0FE01EB5DFA4E8491CC0FDD1F00
:10AE3000CC0FDD1FFE01EC5CFA4E459055906590FD
:10AE40007490682F880F770B880B990B0E94CAAEFD
:10AE50004B015C0120E030E040EC5FE3C301B20154
:10AE60000E9466B0A50194010E9466B0AB01BC01CE
:10AE700000E010E098018F2DE9DEFE01E85DFA4E5A
:10AE80002591359145915491C501B4010E9466B058
:10AE90004B015C0120E030E0A9010E9428AE88232C
:10AEA000C1F0B501A401705800E010E098018F2DA9
:10AEB000CDDE8F2D98DE2B013C01A5019401C5014B
:10AEC000B4010E944FADAB01BC01930182018F2DF3
:10AED000BDDE8F2D70DFBADAFE01E855FA4FCE5A8B
:10AEE000DD4F88819981AA81BB8180839183A28370
:10AEF000B383DF91CF911F910F91FF90BF90AF90DF
:10AF00009F908F907F906F905F904F90089580E119
:10AF1000E0EFF5E0DF01982F1D929A95E9F7E3EC59
:10AF2000F5E0DF01982F1D929A95E9F7ECEDF5E039
:10AF3000DF011D928A95E9F71092D8051092D90584
:10AF40001092DA051092DB058CE096E00E9406A7CD
:10AF50001092AC061092AF061092AD061092AE069B
:10AF60001092A90608954F925F926F927F928F92EE
:10AF70009F92AF92BF92CF92DF92EF92FF920F9388
:10AF80001F93CF93DF93CDB7DEB768970FB6F894D2
:10AF9000DEBF0FBECDBF8C015B014A01FC01EF5B40
:10AFA000FF4F60817181828193810E94C8AE6B01E5
:10AFB0007C01D5012D913D914D915C910E9466B02F
:10AFC0000E9415AE0E949CAE69877A878B879C870A
:10AFD000F4012081318142815381C701B6010E9471
:10AFE00066B00E9415AE0E949CAE6D877E878F87EB
:10AFF000988B29853A854B855C8528373105410535
:10B00000510540F488E790E0A0E0B0E089879A8796
:10B01000AB87BC872D853E854F85588928373105FC
:10B020004105510540F488E790E0A0E0B0E08D874D
:10B030009E87AF87B88B9801235B3F4FD9018D91D5
:10B040009D910D90BC91A02D89839A83AB83BC8385
:10B05000BC01CD010E94CAAE2B013C0169857A85F5
:10B060008B859C850E94C8AE698B7A8B8B8B9C8B61
:10B0700020E030E0A901C301B2010E9428AE88237C
:10B0800029F1A7019601C701B6010E9466B04B01E4
:10B090005C0129893A894B895C89CA01B9010E94FE
:10B0A00066B09B01AC01C501B4010E944EAD4B01DD
:10B0B0005C01A3019201C301B2010E944FAD9B014B
:10B0C000AC01C501B4010E942FAE03C060E070E086
:10B0D000CB010E9415AE0E949CAE6D837E838F8350
:10B0E000988769817A818B819C81909580957095F4
:10B0F00061957F4F8F4F9F4F0E94CAAE4B015C01FD
:10B100006D857E858F8598890E94C8AE69837A8314
:10B110008B839C8320E030E0A901C501B4010E942B
:10B1200028AE882349F129813A814B815C81CA018B
:10B13000B9010E9466B06D8B7E8B8F8B988FA701B3
:10B140009601C701B6010E9466B09B01AC016D89F2
:10B150007E898F89988D0E944EAD6B017C01A5017F
:10B160009401C501B4010E944FAD9B01AC01C70120
:10B17000B6010E942FAE03C060E070E0CB010E94D8
:10B1800005AFF80185A096A0A7A0B0A47501640141
:10B190002D813E814F815885C21AD30AE40AF50AEF
:10B1A0000E949CAEC61AD70AE80AF90AF7FE73C0D5
:10B1B00020E030E0A901C301B2010E9428AE88233B
:10B1C00009F443C0A3019201C301B2010E944FAD33
:10B1D0006B017C01C501B4010E94C8AE9B01AC01AA
:10B1E000C701B6010E9466B06B017C0129893A89CA
:10B1F0004B895C89CA01B9010E9466B09B01AC0110
:10B20000C701B6010E944EAD6B017C0129813A81D4
:10B210004B815C81CA01B9010E9466B09B01AC01FF
:10B22000C701B6010E944FAD6B017C0120E030E008
:10B2300040E850E4C301B2010E9466B09B01AC013A
:10B24000C701B6010E942FAE03C060E070E0CB01E1
:10B250000E9415AE7B016C0120E030E0A9010E9444
:10B260002BB0181624F0E12CF12CC12CD12CB701F5
:10B27000C6010E949CAE6D837E838F83988786165D
:10B280009706A806B90620F48D829E82AF82B88602
:10B29000C12CD12C76018D819E81AF81B885F801BA
:10B2A00081A792A7A3A7B4A7C80ED91EEA1EFB1EAA
:10B2B000C5A6D6A6E7A6F0AAEB5BFF4F29853A857F
:10B2C0004B855C85208331834283538334968D85FF
:10B2D0009E85AF85B88980839183A283B383689666
:10B2E0000FB6F894DEBF0FBECDBFDF91CF911F9197
:10B2F0000F91FF90EF90DF90CF90BF90AF909F9015
:10B300008F907F906F905F904F9008952F923F9213
:10B310004F925F926F927F928F929F92AF92BF9265
:10B32000CF92DF92EF92FF920F931F93CF93DF9311
:10B33000009709F471C08B01EC01D984CA847B8425
:10B340006C848D809E80AF80B8842D2D3C2D472D40
:10B35000562DC501B4010E9428AE811108C0011507
:10B36000110509F459C0F801808180FF55C088811A
:10B3700081FD34C00115110531F0F80125803680BA
:10B380004780508408C08BE0282E87ED382E83E25A
:10B39000482E8BE3582E89899A89AB89BC89BC01D8
:10B3A000CD0190589B01AC010E944FAD2D853E858B
:10B3B0004F8558890E9466B09B01AC01C201B10162
:10B3C0000E944EAD7B018C019B01AC016D2D7C2D4B
:10B3D000872D962D0E9428AE87FF04C0ED2CFC2CF3
:10B3E000072D162D9701A801C501B4010E9428AEB2
:10B3F000882391F0888181608883CE010E94AD37D7
:10B40000882321F088818E7F888306C0A701B80138
:10B410004D835E836F837887DF91CF911F910F916A
:10B42000FF90EF90DF90CF90BF90AF909F908F9064
:10B430007F906F905F904F903F902F900895FF9274
:10B440000F931F93CF93DF93C091AF06C150CF707E
:10B45000D091AD068091AF06D817E9F060E070E0BA
:10B4600086E5F82ECD17B9F0FC9E80011124005519
:10B47000194FF801808183FD03C0C80147DFB8017F
:10B48000C150CF708091AD06D81761F3CD1719F078
:10B49000DF5FDF70F7CFDF91CF911F910F91FF90AA
:10B4A00008954F925F926F927F928F929F92AF9288
:10B4B000BF92FF920F931F93CF93DF93009709F4EE
:10B4C00059C0F42EEB018C01FC01808181FD3CC050
:10B4D00045805680678070848D809E80AF80B88460
:10B4E000A5019401C301B2010E9428AE87FF2CC0C0
:10B4F000F80181899289A389B489BC01CD01905852
:10B500009B01AC010E944FADF8012585368547852A
:10B5100050890E9466B09B01AC01C301B2010E9438
:10B520004EAD2B013C01A50194010E9428AE87FF7E
:10B530000BC0888181608883CE010E94AD3788234B
:10B5400091F088818E7F888329853A854B855C853B
:10B550006D817E818F8198850E9428AE81110AC0FD
:10B56000F092AD0607C04D825E826F827886F092BF
:10B57000AD06EACFDF91CF911F910F91FF90BF9061
:10B58000AF909F908F907F906F905F904F900895B5
:10B59000CF92DF92EF92FF920F931F93CF93DF939F
:10B5A0001091AD06C0E0D0E086E5C82E8091AF06D0
:10B5B000181709F1C19EB0011124CB018055994F94
:10B5C0007C01FC01808183FD0AC00E2DDF2C2097B9
:10B5D00069F0CE010E94AD37882341F002C00C2FE4
:10B5E000DD2E1F5F1F70C02FDD2DE0CF412FB70173
:10B5F000CE0157DFF6CFDF91CF911F910F91FF90D2
:10B60000EF90DF90CF9008952F923F924F925F92EC
:10B610006F927F928F929F92AF92BF92CF92DF9262
:10B62000EF92FF920F931F93CF93DF93CDB7DEB7C7
:10B630002E970FB6F894DEBF0FBECDBF2091AC069B
:10B6400029873091AF063B8796E58B85E9858E1774
:10B6500059F08B8581508F70989FF0011124E0552F
:10B66000F94F208123FD0DC0812C912CA12CB12CF0
:10B670001A861C861D861E86212C312C00E010E0C7
:10B680001AC08B87E2CFF6E52985F29FC00111240D
:10B69000FC01E055F94F1F01808183FF11C0FA843E
:10B6A000EC84DD84CE8489858F5F8F708987FA86EC
:10B6B000EC86DD86CE86F9852B85F213E4CF93C028
:10B6C00065817681878190850E94D3B0F62EE72E22
:10B6D000D82EC92E0115110509F47FC0F80180810B
:10B6E00080FD04C0F101808180FF77C0F801808176
:10B6F00081608083C8010E94AD3781116AC0F80162
:10B7000061817281838194810E94D3B02B013C01BD
:10B710009B01AC0160E070E080E89FE30E942FAEE7
:10B720004B015C019B01AC016F2D7E2D8D2D9C2D5D
:10B730000E9466B069837A838B839C83A501940100
:10B740006A857C858D859E850E9466B06D837E832B
:10B750008F839887AE014F5F5F4FBE016B5F7F4F56
:10B76000C80101DCF80186A9882399F12091D3054D
:10B770003091D4054091D5055091D605FD96608154
:10B780007181828193810E9466B0209181063091FF
:10B79000820640918306509184060E9466B04B0158
:10B7A0005C019B01AC01C301B2010E9466B00E9422
:10B7B0009CAEF80172AF61AFA50194016F2D7E2D93
:10B7C0008D2D9C2D0E9466B00E949CAEF80174AF36
:10B7D00063AFF80180818E7F80838F2C9E2CAD2CEF
:10B7E000BC2C810160CF2114310409F473C0F10134
:10B7F000808181608083C8010E94AD37811166C05D
:10B80000F10161817281838194810E94D3B06B01C7
:10B810007C019B01AC0160E070E080E89FE30E9446
:10B820002FAE2B013C012DEC3CEC4CE45DE30E947F
:10B8300066B069837A838B839C83A3019201B401F0
:10B84000C5010E9466B06D837E838F839887AE01A9
:10B850004F5F5F4FBE016B5F7F4FC10184DBF10122
:10B8600086A9882399F12091D3053091D405409180
:10B87000D5055091D605FD966081718182819381B5
:10B880000E9466B020918106309182064091830625
:10B89000509184060E9466B04B015C019B01AC0193
:10B8A000C701B6010E9466B00E949CAEF10172AF62
:10B8B00061AF2DEC3CEC4CE45DE3C501B4010E94AA
:10B8C00066B00E949CAEF10174AF63AFF10180815C
:10B8D0008E7F80832E960FB6F894DEBF0FBECDBF4D
:10B8E000DF91CF911F910F91FF90EF90DF90CF905C
:10B8F000BF90AF909F908F907F906F905F904F9090
:10B900003F902F9008958091AF069091AD068150A1
:10B910008F70891711F093DD3BDE76CEAF92BF9228
:10B92000CF92DF92EF92FF920F931F93CF9390915C
:10B93000AF068091AC06981791F0E091AC0686E5D1
:10B94000E89FF0011124EF5FF84FC0818091AC06B1
:10B950009091AF06891729F08F5F8F70F9CFC09152
:10B96000EF04CC2339F10E94E0110091BF05109142
:10B97000C0052091C1053091C205DC01CB01011544
:10B9800011052105310571F48C599F4FAF4FBF4F01
:10B990008093BF059093C005A093C105B093C205E5
:10B9A000CFEF21C0801B910BA20BB30BB7FF1BC0C5
:10B9B000CFEF19C01092BF051092C0051092C105BB
:10B9C0001092C20560E070E020E04FEF50E088E0A8
:10B9D000CF911F910F91FF90EF90DF90CF90BF908C
:10B9E000AF900C94DB196C2F70E080E090E01F9218
:10B9F0001F921F922FEF2F9326E4A22EB12CC12C61
:10BA0000D12CE12CF12C8701EA9421E030E040E0D8
:10BA100050E00E94B6150F900F900F900F90D4CF6A
:10BA2000CF92DF92EF92FF920F931F93CF93DF930A
:10BA3000CDB7DEB728970FB6F894DEBF0FBECDBFE7
:10BA400020913006222309F44AC06A018B017C014F
:10BA500020E030E040E450E4FC01608171818281AB
:10BA600093810E944FAD6D837E838F83988720E002
:10BA700030E04EE353E4F80160817181828193816B
:10BA80000E944EAD69837A838B839C839601AE01BD
:10BA90004F5F5F4FBE016B5F7F4F8CE096E00E946F
:10BAA0003EA620E030E040E450E46D817E818F814D
:10BAB00098850E944EADF7016083718382839383E2
:10BAC00020E030E04EE353E469817A818B819C81F0
:10BAD0000E944FADF801608371838283938328961F
:10BAE0000FB6F894DEBF0FBECDBFDF91CF911F918F
:10BAF0000F91FF90EF90DF90CF9008950F931F93D9
:10BB0000CF93DF93CDB7DEB7AC970FB6F894DEBF17
:10BB10000FBECDBF20913006222309F450C08C0106
:10BB20006CE076E0CE0101960E94C1A720E030E0F3
:10BB300040E450E4F80160817181828193810E9428
:10BB40004FAD69A77AA78BA79CA720E030E04EE312
:10BB500053E4F80164817581868197810E944EAD1E
:10BB60006DA37EA38FA398A79801285F3F4FAE01D6
:10BB70004B5D5F4FBE01675D7F4FCE0101960E9416
:10BB80003EA620E030E040E450E469A57AA58BA50C
:10BB90009CA50E944EADF8016083718382839383DC
:10BBA00020E030E04EE353E46DA17EA18FA198A583
:10BBB0000E944FADF8016483758386839783AC96AA
:10BBC0000FB6F894DEBF0FBECDBFDF91CF911F91AE
:10BBD0000F91089580916F0081FB992790F981FF63
:10BBE00005C080916F008D7F80936F008091AC06BF
:10BBF0008093AF068093AD068093AE0684E6809373
:10BC0000A90628EE33E03093AB062093AA069923C9
:10BC100029F080916F00826080936F0081E08093B3
:10BC20007E0508950C94DC3DCF93C82F0E94053EFD
:10BC30000E94CAAE24E0C29FF0011124EF5BF94FCD
:10BC400020813181428153810E9466B0CF91089555
:10BC50009091AF068091AC06981719F00E94B6AC8F
:10BC6000F7CF8091AA069091AB06892BB9F70C9477
:10BC7000AAABCF93C82F0E94BE3D0E94CAAE24E05B
:10BC8000C29FF0011124EF5BF94F20813181428185
:10BC900053810E9466B0CF9108959091AF06809134
:10BCA000AC06981719F00E94B6ACF7CF8091AA069F
:10BCB0009091AB06892BB9F708952F923F924F923E
:10BCC0005F926F927F928F929F92AF92BF92CF922C
:10BCD000DF92EF92FF920F931F93CF93DF93CDB735
:10BCE000DEB7CE56D1090FB6F894DEBF0FBECDBF7A
:10BCF0001C01AB966FAFAB976E965FAF4EAF6E9772
:10BD000068963FAF2EAF68976596EFAE65972C9615
:10BD1000FFAE2C9769960FAF699761961FAF619739
:10BD20001C2D2E96BFAEAEAE2E97FA01808191816A
:10BD3000A281B3814091F0055091F1056091F20527
:10BD40007091F305841B950BA60BB70B89A79AA7D7
:10BD5000ABA7BCA784819581A681B7814091F405EA
:10BD60005091F5056091F6057091F705841B950BD0
:10BD7000A60BB70B8DA39EA3AFA3B8A78085918513
:10BD8000A285B3854091F8055091F9056091FA05B7
:10BD90007091FB05841B950BA60BB70B89A39AA387
:10BDA000ABA3BCA3C484D584E684F7848091FC054E
:10BDB0009091FD05A091FE05B091FF05A7019601A8
:10BDC000281B390B4A0B5B0B2BAB3CAB4DAB5EAB73
:10BDD000232B242B252B09F49AC06091F404709135
:10BDE000F5048091F6049091F7042091C904211183
:10BDF0002BC00E9497AE20911F0230912002621743
:10BE0000730714F5C092FC05D092FD05E092FE0583
:10BE1000F092FF056896EEADFFAD68978485958535
:10BE2000A685B7858093CF059093D005A093D105C3
:10BE3000B093D2050E946B1683E895E10E945D16CF
:10BE40001BAA1CAA1DAA1EAA6BA97CA98DA99EA922
:10BE50000E94CAAE24E0129FF0011124EE59FD4F5A
:10BE600020813181428153810E9466B06B017C0147
:10BE700020E030E0A9010E942BB087FF04C0F7FA50
:10BE8000F094F7F8F09460918106709182068091A9
:10BE90008306909184060E9497AE9B01AC01A8ECAA
:10BEA000B0E00E94C1B10E94CAAE9B01AC01C701C3
:10BEB000B6010E942BB0181654F56E96EEADFFAD8C
:10BEC0006E9784859585A685B7858093FC059093AC
:10BED000FD05A093FE05B093FF056896EEADFFAD9E
:10BEE000689784859585A685B7858093CF059093BF
:10BEF000D005A093D105B093D2050E946B1684E6BD
:10BF000095E10E945D161BAA1CAA1DAA1EAA49A49F
:10BF10005AA46BA47CA4D301C2018827B7FD8395E2
:10BF20009927AA27BB27082F8DA09EA0AFA0B8A451
:10BF3000B7FC0260C9A0DAA0EBA0FCA0F7FC04608B
:10BF40002BA93CA94DA95EA957FD08606BA97CA946
:10BF50008DA99EA90E94CAAE34E0139FF00111245E
:10BF6000EE59FD4F20813181428153810E9466B09C
:10BF70006FA778AB89AB9AAB20E030E0A9010E94B3
:10BF80002BB087FF06C06FA578A989A99AA99058F8
:10BF900004C06FA578A989A99AA920E030E040E003
:10BFA0005FE30E944FAD0E949CAE2B966CAF7DAFBD
:10BFB0008EAF9FAF2B97D1011C92D5960C934FAAB1
:10BFC00058AE69AE7AAE77FE0BC022273327A9019F
:10BFD00024193509460957092FAB38AF49AF5AAF75
:10BFE0008FA998ADA9ADBAADF101858B968BA78BC2
:10BFF000B08F23968CAE9DAEAEAEBFAE2397B7FE8C
:10C000000DC022273327A901281939094A095B09DC
:10C0100023962CAF3DAF4EAF5FAF239723968CADE9
:10C020009DADAEADBFAD2397F101818F928FA38FF0
:10C03000B48F2796CCAEDDAEEEAEFFAE2797F7FEFF
:10C040000DC022273327A9012C193D094E095F098C
:10C0500027962CAF3DAF4EAF5FAF279727968CAD9D
:10C060009DADAEADBFAD2797F101858F968FA78FA0
:10C07000B0A3C301B2010E94CAAE20914106309123
:10C08000420640914306509144060E9466B06BAF51
:10C090007CAF8DAF9EAF698B7A8B8B8B9C8BC501F0
:10C0A000B4010E94CAAE20914506309146064091E7
:10C0B0004706509148060E9466B02B013C016D8BEB
:10C0C0007E8B8F8B988FC701B6010E94CAAE2091DC
:10C0D000490630914A0640914B0650914C060E9409
:10C0E00066B04B015C01698F7A8F8B8F9C8F20919A
:10C0F0004D0630914E0640914F06509150066FA567
:10C1000078A989A99AA90E9466B06B017C016D8FFC
:10C110007E8F8F8F98A32FA938AD49AD5AAD2630A9
:10C1200031054105510554F523968CAD9DADAEAD5D
:10C13000BFAD23970697A105B10504F527962CAD51
:10C140003DAD4EAD5FAD2797263031054105510518
:10C15000ACF420E030E0A901C701B6010E942BB089
:10C1600087FF04C0F7FAF094F7F8F094D1011D9618
:10C17000CD92DD92ED92FC92509752C02E96EEAD8C
:10C18000FFAD2E97C080D180E280F38020E030E0C8
:10C19000A901C701B6010E9428AE882341F0D10150
:10C1A0001D96CD92DD92ED92FC9250972BC02BAD57
:10C1B0003CAD4DAD5EADCA01B9010E9466B06B01E8
:10C1C0007C01A3019201C301B2010E9466B09B01F0
:10C1D000AC01C701B6010E944FAD6B017C01A50106
:10C1E0009401C501B4010E9466B09B01AC01C70176
:10C1F000B6010E944FAD0E94D3B0F10165877687EA
:10C200008787908B71019E012F5D3F4FAE014B5D83
:10C210005F4FBE01675D7F4F86E694E00E94E01DA0
:10C220002B96CCACDDACEEACFFAC2B97D10191964C
:10C23000CD92DD92ED92FC92949755964D915D9141
:10C240006D917C9158975D96CD90DD90ED90FC902E
:10C25000909759968D919D910D90BC91A02D8C1524
:10C260009D05AE05BF0510F4D701C60184179507DB
:10C27000A607B70710F4DB01CA012B96CCACDDACE6
:10C28000EEACFFAC2B978C159D05AE05BF0510F4E9
:10C29000D701C601F10185A396A3A7A3B0A706976E
:10C2A000A105B105B0F18091EF04EF5AFF4F8083F3
:10C2B000452B462B472B09F01798F101818D928D64
:10C2C000A38DB48D892B8A2B8B2B09F01698F10145
:10C2D000858D968DA78DB0A1892B8A2B8B2B09F08C
:10C2E00015982B96CCACDDACEEACFFAC2B97CD28E3
:10C2F000CE28CF28D1F08091D705882319F081501E
:10C300008093D705111108C0149880E28093D70557
:10C3100003C080E00C94CA69E090A106F090A206E8
:10C320000091A3061091A40608C0E090A506F09025
:10C33000A6060091A7061091A8069701A801659688
:10C340006FAD65972C967FAD2C9769968FAD6997E9
:10C3500061969FAD61970E9428AE87FD02C00C9444
:10C36000BC69D1011D962D913D914D915C915097E5
:10C370006C962CAF3DAF4EAF5FAF6C9760E070E056
:10C3800080E89FE30E942FAE60966CAF7DAF8EAFCA
:10C390009FAF60979B01AC01B701C8010E9466B0D6
:10C3A0004B015C018091AF069091AE06891B8F70A6
:10C3B0002C968FAF2C97A501940160E074E284E77E
:10C3C00099E40E942FAE0E9436B06B017C012C963E
:10C3D0008FAD2C9782508630C0F580917106909178
:10C3E0007206A0917306B0917406C816D906EA06C3
:10C3F000FB0658F58C199D09AE09BF09BC01CD019A
:10C40000660F771F881F991F2C96BFAD2C970B2F97
:10C4100010E020E030E0A90198010E9466B1CA0155
:10C42000B9010E94C8AE0E9436B06C0D7D1D8E1DF4
:10C430009F1D0E94C8AE9B01AC0160E074E284E7DE
:10C4400099E40E942FAE4B015C01A50194016C960A
:10C450006CAD7DAD8EAD9FAD6C970E9466B09B01BB
:10C46000AC010E9466B0A2966CAF7DAF8EAF9FAF5D
:10C47000A297F1016183728383839483C5A0D6A0C0
:10C48000E7A0F0A42396CCAEDDAEEEAEFFAE2397D0
:10C49000C701B6010E94C8AE27966CAF7DAF8EAFC4
:10C4A0009FAF2797A50194010E9466B00E9415AE28
:10C4B0000E949CAEA6966CAF7DAF8EAF9FAFA69745
:10C4C000F101EF5BFF4F6083718382839383FE01F1
:10C4D0007196FCAFEBAF9E012F5F3F4F66963FAF6B
:10C4E0002EAF669745E856E0A8965FAF4EAFA89787
:10C4F000CE0181969EA78DA762963FAF2EAF629721
:10C500001FA61FAA00E81FE3ABADBCAD6D917D91E6
:10C510008D919D91BCAFABAFA50194010E9466B017
:10C520006B017C016296EEADFFAD629761937193F2
:10C53000819391936296FFAFEEAF629720E030E077
:10C54000A9010E942BB087FF04C0F7FAF094F7F816
:10C55000F094A896AEADBFADA8974D905D906D904C
:10C560007D90A896BFAFAEAFA897A3019201C70177
:10C57000B6010E942BB01816A4F4A7019601C301BE
:10C58000B2010E942FAE6B017C019B01AC016FA533
:10C590007FA9C8010E942BB018161CF4CFA6DFAAF1
:10C5A0008701CBACDCACEDA4FEA4CE14DF0409F013
:10C5B000ABCF20E030E040E85FE36FA57FA9C80182
:10C5C0000E9428AE87FF4BC06E0121E1C20ED11C34
:10C5D0006696EEACFFAC66972FA53FA9A801D701E0
:10C5E0006D917D918D919C910E9466B0F701619350
:10C5F0007193819391937F01EC15FD0569F77101AA
:10C60000F1E4EF0EF11CA6966CAD7DAD8EAD9FAD45
:10C61000A6970E94C8AE2FA53FA9A8010E9466B0A8
:10C620000E949CAED7016D937D938D939C9313973D
:10C630002FA53FA9A8016FA57FA9C8010E9466B0D8
:10C640009B01AC01A2966CAD7DAD8EAD9FADA29766
:10C650000E9466B0F1016183728383839483609644
:10C660002CAD3DAD4EAD5FAD609727966CAD7DAD09
:10C670008EAD9FAD27970E9466B06BAF7CAF8DAF3C
:10C680009EAFD10155968D909D90AD90BC905897DE
:10C690005D96CD90DD90ED90FC909097CFA6D8AAB6
:10C6A000E9AAFAAA5996CD90DD90ED90FC905C979E
:10C6B000CFAAD8AEE9AEFAAE81149104A104B104B8
:10C6C00001F5CD28CE28CF28E1F4CFA4D8A8E9A839
:10C6D000FAA8CD28CE28CF28A1F420919906309130
:10C6E0009A0640919B0650919C060E9466B00E945B
:10C6F00015AE0E949CAE2B013C01D101D6961C9236
:10C7000008C32B96CCACDDACEEACFFAC2B97CD28A0
:10C71000CE28CF2849F060919506709196068091B9
:10C7200097069091980608C060919D0670919E06AC
:10C7300080919F069091A0062BAD3CAD4DAD5EADB6
:10C740000E9466B00E9415AE0E949CAE2B013C0177
:10C750002B96CCACDDACEEACFFAC2B97CD28CE2825
:10C76000CF28C9F020E030E0A9016091D305709195
:10C77000D4058091D5059091D6050E9428AE8823D6
:10C7800051F081E0CBA8DCA8EDA8FEA81C141D0484
:10C790001E041F040CF080E0D101D6968C938823F0
:10C7A00009F4CAC02091C3053091C4054091C50564
:10C7B0005091C6056896EEADFFAD689760817181B6
:10C7C000828193810E944EAD6BAB7CAB8DAB9EABF7
:10C7D0002091C7053091C8054091C9055091CA05FF
:10C7E0006896AEADBFAD689714966D917D918D91B1
:10C7F0009C9117970E944EAD2B966CAF7DAF8EAF7C
:10C800009FAF2B972091CB053091CC054091CD0562
:10C810005091CE056896EEADFFAD68976085718545
:10C82000828593850E944EAD6B017C012BA93CA9AA
:10C830004DA95EA9CA01B9010E9466B06BAB7CAB81
:10C840008DAB9EAB2B962CAD3DAD4EAD5FAD2B971A
:10C85000CA01B9010E9466B09B01AC016BA97CA919
:10C860008DA99EA90E944FAD6BAB7CAB8DAB9EABEF
:10C87000A7019601C701B6010E9466B09B01AC01F9
:10C880006BA97CA98DA99EA90E944FAD0E94D3B02F
:10C890006B017C012091CF053091D0054091D105ED
:10C8A0005091D2056896AEADBFAD68971C966D915C
:10C8B0007D918D919C911F970E944EADA70196018D
:10C8C0000E942FAE6B017C01F101FD9660837183A4
:10C8D0008283938320E030E040E450E40E942BB058
:10C8E00018161CF4F10116AA27C02091D305309127
:10C8F000D4054091D5055091D605C701B6010E94D7
:10C9000066B09B01AC0160913D0670913E0680913E
:10C910003F06909140060E942FAE2BAD3CAD4DAD31
:10C920005EAD0E9466B00E949CAE641575058605DA
:10C93000970510F42B013C018091EC059091ED05D9
:10C94000A091EE05B091EF05F101C1A0D2A0E3A046
:10C95000F4A0CBAADCAAEDAAFEAA2396CCACDDAC4F
:10C96000EEACFFAC23978C159D05AE05BF0508F412
:10C97000D1C081149104A104B10431F12091510678
:10C9800030915206409153065091540624153505B6
:10C9900046055705C8F4C701B6010E9430B16B01C6
:10C9A0007C01A3019201C501B4010E9430B1C616F9
:10C9B000D706E806F90640F4C701B601A5019401BF
:10C9C0000E9466B129013A01CFA8D8ACE9ACFAAC13
:10C9D000CD28CE28CF2871F12091550630915606EA
:10C9E00040915706509158062415350546055705C0
:10C9F00008F523966CAD7DAD8EAD9FAD23970E945B
:10CA000030B16B017C01A30192016FA978AD89ADB2
:10CA10009AAD0E9430B1C616D706E806F90650F462
:10CA2000C701B6012FA938AD49AD5AAD0E9466B114
:10CA300029013A01CFA4D8A8E9A8FAA8CD28CE2880
:10CA4000CF2871F12091590630915A0640915B062A
:10CA500050915C06241535054605570508F52396C3
:10CA60006CAD7DAD8EAD9FAD23970E9430B16B0153
:10CA70007C01A30192016FA578A989A99AA90E94B6
:10CA800030B1C616D706E806F90650F4C701B6015C
:10CA90002FA538A949A95AA90E9466B129013A01CE
:10CAA000CBA8DCA8EDA8FEA8CD28CE28CF2809F475
:10CAB00030C120915D0630915E0640915F06509135
:10CAC0006006241535054605570508F022C1239652
:10CAD0006CAD7DAD8EAD9FAD23970E9430B16B01E3
:10CAE0007C01A30192016BA97CA98DA99EA90E943A
:10CAF00030B1C616D706E806F90608F00AC1C70124
:10CB0000B6012BA93CA94DA95EA90E9466B12901D5
:10CB10003A01FFC081149104A104B104B9F16091FC
:10CB200051067091520680915306909154066415F7
:10CB300075058605970550F50E94C8AE27962CAD61
:10CB40003DAD4EAD5FAD27970E9466B06B017C0195
:10CB5000C501B4010E94C8AE4B015C01C301B20122
:10CB60000E94C8AEA50194010E9466B0A70196017B
:10CB70000E942BB0181654F4A5019401C701B60108
:10CB80000E942FAE0E949CAE2B013C01CFA8D8ACD6
:10CB9000E9ACFAACCD28CE28CF28C9F16091550672
:10CBA0007091560680915706909158066415750548
:10CBB0008605970560F50E94C8AE27962CAD3DAD61
:10CBC0004EAD5FAD27970E9466B06B017C016FA9E7
:10CBD00078AD89AD9AAD0E94C8AE4B015C01C3012E
:10CBE000B2010E94C8AEA50194010E9466B0A701DF
:10CBF00096010E942BB0181654F4A5019401C701A8
:10CC0000B6010E942FAE0E949CAE2B013C01CFA426
:10CC1000D8A8E9A8FAA8CD28CE28CF28C9F16091D4
:10CC2000590670915A0680915B0690915C066415D6
:10CC300075058605970560F50E94C8AE27962CAD50
:10CC40003DAD4EAD5FAD27970E9466B06B017C0194
:10CC50006FA578A989A99AA90E94C8AE4B015C0169
:10CC6000C301B2010E94C8AEA50194010E9466B042
:10CC7000A70196010E942BB0181654F4A501940147
:10CC8000C701B6010E942FAE0E949CAE2B013C0151
:10CC9000CBA8DCA8EDA8FEA8CD28CE28CF28C9F1C6
:10CCA00060915D0670915E0680915F0690916006CE
:10CCB000641575058605970560F50E94C8AE279630
:10CCC0002CAD3DAD4EAD5FAD27970E9466B06B01B8
:10CCD0007C016BA97CA98DA99EA90E94C8AE4B01BD
:10CCE0005C01C301B2010E94C8AEA50194010E947B
:10CCF00066B0A70196010E942BB0181654F4A50146
:10CD00009401C701B6010E942FAE0E949CAE2B0178
:10CD10003C01F101E35BFF4F4082518262827382EA
:10CD2000C301B2010E94C8AE6B017C012BAD3CADCA
:10CD30004DAD5EAD0E942FAE64966CAF7DAF8EAFF1
:10CD40009FAF6497D10151966D937D938D939C9382
:10CD500054972DEB37E346E051E4C701B6010E943A
:10CD600066B00E949CAEF10161AB72AB83AB94AB39
:10CD700086A9882381F1FD962081318142815381EA
:10CD80006091D3057091D4058091D5059091D60519
:10CD90000E9466B064962CAD3DAD4EAD5FAD64971C
:10CDA0000E9466B0209181063091820640918306F0
:10CDB000509184060E9466B09B01AC0160E074E271
:10CDC00084EF99E40E942FAE0E949CAED101D896C8
:10CDD0007C936E93D797D1011196CD90DD90ED9015
:10CDE000FC901497A296CCAEDDAEEEAEFFAEA2974D
:10CDF000C701B6010E94D3B06FAB28967FAF2897CA
:10CE00008FAF24969FAF2497E1E3F6E0A496FFAF9F
:10CE1000EEAFA4973E01F1E16F0E711C21E336E005
:10CE20002E963FAF2EAF2E9766964EAC5FAC6697B0
:10CE30006BAB7FA7182F092F1BAED201CD90DD90D1
:10CE4000ED90FD902D0120E030E0A901C701B60171
:10CE50000E942BB087FF04C0F7FAF094F7F8F09423
:10CE60002E96EEADFFAD2E9781909190A190B1904E
:10CE70002E96FFAFEEAF2E97A5019401C701B60124
:10CE80000E942BB018160CF043C0FBADFF2349F1F4
:10CE9000A50194016FA928967FAD28978FAD2496A0
:10CEA0009FAD24970E9466B04B015C012BA93FA562
:10CEB000412F502FC701B6010E9466B0A501940111
:10CEC0000E942BB0181614F5A7019601C501B401F4
:10CED0000E942FAE6BAB7FA7182F092F21E02BAF3D
:10CEE00017C0A7019601C501B4010E942FAE9B0196
:10CEF000AC016BA97FA5812F902F0E9466B06BAB10
:10CF00007FA7182F092F31E03BAF02C041E04BAFA4
:10CF10004614570409F091CFCBA8AC96CFAEAC978E
:10CF2000DFA4AD96DFAEAD97AE961FAFAE97AF96CE
:10CF30000FAFAF972C96EFAC2C97EE2009F475C18C
:10CF4000C090D805D090D905E090DA05F090DB05C7
:10CF50002DEB37E346E855E3C701B6010E9428AE42
:10CF600087FD63C1C701B6010E94D3B06B017C018C
:10CF70009B01AC016FA928967FAD28978FAD2496B1
:10CF80009FAD24970E9428AE87FD08C0CFAA28969F
:10CF9000DFAE2897EFAE2496FFAE24979601A70147
:10CFA0006FA928967FAD28978FAD24969FAD2497C3
:10CFB0000E942FAEAA966CAF7DAF8EAF9FAFAA979F
:10CFC0002CED35E02E963FAF2EAF2E97C12CD12CF5
:10CFD00080E8E82E8FE3F82ECBAEDCAEEDAEFEAEF1
:10CFE0002C961FAE2C972E96AEADBFAD2E976D91A1
:10CFF0007D918D919D912E96BFAFAEAF2E97AA9643
:10D000002CAD3DAD4EAD5FADAA970E9466B06B01F1
:10D010007C016696EEADFFAD669781909190A190F0
:10D02000B1906696FFAFEEAF66972C96FFAD2C974A
:10D03000FF2391F02BAD3CAD4DAD5EAD0E9466B0CF
:10D040006B017C012BAD3CAD4DAD5EADC501B401B6
:10D050000E9466B04B015C01A5019401C701B601B5
:10D060000E942BB020E030E0A90118164CF5C50154
:10D07000B4010E942BB018164CF020E030E0A9015A
:10D08000C701B6010E9428AE87FF09C0A50194011F
:10D09000C701B6010E944EAD2B013C0139C02401ED
:10D0A000350177FA709477F87094A3019201C70163
:10D0B000B6010E942BB018165CF52601370128C076
:10D0C000C501B4010E9428AE87FD09C020E030E010
:10D0D000A901C701B6010E942BB018164CF4A70194
:10D0E0009601C501B4010E944EAD2B013C0110C058
:10D0F0002601370177FA709477F87094A5019401AE
:10D10000C301B2010E942BB0181614F0240135019E
:10D11000A496AEADBFADA497CD90DD90ED90FD90FF
:10D12000A496BFAFAEAFA497A7019601C301B20109
:10D130000E942BB01816CCF4A3019201C701B601CE
:10D140000E942FAE9B01AC016BAD7CAD8DAD9EAD51
:10D150000E9466B06BAF7CAF8DAF9EAF2C96BFAD1B
:10D160002C97BF5F2C96BFAF2C972E96EEADFFADE0
:10D170002E97EC5EF54009F036CF2C96CFAC2C976D
:10D18000CC20B1F02BAD3CAD4DAD5EAD6FA9289676
:10D190007FAD28978FAD24969FAD24970E9466B0EF
:10D1A0006FAB28967FAF28978FAF24969FAF2497B9
:10D1B00024EA30E74DE75FE36FA928967FAD289713
:10D1C0008FAD24969FAD24970E9466B06B017C01C1
:10D1D0009B01AC016091BB057091BC058091BD05C0
:10D1E0009091BE050E942BB01816ACF4A7019601D1
:10D1F0006BA97FA5812F902F0E942BB01816ACF041
:10D20000FFA8FBAA2896CFAC2897CFA61FAD2496DF
:10D210000FAD24970AC0DFA8DBAA2896EFAC2897A9
:10D22000EFA61FAD24960FAD2497AC968FADAC97AB
:10D23000AD969FADAD97AE96AFADAE97AF96BFAD85
:10D24000AF978093BB059093BC05A093BD05B093A9
:10D25000BE052BA93FA5412F502F6BA97FA5812F7C
:10D26000902F0E9466B07B018C01CB01D801F101A7
:10D2700081879287A387B48764966CAD7DAD8EADB0
:10D280009FAD649790589B01AC010E944FAD6C9686
:10D290002CAD3DAD4EAD5FAD6C970E9466B09B016D
:10D2A000AC016BE077ED83E29BE30E944EAD5B0146
:10D2B0006C01AB96FFADAB97FF2361F09B01AC0116
:10D2C000B701C8010E9428AE87FD09C09A2D8B2D99
:10D2D000860107C09BE087ED03E21BE302C09E2DA1
:10D2E0008F2D492F582FB801D10115964D935D937D
:10D2F0006D937C9318971C919501A601A2966CAD35
:10D300007DAD8EAD9FADA2970E9428AE181614F485
:10D3100081E001C083E0182BF101108380E1FE0160
:10D320003196ACEDB5E001900D928A95E1F7F101EF
:10D3300081819281A381B4818093D8059093D9058E
:10D34000A093DA05B093DB0580E16E96EEADFFADFC
:10D350006E97A0EFB5E001900D928A95E1F780E11C
:10D360006896EEADFFAD6897A3ECB5E001900D9225
:10D370008A95E1F781E00EC06596EFAC65972C9633
:10D38000FFAC2C9769960FAD699761961FAD6197B9
:10D390000C94B161C259DF4F0FB6F894DEBF0FBED7
:10D3A000CDBFDF91CF911F910F91FF90EF90DF9054
:10D3B000CF90BF90AF909F908F907F906F905F9035
:10D3C0004F903F902F9008956F927F928F929F92EF
:10D3D000AF92BF92CF92DF92EF92FF920F931F9383
:10D3E000CF93DF9300D01F92CDB7DEB74C013B0146
:10D3F0008091AA069091AB06892BD9F59091AF0642
:10D400008091AC06981B9F709F3059F429833A8312
:10D410004B835C830E94B6AC5C814B813A8129814D
:10D42000EDCFD090AF068091AF0666E5869FC00134
:10D4300011245701C02E79018A019301A40160E0F3
:10D440008055994F0E945D5E8823A9F02091AF0618
:10D450009091AC06291303C094E69093A90691E03D
:10D460009D0D9F709093AF0689830E94835C898194
:10D4700003C080E001C081E00F900F900F900F90EB
:10D48000DF91CF911F910F91FF90EF90DF90CF90A0
:10D49000BF90AF909F908F907F906F9008958091F4
:10D4A000AF069091AC06891B8F708F3019F40E94E3
:10D4B000B6ACF5CF8091AF068F5F8F70E091AF066D
:10D4C00096E59E9FF0011124E055F94FDF011D9272
:10D4D0009A95E9F798E090834091F0055091F10515
:10D4E0006091F2057091F305458B568B678B708FB9
:10D4F0004091F4055091F5056091F6057091F7059E
:10D50000418F528F638F748F4091F8055091F905C8
:10D510006091FA057091FB05458F568F678F70A358
:10D520004091FC055091FD056091FE057091FF054D
:10D5300041A352A363A374A32091AF069091AC06BC
:10D54000291303C094E69093A9068093AF060C9428
:10D5500091342F923F924F925F926F927F928F926F
:10D560009F92AF92BF92CF92DF92EF92FF920F9372
:10D570001F93CF93DF93CDB7DEB7A9970FB6F8947B
:10D58000DEBF0FBECDBFF801A091AA06B091AB06D9
:10D59000AB2B09F0A7C016010E2DF8A7EFA33EA3F1
:10D5A0002DA36A017B01FC01408051806280738061
:10D5B0002091750630917606409177065091780655
:10D5C000C301B2010E9466B00E9436B0698B7A8BAB
:10D5D0008B8B9C8BD7018D909D90AD90BC902091B2
:10D5E000790630917A0640917B0650917C06C50100
:10D5F000B4010E9466B00E9436B06D8B7E8B8F8B1B
:10D60000988FD6012D913D914D915C9129A33AA31C
:10D610004BA35CA320917D0630917E0640917F064E
:10D620005091800669A17AA18BA19CA10E9466B04D
:10D630000E9436B0698F7A8F8B8F9C8FEDA1FEA1EF
:10D64000C080D180E280F3802091810630918206F3
:10D650004091830650918406C701B6010E9466B0CE
:10D660000E9436B06D8F7E8F8F8F98A349825A8229
:10D670006B827C828D829E82AF82B88629A13AA17C
:10D680004BA15CA129873A874B875C87CD86DE86D4
:10D69000EF86F88A2091A70323FF10C06093FC0552
:10D6A0007093FD058093FE059093FF05C092CF0512
:10D6B000D092D005E092D105F092D205AFA1B8A5E5
:10D6C0002D913D914D915C917101BE016F5F7F4F36
:10D6D000CE01419679DE882331F089A70E949134EA
:10D6E00089A501C080E0A9960FB6F894DEBF0FBEF1
:10D6F000CDBFDF91CF911F910F91FF90EF90DF9001
:10D70000CF90BF90AF909F908F907F906F905F90E1
:10D710004F903F902F900895AF92BF92CF92DF929B
:10D72000EF920F931F93CF93DF93CDB7DEB764973C
:10D730000FB6F894DEBF0FBECDBFA98ABA8ACB8AD6
:10D74000DC8AFC0180819181A281B38189839A83E3
:10D75000AB83BC83FB0180819181A281B3818D83E6
:10D760009E83AF83B887FA0180819181A281B381C2
:10D7700089879A87AB87BC87F90180819181A281D3
:10D78000B3818D879E87AF87B88BAE01475F5F4FB0
:10D79000BE016B5F7F4FCE0101960E94105DCE01EE
:10D7A00041966C019E01235F3F4FAE01475F5F4F83
:10D7B000BE016B5F7F4F4097CCDE64960FB6F89446
:10D7C000DEBF0FBECDBFDF91CF911F910F91EF90C4
:10D7D000DF90CF90BF90AF9008958F929F92AF92BD
:10D7E000BF92EF92FF920F931F93CF93DF937B0132
:10D7F0008A01E901FC0180809180A280B3802091A0
:10D800007506309176064091770650917806C501ED
:10D81000B4010E9466B00E9436B06093F005709328
:10D82000F1058093F2059093F305209179063091EC
:10D830007A0640917B0650917C06F70160817181E8
:10D84000828193810E9466B00E9436B06093F40595
:10D850007093F5058093F6059093F70520917D066A
:10D8600030917E0640917F0650918006F8016081DC
:10D870007181828193810E9466B00E9436B060936C
:10D88000F8057093F9058093FA059093FB052091B4
:10D89000810630918206409183065091840668810A
:10D8A00079818A819B810E9466B00E9436B0609324
:10D8B000FC057093FD058093FE059093FF05809213
:10D8C000C3059092C405A092C505B092C605F701A4
:10D8D00080819181A281B3818093C7059093C8050F
:10D8E000A093C905B093CA05F80180819181A281F6
:10D8F000B3818093CB059093CC05A093CD05B093D5
:10D90000CE0588819981AA81BB818093CF059093B0
:10D91000D005A093D105B093D2059091AF06809128
:10D92000AC06981759F0DF91CF911F910F91FF909E
:10D93000EF90BF90AF909F908F90B1CD0E944D5EC1
:10D9400080916F0081FBCC27C0F981FF05C08091D9
:10D950006F008D7F80936F002CEF35E048EF55E02E
:10D9600064EF75E080EF95E00E94C137CC2329F089
:10D9700080916F00826080936F00DF91CF911F9143
:10D980000F91FF90EF90BF90AF909F908F90089570
:10D99000CF93DF93CDB7DEB760970FB6F894DEBFB5
:10D9A0000FBECDBFFC0180819181A281B3818983AB
:10D9B0009A83AB83BC83FB0180819181A281B38177
:10D9C0008D839E83AF83B887FA0180819181A28184
:10D9D000B38189879A87AB87BC87F9018081918160
:10D9E000A281B3818D879E87AF87B88BAE01475FD9
:10D9F0005F4FBE016B5F7F4FCE0101960E94105DAD
:10DA00009E01235F3F4FAE01475F5F4FBE016B5FDB
:10DA10007F4FCE010196E1DE60960FB6F894DEBF2F
:10DA20000FBECDBFDF91CF910895CF92DF92EF92DD
:10DA3000FF92FC01C080D180E280F38020918106BA
:10DA4000309182064091830650918406C701B60149
:10DA50000E9466B00E9436B06093FC057093FD058D
:10DA60008093FE059093FF05C092CF05D092D0051C
:10DA7000E092D105F092D2059091AF068091AC066C
:10DA8000981729F0FF90EF90DF90CF9008CD0E947B
:10DA90004D5E80916F0081FB992790F981FF05C051
:10DAA00080916F008D7F80936F004091FC055091B5
:10DAB000FD056091FE057091FF054093210550938F
:10DAC00022056093230570932405992329F0809102
:10DAD0006F00826080936F00FF90EF90DF90CF9097
:10DAE0000895CF92DF92EF92FF920F931F93CF93FF
:10DAF000DF93C1E6D6E001E516E0C12CD12C76011A
:10DB0000C39469917991899199910E94C8AE2889AD
:10DB100039894A895B890E9466B00E949CAEF801EF
:10DB200061937193819391938F01C616D706E8068E
:10DB3000F90610F46B017C01F6E0C137DF0709F745
:10DB40006FEF7FEFCB01A70196010E9466B1209392
:10DB5000EC053093ED054093EE055093EF05DF9112
:10DB6000CF911F910F91FF90EF90DF90CF9008958C
:10DB70000F931F93CF93DF9305E716E0C1E4D6E040
:10DB8000F80121913191419151918F0160E070E054
:10DB900080E89FE30E942FAE6993799389939993CC
:10DBA000F6E0C135DF0761F72EE532E04AE552E0E5
:10DBB00066E572E082E592E0EBDEDF91CF911F91A6
:10DBC0000F918FCF80E19CE00C94875781548A316C
:10DBD00008F041C0A82FB0E04091390C50913A0CA8
:10DBE00060913B0C70913C0C04C0769567955795FD
:10DBF00047958A95D2F740FF2EC0E091440CF091F2
:10DC0000450CA15EB34F8C918823E9F0E80FF11D1C
:10DC1000808190ED980F9A3098F08E3211F48181C6
:10DC20000CC08D3211F08B3271F4818190ED980F20
:10DC30009A3030F08E3239F4828180538A3018F471
:10DC40009E2F8F2F02C090E080E09093400C809335
:10DC5000410C81E0089580E00895B8DF882341F009
:10DC600081E02091400C3091410C232B09F480E09D
:10DC700008950F931F93CF938091400C9091410C86
:10DC8000009711F1FC018F01C1912C2F2F7DA9F07C
:10DC9000C53411F0C536B9F7F801108260E070E0C4
:10DCA0008091400C9091410C0E94CBB1F801C0834F
:10DCB000562F472F382F292F0BC060E070E0CF91EF
:10DCC0001F910F910C94CBB150E040E030E020E088
:10DCD000652F742F832F922FCF911F910F9108954D
:10DCE0008091400C9091410C009731F04AE050E057
:10DCF00060E070E00C9431B360E070E0CB01089517
:10DD0000CF9384E5AADF882359F1EADF97FD24C089
:10DD1000E7DF6F3F71058105910509F0FCF4E0DF55
:10DD2000C62F1616FCF40E946B168DE40E94C71BCA
:10DD30006AE070E080913D0C90913E0C0E94BA1C0C
:10DD40006C2FCC0F770B86EF95E10E948E168AE040
:10DD50000E94C71B8FEF07C0C0E004C0CFEF02C016
:10DD600080E001C08C2FCF910895BF92CF92DF92B7
:10DD7000EF92FF920F931F93CF93DF9388EAE82EE1
:10DD800085E0F82E02E512E096E1C92E9CE0D92E3E
:10DD9000CBE4D3E0BC2E84E0B80E89915EDF88230B
:10DDA000B1F067DFF6012081211104C02091B80590
:10DDB000222339F0F80120813181428153810E9470
:10DDC0004FADF70160837183828393830AC0F801AA
:10DDD00080819181A281B381F70180839183A283A5
:10DDE000B383F4E0EF0EF11C0C5F1F4F8FEFC81AE6
:10DDF000D80ABC12D2CF86E430DF8823B9F039DFED
:10DE000020E030E0A9010E942BB018167CF431DF2D
:10DE100020E030E040E752E40E942FAE60934E02D3
:10DE200070934F028093500290935102DF91CF91F3
:10DE30001F910F91FF90EF90DF90CF90BF900895CA
:10DE4000CF92DF92EF92FF926B017C010E94E01172
:10DE5000C60ED71EE81EF91E0E94E011DC01CB01A0
:10DE60008C199D09AE09BF09B7FF03C00E94B6AC6B
:10DE7000F3CFFF90EF90DF90CF9008956F927F9255
:10DE80008F929F92AF92BF92CF92DF92EF92FF92CA
:10DE90000F931F93CF93DF93CDB7DEB73C01A090D4
:10DEA000440CB090450CCDB6DEB66AE070E0C3011C
:10DEB0000E949EB57C01009721F08C01061917097C
:10DEC00004C0C3010E94A9B58C01C80101962DB7F9
:10DED0003EB7281B390B0FB6F8943EBF0FBE2DBFBF
:10DEE0008DB79EB701964C01A801B3010E94CAB537
:10DEF000F401E00FF11F1082C40148D581E034D055
:10DF0000E114F10451F037019FEF691A790A0FB655
:10DF1000F894DEBE0FBECDBEC6CF0FB6F894DEBEFF
:10DF20000FBECDBEC501DF91CF911F910F91FF9024
:10DF3000EF90DF90CF90BF90AF909F908F907F90A9
:10DF40006F9024C5CF93C3E00E944F89882341F08E
:10DF5000C15019F00E94BDABF7CFCF910C94EAAB42
:10DF60008FED95E1CF918ACFCF93C82F41E04093B9
:10DF7000150C90913F0C9D3409F45EC0943509F462
:10DF8000F7C1973409F0F8C120913D0C30913E0C57
:10DF90002B31310509F43EC0CCF42430310544F472
:10DFA0002230310564F537FDE7C10E94F198E7C1E1
:10DFB0002C30310561F12531310509F4E0C12430FF
:10DFC000310509F0D9C10E94FA98D9C12A35310525
:10DFD00051F154F42D31310521F1FCF02E31310590
:10DFE00009F0CAC151D2CBC12C35310511F1F4F081
:10DFF000293A314009F0C0C10E940587C0C181E0C3
:10E000002230310509F080E00E94379DB8C10E949E
:10E010000594B5C10E940994B2C180E00E94B97D07
:10E02000AEC190DFACC11092B805A9C14093B8054C
:10E03000A6C10E94D47BA3C120913D0C30913E0C1F
:10E040002937310509F45DC10CF083C0283631054C
:10E0500009F42AC10CF044C02C34310509F421C163
:10E0600004F52231310509F43EC164F437FD84C161
:10E07000223031050CF40DC12131310509F07CC18C
:10E080009ED77DC12A32310509F405C12B343105F3
:10E0900009F404C12F31310509F06EC10E94AD7A37
:10E0A0006EC12335310509F41BC16CF421353105EE
:10E0B00009F411C10CF011C12D34310509F05CC116
:10E0C0000E94EB795CC12535310509F40EC10CF4D1
:10E0D0000AC12C35310509F04FC10E9498954FC1F6
:10E0E0002037310509F44BC1CCF42C36310509F445
:10E0F00046C15CF42A36310509F4E7C00CF0E8C0EB
:10E100000E948BA31092150C41C12E36310509F4E3
:10E11000CEC00CF0CFC00E9404A331C12537310519
:10E1200009F4E8C06CF42237310509F4E0C00CF4BE
:10E13000C3C02337310509F01FC10E94667B1FC190
:10E140002737310509F4D8C00CF0D9C00E941A7BDA
:10E1500016C12E3581E0380709F408C10CF04BC018
:10E16000233D310509F4D8C01CF5293C310509F4DB
:10E17000CAC07CF42B39310509F4A4C02E3B31050B
:10E1800009F49DC02C38310509F0F6C00E945BA24D
:10E19000F6C02C3C310509F4B9C02D3C310509F419
:10E1A000B8C02B3C310509F0E7C00E943297E7C0A8
:10E1B0002D3281E0380709F4B6C07CF42D3D3105DD
:10E1C00009F4ACC0223E310509F4ABC02C3D310549
:10E1D00009F0D2C00E944795D2C02F3281E03807A3
:10E1E00009F4A7C00CF4A2C02033314009F0C4C028
:10E1F0000E94D594C4C0243F81E0380709F4A8C028
:10E2000014F5223981E0380709F49AC06CF42039FA
:10E2100081E0380709F490C00CF090C02F353140F0
:10E2200009F0AAC0ABD5ABC0243A81E0380709F4A5
:10E2300089C0293A81E0380709F487C02A3931407A
:10E2400009F09AC09CC0283F81E0380709F486C0D5
:10E250004CF4263F81E0380709F47CC00CF07CC008
:10E2600010D58DC0243883E0380709F479C034F420
:10E270002335334009F080C040D281C02B3883E081
:10E28000380709F470C0273E334009F075C093D7B2
:10E2900076C0ACD274C00E94887971C00E94E779C0
:10E2A0006EC00E94E9796BC00E94E1A268C00E9422
:10E2B000BA7B65C00AD763C00E94D87A60C00E944A
:10E2C00074A25DC00E949AA25AC00E945AA357C06D
:10E2D0000E9484A354C05ED752C00E94EA984FC0E7
:10E2E0000E94ED984CC06DD64AC018D648C00E9416
:10E2F000167B45C07AD243C00E940E7B40C081D7B6
:10E300003EC082D73CC00E94039739C00E945797F5
:10E3100036C00E94CD9733C07CD731C00E947A941A
:10E320002EC0C0D52CC00E94539829C00E946C9664
:10E3300026C00E94A6A123C06AD721C09BD01FC0BF
:10E340009ED01DC00E9435881AC00E94637C17C0F1
:10E3500096D415C098D413C098D411C0BBD40FC0A4
:10E360000E948D930CC00E94559409C0D2D407C05E
:10E3700080913D0C1ED603C08EE19CE072D41092B9
:10E38000150CC11103C0CF910C94C19FCF9108957A
:10E39000CF93DF93C091C10E80E6C89FE0011124A6
:10E3A000C052D34F8091A70380FF05C00E946B1617
:10E3B000CE010E941E1CCE01E9D280E0DF91CF91F8
:10E3C000D3CDCF92DF92EF92FF920F931F930E94D3
:10E3D000E0116B017C018091E10E81112FC08091D1
:10E3E0006802882359F18091150C882339F14091F6
:10E3F000110C5091120C6091130C7091140C970138
:10E400008601041B150B260B370B37FD2CC0833000
:10E4100079F03CF4813094F00E946B168DEC95E11C
:10E420000BC0843059F40E946B168EE995E104C04C
:10E430000E946B1686EB95E10E945D1620916802A2
:10E4400030E0A8EEB3E00E94ACB1DC01CB018C0D52
:10E450009D1DAE1DBF1D8093110C9093120CA093B7
:10E46000130CB093140C1F910F91FF90EF90DF905D
:10E47000CF90089581E00E941A4F0C94FE5180E0E5
:10E480000E941A4F0C94FE518F929F92AF92BF92AE
:10E49000CF92DF92EF92FF920F931F93CF93DF9370
:10E4A000CDB7DEB728970FB6F894DEBF0FBECDBF4D
:10E4B000C0905202D0905302E0905402F090550266
:10E4C00088E5CBDB811108C020E030E0A901C7015D
:10E4D000B6010E944FAD01C0CCDB6D837E838F837C
:10E4E0009887C0905602D0905702E0905802F09062
:10E4F000590289E5B2DB811108C020E030E0A901B2
:10E50000C701B6010E944FAD01C0B3DB6B017C01B6
:10E5100069837A838B839C838D809E80AF80B8844F
:10E5200022ED30E040EE50EC0E942BB087FDD2C0CF
:10E5300027E030E04EE353E4C701B6010E9428AE65
:10E5400018160CF4C7C023EA31E040E450ECC501D2
:10E55000B4010E942BB087FDBDC027E030E042E24D
:10E5600053E4C501B4010E9428AE18160CF4B2C0E1
:10E5700027E030E041E253E4C501B4010E9428AE37
:10E5800018160CF4A7C027E030E041E253E4C701BD
:10E59000B6010E9428AE18160CF49CC080E00E94C0
:10E5A000BB1D0E94FE5385E458DB182F8823B1F071
:10E5B0008091400C9091410C892B09F489C090DB2B
:10E5C00097FD0FC08DDB6F3F71058105910509F047
:10E5D0004CF486DB61117CC040E005C085E4F6DACE
:10E5E00077C010E0412F01E021E0BE016F5F7F4F57
:10E5F000CE0105960E94BB4F6B017C019B01AC01D3
:10E600000E9414B181115FC08D809E80AF80B8845C
:10E6100020E030E0A901C501B4010E9428AE87FDC9
:10E6200005C027E137EB41E558E304C027E137EBAC
:10E6300041E558EBC501B4010E944FADAB01BC01EF
:10E6400083E196E10E94A81689809A80AB80BC8005
:10E6500020E030E0A901C501B4010E9428AE87FD89
:10E6600005C027E137EB41E558E304C027E137EB6C
:10E6700041E558EBC501B4010E944FADAB01BC01AF
:10E680008EE096E10E94A81620E030E0A901C701C3
:10E69000B6010E9428AE87FD05C027E137EB41E5B2
:10E6A00058E304C027E137EB41E558EBC701B60159
:10E6B0000E944FADAB01BC0189E096E10E94A81613
:10E6C0008AE00E94C71B0E941D540E94FE5102C096
:10E6D00041E089CF28960FB6F894DEBF0FBECDBFBC
:10E6E000DF91CF911F910F91FF90EF90DF90CF902E
:10E6F000BF90AF909F908F900895EF92FF920F93ED
:10E700001F93CF93DF938AE561DA882309F456C01B
:10E710008091400C9091410C009709F44FC0FC018E
:10E720007F01C1912C2F2F7D89F0C53411F0C536A2
:10E73000B9F7F701108260E070E08091400C909191
:10E74000410C0E94CBB1F701C08304C060E070E0CF
:10E750000E94CBB18B01D82FC92F20E030E040E0E0
:10E7600050EC0E942BB087FD1DC020E030E040EA55
:10E7700050E4B8018D2F9C2F0E9428AE181694F0FB
:10E78000C801AD2FBC2F8093920590939305A09361
:10E790009405B0939505DF91CF911F910F91FF9054
:10E7A000EF9008950E946E168CE296E1DF91CF9172
:10E7B0001F910F91FF90EF900C945D160E946B16C5
:10E7C0004091920550919305609194057091950543
:10E7D0008BE196E10E94A8168AE0DF91CF911F910C
:10E7E0000F91FF90EF900C94C71B0895CF92DF928A
:10E7F000EF92FF920F931F93CF93DF93C091420C40
:10E80000D091430C80E529DA8823D1F08091400C27
:10E810009091410C009749F04AE050E060E070E0D0
:10E820000E9459B46B017C0103C0C12CD12C76012C
:10E8300011E0C114D104E104F10431F410E004C08A
:10E8400010E0C12CD12C760183E507DA882309F486
:10E8500086C08091400C9091410C009701F1FC0121
:10E860007F010191202F2F7D89F0053411F00536AD
:10E87000B9F7F701108260E070E08091400C909150
:10E88000410C0E94CBB1F701008304C060E070E04E
:10E890000E94CBB1B62FA72FF82FE92F04C0B0E00C
:10E8A000A0E0F0E0E0E020E030E04AE754E46B2F45
:10E8B0007A2F8F2F9E2F0E9466B00E949CAE6B0114
:10E8C0007C01111109C0672B682B692B29F4209753
:10E8D00019F08881811102C010E001C011E00E948E
:10E8E0004D5E112329F00E946B16CE010E941E1C62
:10E8F00083E08093150C81E08093E20EC114D10473
:10E90000E104F10429F10E94E011C60ED71EE81EB1
:10E91000F91E0E94E011DC01CB018C199D09AE09A2
:10E92000BF09B7FD0EC01092E20E81E08093150C76
:10E93000DF91CF911F910F91FF90EF90DF90CF90DB
:10E9400008958091E20E882371F30E94B6ACE1CF66
:10E950008091E20E882339F30E94B6ACF9CF1111F1
:10E96000BBCFB5CF1092430C1092420C8FE3809333
:10E970003F0C10923E0C10923D0C1092390C1092EC
:10E980003A0C10923B0C10923C0C08953F924F921F
:10E990005F926F927F928F929F92AF92BF92CF922F
:10E9A000DF92EF92FF920F931F93CF93DF931F920B
:10E9B0001F92CDB7DEB789839A83D4DF8981282F50
:10E9C0009A81392FF90180812F5F3F4F8032D1F337
:10E9D0008E34B1F4818190ED980F9A3020F08D3211
:10E9E00011F08B3269F43296DF0131962C9120536D
:10E9F0002A30D0F3CD01FC01019620812032D9F3D9
:10EA0000F093450CE093440C8F010F5F1F4F308053
:10EA10006AE270E0C8010E9400B6009731F0FC0184
:10EA2000319780818032E1F311828DE4381631F024
:10EA3000E4E53E1619F0F7E43F12FFC0F8018081CB
:10EA40000F5F1F4F8032D1F380538A3008F0F5C03A
:10EA500030923F0C10923E0C10923D0C4AE02091F7
:10EA60003D0C30913E0C429FC001439F900D1124FC
:10EA700090933E0C80933D0C3196DF0111972C91C1
:10EA8000022E000C330B20533109280F391F30930D
:10EA90003E0C20933D0C808180538A3000F3DF01CF
:10EAA00031968C918032D9F38DE438121AC02E3110
:10EAB000310591F03CF42731310571F02C313105ED
:10EAC00081F40AC02537310564F02737310524F079
:10EAD000203AE3E03E0729F4B093430CA093420CA4
:10EAE000ACC01092430C1092420C5091440CC12CBB
:10EAF000D12C7601C394FD0131964C91442309F445
:10EB00009CC04132A9F48DE4381212C02032310584
:10EB100079F4F093430CE093420C63E270E0CF0190
:10EB20000E9400B6009709F488C0FC01108285C0DD
:10EB300041544A3108F055C0BF01FB0180816F5F2D
:10EB40007F4F8032D1F390ED980F9A3008F18E32DA
:10EB500011F481810CC08D3211F08B3259F4818116
:10EB600090ED980F9A30A0F08E3221F4828180537C
:10EB70008A3070F08091420C9091430C892B09F0FF
:10EB800059C0CF0101979093430C8093420C52C01F
:10EB9000CF01A42FB0E04601570104C0880C991C96
:10EBA000AA1CBB1C4A95D2F74090390C50903A0CE5
:10EBB00060903B0C70903C0C84289528A628B728C0
:10EBC0008092390C90923A0CA0923B0CB0923C0C83
:10EBD000009711F0851B01C080E0A15EB34F8C93BC
:10EBE0000AC08091420C9091430C892B21F4B09380
:10EBF000430CA093420C808181548A3130F4DF01B0
:10EC00007ACF80ED890F8A3040F44E2F6F2F91918B
:10EC10009111F7CF842F962F07C083ED890F823093
:10EC2000A0F39B3291F3F6CFFC0101964081403274
:10EC3000D9F3E5CF80E090E0ACCF0F900F90DF915B
:10EC4000CF911F910F91FF90EF90DF90CF90BF90E9
:10EC5000AF909F908F907F906F905F904F903F907C
:10EC600008950E946B166091440C7091450C8AE4E3
:10EC700096E10E94711687E496E10C945D160C945F
:10EC8000D7400C94134F0C94C744CF9383E50E9454
:10EC9000E66DC82F882331F08091400C9091410C93
:10ECA000892B41F483E50E94E66DC1E08C2FCF9162
:10ECB0000C94304615D897FD0BC012D86F3F7105E4
:10ECC0008105910509F094F70BD8C1E06111EECFF1
:10ECD000C0E0ECCF0E940C4F882331F00E946B16ED
:10ECE0008DE596E10C945D1608950E94706E97FD77
:10ECF0000CC00E94706E6F3F71058105910509F08F
:10ED000034F40E94706E862F089580E008958FEF8E
:10ED100008950F931F93CF9383E50E94E66D8111B1
:10ED200004C00FE413E0C0E00DC0C0E0DEDF682FD8
:10ED30008C2F0E944F3FCF5FC530C1F7F2CFCF5F1E
:10ED4000C43069F0F80181918F010E94E66D88233B
:10ED5000B1F3CBDF682F8C2F0E944F3FF0CF82E4BE
:10ED60000E94E66D882329F0C0DF682F84E00E94AE
:10ED70004F3FCF911F910F910C94FC3F0F931F9326
:10ED8000CF9383E50E942D6E882309F465C0ADDF23
:10ED9000823029F1833009F43FC0813009F05CC032
:10EDA0000FE413E0C0E0F80181918F010E942D6E05
:10EDB000882339F09ADF2FEF4FEF682F8C2F0E94B6
:10EDC000F83ECF5FC43079F782E40E942D6E88232D
:10EDD00009F442C08ADF2FEF4FEF682F3AC00FE4EB
:10EDE00013E0C0E0F80181918F010E942D6E88230D
:10EDF00039F07BDF2FEF482F6FEF8C2F0E94F83E0A
:10EE0000CF5FC43079F782E40E942D6E882321F110
:10EE10006CDF2FEF482F1CC00FE413E0C0E0F801B7
:10EE200081918F010E942D6E882339F05EDF282F9B
:10EE30004FEF6FEF8C2F0E94F83ECF5FC43079F711
:10EE400082E40E942D6E882339F04FDF282F4FEF88
:10EE50006FEF84E00E94F83ECF911F910F910C94C8
:10EE6000FC3FCF93DF931F921F92CDB7DEB769832C
:10EE70007A830E94E66D69817A81882361F08091AE
:10EE8000400C9091410C009731F04AE050E060E076
:10EE900070E00E9431B3972F862F0F900F90DF9173
:10EEA000CF9108951F93CF93DF9380E50E94E66D85
:10EEB000882381F160E070E080E5D3DF182F6FEFE9
:10EEC0007FEF83E5CEDFEC010196039718F517FD80
:10EED00021C00E944D5ECF3F8FEFD80729F02197C8
:10EEE00071F4C1E0D0E00DC0812F0E94341431E0F4
:10EEF00020E0892B09F030E0C32FD22F02C0C0E000
:10EF0000D0E0812F0E9434148C179D0719F00E94C5
:10EF1000B6ACF7CFDF91CF911F9108950F931F9358
:10EF2000CF9383E50E94E66D882309F43EC080916B
:10EF3000400C9091410C009701F1FC018F01C191AF
:10EF40002C2F2F7D89F0C53411F0C536B9F7F801A3
:10EF5000108260E070E08091400C9091410C0E9422
:10EF6000CBB1F801C08304C060E070E00E94CBB177
:10EF7000B62FA72FF82FE92F04C0B0E0A0E0F0E0F3
:10EF8000E0E020E030E04AE754E46B2F7A2F8F2F47
:10EF90009E2F0E9466B00E949CAE6093DD0E70931F
:10EFA000DE0E8093DF0E9093E00ECF911F910F91B4
:10EFB000089520E040E050E0BA010C9440340C94F5
:10EFC000A3AB0F931F93CF9383E50E94E66D882335
:10EFD00091F18091400C9091410C009761F1FC01FE
:10EFE0008F01C1912C2F2F7D89F0C53411F0C536CA
:10EFF000B9F7F801108260E070E08091400C9091C8
:10F00000410C0E94CBB1F801C08304C060E070E005
:10F010000E94CBB120E030E04AE754E40E9466B0A1
:10F020000E949CAE6093690270936A0280936B02A7
:10F0300090936C0246C088E50E94E66D811114C071
:10F0400089E50E94E66D81110FC08AE50E94E66D98
:10F0500081110AC085E40E94E66D811105C0CF913F
:10F060001F910F910C94285E0E944D5E88E50E94CE
:10F07000E66D882331F0179A8091B9058E7F8093D1
:10F08000B90589E50E94E66D882331F0169A8091D2
:10F09000B9058D7F8093B9058AE50E94E66D8823C6
:10F0A00031F0159A8091B9058B7F8093B90585E47D
:10F0B0000E94E66D882329F0CF911F910F910C9447
:10F0C000A8ABCF911F910F910895FF920F931F93BB
:10F0D000CF93DF9383E50E94E66D8823F1F083E50B
:10F0E0000E94E66D811102C060E015C08091400C65
:10F0F0009091410C892BC1F30E94706E97FDF4CF63
:10F100000E94706E6F3F71058105910511F00CF042
:10F110003FC00E94706E6093A7030E946B168CE93B
:10F1200096E10E945D168091A703882329F102E9E8
:10F1300016E1C0E0D0E020E08091A70390E00C2E23
:10F1400002C0959587950A94E2F780FF0EC0FF24D0
:10F15000F394F20E222319F08CE20E94C71BF801EF
:10F16000859194910E945D162F2D21960E5F1F4F61
:10F17000C530D10509F704C08EE896E10E945D16FE
:10F180008AE0DF91CF911F910F91FF900C94C71BE4
:10F190006FEFC1CF0E94F4250E94F3A80E94285E61
:10F1A00060E070E080E00E94842068EE73E080E020
:10F1B00090E00C941B1681E080936E0283E50E9420
:10F1C000E66D882331F08091400C9091410C892BA1
:10F1D00039F483E50E94E66D811112C00C9420A0E1
:10F1E0000E94706E97FDFACF0E94706E6F3F71059E
:10F1F0008105910509F024F40E94706E662371F375
:10F20000089581E00C94DD3280E00C94DD320C94A2
:10F210004D5ECF930E946B1683EC96E10E945D16C3
:10F2200083E50E94E66DC82F8823D1F08091400CC1
:10F230009091410C892B91F00E94706E97FD0DC04A
:10F240000E94706E6F3F71058105910509F034F4DD
:10F250000E94706EC1E0611101C0C0E0C09347021E
:10F26000809147020E94E2168BEB96E10E945D16A8
:10F2700040912F0250913002609131027091320220
:10F2800089EB96E10E94A81640913702509138020E
:10F290006091390270913A0286EB96E10E94A816BD
:10F2A00040913F02509140026091410270914202B0
:10F2B00083EB96E10E94A8168BEA96E10E945D1608
:10F2C00040913302509134026091350270913602C0
:10F2D00089EA96E10E94A81640913B0250913C02B7
:10F2E00060913D0270913E0286EA96E10E94A81666
:10F2F0004091430250914402609145027091460250
:10F3000083EA96E10E94A8168AE0CF910C94C71B6D
:10F310000F931F93CF93DF9383E50E942D6E882375
:10F3200009F450C0E2DC182F80E50E942D6E811197
:10F330000AC081E0111101C080E0DF91CF911F91DF
:10F340000F910C94051680E50E942D6E882331F0F4
:10F350000E94706EEB0177FD35C002C0CDE0D0E0B9
:10F360000C2F89E40E942D6E882351F08091400C6F
:10F370009091410C892B49F0B8DC811106C017C06F
:10F3800089E40E94E66D882391F061E08C2F0E9451
:10F39000C913612F8C2F0E940514612F70E08C2FF0
:10F3A0000E94AC12083071F41093EF040BC0802F50
:10F3B0000E946CAB882349F3DF91CF911F910F918D
:10F3C0000C9494ABDF91CF911F910F9108950C9401
:10F3D0006CA90C9408A90C94F3A84F925F926F92B9
:10F3E0007F92AF92BF92CF92DF92EF92FF92CF9334
:10F3F000DF93EB01FC0160817181828193812CE3B9
:10F40000C22ED12CE12CF12CA70196010E9466B1ED
:10F41000B62EA72ECA01B901A70196010E9466B1B6
:10F420006B017C01CA01B90128E130E040E050E005
:10F430000E9466B12B013C01C9016DE671E00E949A
:10F440003FB161157105D9F0AF92BF92DF92CF92B3
:10F450005F924F929F938F937F936F938BEF96E181
:10F460009F938F93DF93CF930E942BB68DB79EB758
:10F470000E960FB6F8949EBF0FBE8DBF61C0009769
:10F48000C9F0AF92BF92DF92CF925F924F929F935B
:10F490008F938BEE96E19F938F93DF93CF930E9490
:10F4A0002BB6EDB7FEB73C960FB6F894FEBF0FBE75
:10F4B000EDBF46C04114510461047104B9F0AF922C
:10F4C000BF92DF92CF925F924F928FED96E19F9322
:10F4D0008F93DF93CF930E942BB68DB79EB70A967A
:10F4E0000FB6F8949EBF0FBE8DBF2AC0C114D104C1
:10F4F000E104F104A9F0AF92BF92DF92CF9287EDC1
:10F5000096E19F938F93DF93CF930E942BB6EDB735
:10F51000FEB738960FB6F894FEBF0FBEEDBF10C011
:10F52000AF92BF9283ED96E19F938F93DF93CF933A
:10F530000E942BB60F900F900F900F900F900F908E
:10F54000DF91CF91FF90EF90DF90CF90BF90AF9081
:10F550007F906F905F904F900895CF93DF93CDB7DA
:10F56000DEB769970FB6F894DEBF0FBECDBF0E941D
:10F5700038A96E8B7F8B888F998FBE016F5F7F4F0D
:10F58000CE0146962ADF0E946B16BE016F5F7F4F49
:10F590008FE097E10E9471168AE00E94C71B69966E
:10F5A0000FB6F894DEBF0FBECDBFDF91CF910895A7
:10F5B00083E50E94E66D882331F08091400C9091A4
:10F5C000410C892B71F40E946B164091680250E047
:10F5D00060E070E08CE197E10E94D2168AE00C9422
:10F5E000C71B0E94706E97FD17C00E94706E6F3F20
:10F5F00071058105910509F01CF40E94706E01C02F
:10F600006FEF862F90E0CD971CF460936802089509
:10F610008CE380936802089560E0F3CF81E00E945C
:10F6200005160E94443380E00C9405160E944D5E3E
:10F630000C94FE511F93CF93DF93C091420CD09155
:10F64000430C83E010E040E08150C9F09881292FFD
:10F650002B7F2134C9F729812133B1F7913421F06F
:10F66000953419F441E001C011E09E012E5F3F4F37
:10F67000E9012F5F3F4F98819032D1F3E5CF4111DF
:10F680000E946B16112321F083E297E10E945D1620
:10F69000CE01DF91CF911F910C941E1C0F931F93ED
:10F6A000CF938C01C62F87E297E10E945D16C801B7
:10F6B0000E945D168AE30E94C71B6AE070E08C2FEF
:10F6C00090E0CF911F910F910C94C01C80E598E1C0
:10F6D0000E945D1660E080E498E1E0DF60E08BE28C
:10F6E00098E1DCDF61E084E298E1D8DF60E089E165
:10F6F00098E1D4DF61E089E098E1D0DF60E080E06C
:10F7000098E1CCDF61E086EF97E1C8DF61E08CEE45
:10F7100097E1C4DF61E084EE97E1C0DF61E086ED50
:10F7200097E1BCDF60E088EC97E1B8DF60E089EB4F
:10F7300097E1B4DF60E08BEA97E1B0DF60E085E954
:10F7400097E1ACDF61E084E897E1A8DF60E085E75E
:10F7500097E1A4DF60E080E697E1A0DF61E08DE45F
:10F7600097E19CDF60E080E497E198DF60E08CE265
:10F7700097E194CF8EE40E94E66D8823A1F08091FA
:10F78000400C9091410C009771F04AE050E060E02D
:10F7900070E00E9431B36093C30E7093C40E8093E7
:10F7A000C50E9093C60E08954F925F926F927F920E
:10F7B0009F92AF92BF92CF92DF92EF92FF920F9300
:10F7C0001F93CF93DF9383E5E82E83E0F82E02E5C5
:10F7D00012E0B12C912CA12CF70181917F010E94A4
:10F7E000E66D882309F450C08091400C9091410C43
:10F7F000009709F449C0FC013F01C1912C2F2F7DD6
:10F8000089F0C53411F0C536B9F7F301108260E014
:10F8100070E08091400C9091410C0E94CBB1F301BB
:10F82000C08304C060E070E00E94CBB16B01D82FB0
:10F83000C92FF80120813181428153810E944EAD50
:10F840002B013C012DEB37E346E855EB0E942BB032
:10F8500087FD0AC02DEB37E346E855E3C301B2014B
:10F860000E9428AE181684F4F3E0BF1619F099240C
:10F87000939402C0AA24A394A6016D2F7C2FF801B3
:10F880004083518362837383B3940C5F1F4FF4E012
:10F89000BF12A2CF992019F00E94265203C0A110D6
:10F8A0000E943052DF91CF911F910F91FF90EF9006
:10F8B000DF90CF90BF90AF909F907F906F905F90C0
:10F8C0004F900C94FE51BF92CF92DF92EF92FF9235
:10F8D0000F931F93CF93DF9337E5E32E33E0F32E9F
:10F8E00007E614E06701C0E0D0E0BB24B394F60162
:10F8F00081916F010E94E66D882359F10E944D5E4F
:10F900008091400C9091410C892B19F00E94396E26
:10F9100018C0F8016081662389F070E080E090E013
:10F920000E94CAAE9B01AC01FE01E659FB4F60810B
:10F930007181828193810E942FAE03C060E070E0EC
:10F94000CB01FE01EA58FB4F60837183828393836E
:10F95000B12C24960F5F1F4FCC30D10541F686E4C1
:10F960000E94E66D882381F10E944D5E0E94396EEF
:10F970008B01D82FC92F20E030E040E85FE30E94E0
:10F980002BB018167CF020E030E0A901B8018D2FD3
:10F990009C2F0E9428AE87FF09C000E010E0D0E055
:10F9A000C0E004C000E010E0D0E8CFE320E030E0A9
:10F9B0004FE753E4B8018D2F9C2F0E9466B00E9440
:10F9C0009CAE60938204B12C83E50E94E66D88238F
:10F9D00069F00E944D5E0E94396E60931002709330
:10F9E00011028093120290931302B9C0BB2009F454
:10F9F000B6C081E19AE10E945D1680918204811176
:10FA000004C08EE09AE10E945D1685E09AE10E94B2
:10FA10005D1680918204F4E68F9FC0011124815805
:10FA20009F4F6FEF70E00E9453B170E080E090E074
:10FA30000E94C8AE20E030E048EC52E40E942FAEB5
:10FA4000AB01BC0181EE99E10E94A81684EC99E11A
:10FA50000E945D1682EA99E10E945D1606E714E0B5
:10FA6000C7E5D3E023E0D22EDE0C80E20E94C71B64
:10FA700089910E94C71BF8016191719181919191C7
:10FA80008F0142E050E00E94451D8AE00E94C71BA2
:10FA9000DC12EBCF409110025091110260911202E2
:10FAA000709113028EE799E10E94A8168AE00E94E5
:10FAB000C71B8CE599E10E945D168091670488233D
:10FAC00049F00AE614E0C7E6D4E0CE0193E0D92E6F
:10FAD000D80E31C0809168048111F3CF8091690400
:10FAE0008111EFCF88E499E10E945D162CC080E27D
:10FAF0000E94C71BF70180810E94C71B6881662393
:10FB0000F1F070E080E090E00E94CAAE9B01AC0191
:10FB1000F80160817181828193810E942FAE42E061
:10FB200050E00E94451D2196FFEFEF1AFF0A0C5F7F
:10FB30001F4FDC1641F088818823A9F3D8CF60E0FD
:10FB400070E0CB01ECCF8AE0DF91CF911F910F9154
:10FB5000FF90EF90DF90CF90BF900C94C71BDF9188
:10FB6000CF911F910F91FF90EF90DF90CF90BF90BA
:10FB700008952F923F924F925F926F927F928F9251
:10FB80009F92AF92BF92CF92DF92EF92FF920F932C
:10FB90001F93CF93DF93CDB7DEB769970FB6F89475
:10FBA000DEBF0FBECDBF182F81E00E9405168FE487
:10FBB0000E942D6E8823B9F08091400C9091410CE9
:10FBC000892BB1F00E94706E97FD18C00E94706E74
:10FBD0006F3F71058105910509F054F40E94706E24
:10FBE000611106C00BC08FE40E94E66D882331F0DE
:10FBF0009091BA059770973009F4D8C10E944D5E74
:10FC0000209130062F8B80E00E94BB1D0E94FE5386
:10FC100081E00E94F0321111E5C188E50E94E66D95
:10FC2000082F89E50E94E66D182F8AE50E94E66D8F
:10FC3000382E011105C0111108C0811106C0D2C1B2
:10FC4000112319F08111CEC1012F80E1E2E5F2E02C
:10FC5000A8EAB5E001900D928A95E1F7332019F0FA
:10FC600082E00E94FF5682E50E942D6E882371F18A
:10FC70008091400C9091410C009709F455C0FC0113
:10FC80005F012191322F3F7D99F0253411F0253607
:10FC9000B9F7D5011C9260E070E08091400C909122
:10FCA000410C298F0E94CBB1298DF501208304C01E
:10FCB00060E070E00E94CBB16B017C0120E030E09D
:10FCC000A9010E9428AE882379F106C0C12CD12C4D
:10FCD00030E8E32E40E4F42E011103C0112309F4AF
:10FCE00005C1C601D7018093B0059093B105A093DB
:10FCF000B205B093B30520915A0230915B02409156
:10FD00005C0250915D02B601C7010E942BB018162B
:10FD10005CF419821A821B821C82BE016F5F7F4FC6
:10FD200080EB95E00E94BF53002309F498C1112392
:10FD300009F4D4C010925602109257021092580241
:10FD400010925902109252021092530210925402D1
:10FD5000109255020E942652E5E2F5E12491288F87
:10FD6000E4E3F5E185909590A590B490E8E3F5E1A2
:10FD70004590559065907490A3019201C501B4011E
:10FD80000E942BB018162CF4A5019401C301B201F6
:10FD900004C0A3019201C501B4010E942FAE6B0102
:10FDA0007C01EDE1F5E185919591A591B4918D8767
:10FDB0009E87AF87B88BE9E1F5E185919591A59193
:10FDC000B491898B9A8BAB8BBC8B2D853E854F85EF
:10FDD0005889BC01CD010E9428AE87FD08C02D8442
:10FDE0009E859D8BAF85AE8BB889BD8707C029885E
:10FDF000EA89ED8BFB89FE8B2C892D87A701960163
:10FE0000C701B6010E9466B020E030E040E85FE341
:10FE10000E944FAD0E94D3B09B01AC01622D7D8941
:10FE20008E899D850E9466B069877A878B879C87BB
:10FE3000E6E2F5E1F49020E030E040EC5FE3C3015E
:10FE4000B2010E9466B02B013C016F2DFF0C770BB5
:10FE5000880B990B0E94CAAE9B01AC01C301B20191
:10FE60000E9466B069837A838B839C8320E030E0B4
:10FE700040EC5FE3C501B4010E9466B06B017C01F8
:10FE8000A88D6A2FAA0F770B880B990B0E94CAAE18
:10FE90009B01AC01C701B6010E9466B06D837E83F1
:10FEA0008F839887AE01475F5F4FBE016F5F7F4FC3
:10FEB000CE0105960E94DD530E94B7321092560281
:10FEC0001092570210925802109259021092520248
:10FED00010925302109254021092550280E00E9438
:10FEE000FF561123D1F081E00E94FF560E94265256
:10FEF00080E00E94F032011104C0812C912C540149
:10FF000006C0812C912C20EAA22E20ECB22E1111D9
:10FF10009DC0C12CD12C76019FC00E94265280E04A
:10FF20000E94F032C12CD12C7601812C912C90EAC8
:10FF3000A92E90ECB92E332009F459C019821A82E7
:10FF40001B821C8220E030E040E050E460915A02C5
:10FF500070915B0280915C0290915D020E944EADB7
:10FF60006D837E838F839887BE016F5F7F4FCE0145
:10FF700005960E94BF5320E030E0A901C501B401FD
:10FF80000E9428AE811133C020E030E0A901C701F2
:10FF9000B6010E9428AE81112AC00E94B2328F8918
:10FFA0000E94BB1D0E941D540E94FE5180E00E94D1
:10FFB000051669960FB6F894DEBF0FBECDBFDF9170
:10FFC000CF911F910F91FF90EF90DF90CF90BF9056
:10FFD000AF909F908F907F906F905F904F903F90E9
:10FFE0002F90089511E001E0332433942ECE19822E
:10FFF0001A821B821C82A7019601609156027091A1
:020000021000EC
:10000000570280915802909159020E944EAD6D8323
:100010007E838F839887A50194016091520270912D
:10002000530280915402909155020E944EAD69870F
:100030007A878B879C87AE014F5F5F4FBE016B5FF6
:100040007F4FCE0109960E94DD53A7CFC12CD12C42
:1000500080EAE82E80E4F82E311070CF8CCF111199
:1000600042CF0E94265280E00E94F032812C912CD7
:10007000540175016401F0CF80E1E2E5F2E0A8EA05
:10008000B5E001900D928A95E1F708954F925F9245
:100090006F927F928F929F92AF92BF92CF92DF9298
:1000A000EF92FF920F931F93CF93DF93CDB7DEB7FD
:1000B0002E970FB6F894DEBF0FBECDBF27013801D3
:1000C0002E874A875B876C877D878987D5DF8985FF
:1000D0002E854A855B856C857D858F3F51F094E048
:1000E000899FF0011124E855FA4F408351836283C0
:1000F00073832F3F51F0A4E02A9FF0011124E855AB
:10010000FA4F4082518262827382BFEFCB1651F068
:1001100084E0C89EF0011124E855FA4F8082918254
:10012000A282B3828090A8059090A905A090AA050C
:10013000B090AB0520E030E042E253E4C501B401E9
:100140000E9428AE87FF11C020E030E040E450EC70
:10015000C501B4010E942BB018166CF0812C912CB3
:1001600030E4A32E30ECB32E06C0812C912C22E279
:10017000A22E23E4B22E8092A8059092A905A09207
:10018000AA05B092AB054090AC055090AD056090CB
:10019000AE057090AF0520E030E04EE353E4C301BC
:1001A000B2010E9428AE87FF11C020E030E040EE8F
:1001B00050ECC301B2010E942BB018166CF0412C18
:1001C000512C90EE692E90EC792E06C0412C512CCA
:1001D0008EE3682E83E4782E4092AC055092AD05F4
:1001E0006092AE057092AF058091B0059091B10517
:1001F000A091B205B091B3058D839E83AF83B8877C
:1002000020E030E04FE153E4BC01CD010E9428AE74
:1002100087FF11C020E030E040E050EC6D817E812E
:100220008F8198850E942BB018166CF080E090E0CA
:10023000A0E0B0EC04C080E090E0AFE1B3E48D83D7
:100240009E83AF83B8878D819E81AF81B88580936F
:10025000B0059093B105A093B205B093B30580E0CB
:1002600090E0A8E4B2E489839A83AB83BC83DE0187
:1002700011966D01ED80FE800F811885A30192011A
:10028000C501B4010E940B532E960FB6F894DEBF41
:100290000FBECDBFDF91CF911F910F91FF90EF90D7
:1002A000DF90CF90BF90AF909F908F907F906F9096
:1002B0005F904F9008958F929F92AF92BF92CF928E
:1002C000DF92EF92FF920F931F93CF93DF93EC0196
:1002D0006A017B0120E030E040E45FE368857985D6
:1002E0008A859B850E944FADA70196010E944FAD64
:1002F000AB01BC01812C912C5401CC24CA94850102
:1003000074012FEF82E0C2DEEC80FD800E811F8140
:10031000488159816A817B8121E080E0B7DEDF91ED
:10032000CF911F910F91FF90EF90DF90CF90BF90F2
:10033000AF909F908F9008952F923F924F925F922F
:100340006F927F928F929F92AF92BF92CF92DF92E5
:10035000EF92FF920F931F93CF93DF93CDB7DEB74A
:100360002E970FB6F894DEBF0FBECDBF89878B01E5
:100370004A87222359F0812C912C90E8A92E9EE3E4
:10038000B92E80E090E0A0EAB1E40CC08AE0882EAB
:1003900087ED982E83E2A82E8CE3B82E80E090E0C3
:1003A000A0E8BFE389839A83AB83BC83211105C096
:1003B00080E090E0A0EAB0E404C080E090E0A8E42F
:1003C000B2E48D839E83AF83B88756DE412C512CD7
:1003D0003201B985A4E0BA9FC0011124FC01E8559F
:1003E000FA4F1F01C801110FAA0BBB0B8B879C870B
:1003F000AD87BE872D813E814F815885C301B201F3
:100400000E9428AE87FF3FC06B857C858D859E85C9
:100410000E94CAAEA50194010E9466B09B01AC0186
:10042000D1016D917D918D919C910E944FADF10113
:100430006083718382839383E090B005F090B1056F
:100440000091B2051091B3052091AC053091AD0536
:100450004091AE055091AF056091A8057091A90536
:100460008091AA059091AB05DE0111966D010E9465
:100470000B530E944D5E83B182958170B1E08B2752
:10048000EA858E1324C0398524E0329FF0011124BF
:10049000E855FA4F60817181828193812E960FB663
:1004A000F894DEBF0FBECDBFDF91CF911F910F91AA
:1004B000FF90EF90DF90CF90BF90AF909F908F9084
:1004C0007F906F905F904F903F902F900895A5017F
:1004D0009401C301B2010E944FAD2B013C018ACFB0
:1004E0004F925F926F927F928F929F92AF92BF9244
:1004F000CF92DF92EF92FF920F931F93CF93DF93F0
:10050000CDB7DEB728970FB6F894DEBF0FBECDBFCC
:10051000B82E6B01A42E4901C801B701FF24F39442
:1005200020E030E040EA50E40E9428AE8111F12C36
:10053000A3DD84E0B89E80011124F801E855FA4F4C
:1005400080819181A281B3818D839E83AF83B8879F
:100550002F2D4A2DB6018B2DEFDE2B013C0181148E
:10056000910411F1F11020C041E04A256627772758
:100570006C197D0920E08B2DDFDEA30192010E9422
:100580004EAD6B017C0120E030E0A9010E942BB050
:1005900087FF04C0F7FAF094F7F8F094D401CD92F5
:1005A000DD92ED92FC921397F801E855FA4F8D8198
:1005B0009E81AF81B88580839183A283B38380E0DD
:1005C00090E0A8E4B2E489839A83AB83BC83E09093
:1005D000B005F090B1050091B2051091B3052091DE
:1005E000AC053091AD054091AE055091AF056091DD
:1005F000A8057091A9058091AA059091AB05DE012F
:1006000011966D010E940B53C301B20128960FB6DB
:10061000F894DEBF0FBECDBFDF91CF911F910F9138
:10062000FF90EF90DF90CF90BF90AF909F908F9012
:100630007F906F905F904F9008952F923F924F92CE
:100640005F926F927F928F929F92AF92BF92CF9262
:10065000DF92EF92FF920F931F93CF93DF93CDB76B
:10066000DEB769970FB6F894DEBF0FBECDBF3C0171
:100670004C8B5D8B6E8B7F8B2D878CE0EFE0F3E0F6
:10068000DE01119601900D928A95E1F74C895D8902
:100690006E897F89C3010FDE2D852230D1F060F491
:1006A0002223F1F0213009F073C1212C312C60E8B4
:1006B000462E6FEB562E46C03D853330C9F134309F
:1006C00009F066C1212C312C70E8472E7FEB572EA4
:1006D00036C0212C312CF0E84F2EFFE35F2E2FC0C7
:1006E0009301205E3F4FEC88FD880E891F8941E011
:1006F0006FEF7FEF82E0F4DE6B017C0120E030E001
:1007000040E05FE369857A858B859C850E9466B0B1
:100710009B01AC01C701B6010E944EADF301608799
:10072000718782879387C486D586E686F78630C12F
:10073000212C312CE0E84E2EEFE35E2E03C0DD24A9
:10074000D39401C0D12C2D2D30E03F872E8700237C
:1007500009F463C0C901880F991F880F991F73019D
:10076000E80EF91EE1E0F0E0EC0FFD1FE80FF91FC5
:1007700020E030E040E05FE360817181828193811D
:100780000E9466B0F701E05CFF4F20813181428119
:1007900053810E944EAD9B01AC01C201B101905842
:1007A0000E9466B0F70120813181428153810E940D
:1007B0004FADAB01BC01812C912C5401CC24CA94C7
:1007C000850174012FEF8D2D61DCEC88FD880E8989
:1007D0001F899301205E3F4F41E06FEF7FEF82E082
:1007E0007FDE4B015C01F3016487758786879787FD
:1007F00020E030E040E05FE369857A858B859C8569
:100800000E9466B09B01AC01C501B4010E944EADCF
:10081000F30160877187828793878E859F85880F14
:10082000991F880F991F9301280F391F3F872E8723
:10083000E1E0F0E0EC0FFD1FE80FF91F20E030E0F1
:1008400040E05FE360817181828193810E9466B0A4
:10085000688B798B8A8B9B8B52014101B7FAB094DC
:10086000B7F8B0948E859F85805C9F4F998F888F55
:1008700020E030E040E05FE3FC0160817181828133
:1008800093810E9466B09B01AC01688979898A894D
:100890009B890E944FAD2C893D894E895F890E94BA
:1008A0004FAD9B01AC01C501B4010E9466B0EE855D
:1008B000FF8520813181428153810E944FADAB0180
:1008C000BC01812C912C5401CC24CA948501740163
:1008D0002FEF8D2DDBDB23E333E343E35FE3F30112
:1008E00064857585868597850E944EADAB01BC01F8
:1008F0002FEF82E0CBDBFD85AF2EB12C450128E048
:10090000820E911C880C991C880C991C860C971CD3
:10091000C201B1010E9497AEEC88FD880E891F8943
:10092000940141E08D2DDCDD6B017C0120E030E0A5
:1009300040E05FE3E88DF98D608171818281938170
:100940000E9466B09B01AC01688979898A899B897C
:100950000E944FAD9B01AC01C201B1010E9466B083
:100960009B01AC01C701B6010E944FADEE85FF852A
:100970006083718382839383F5013396EE0FFF1FAB
:10098000EE0FFF1FE60DF71DC082D182E282F382D7
:1009900069960FB6F894DEBF0FBECDBFDF91CF9141
:1009A0001F910F91FF90EF90DF90CF90BF90AF908D
:1009B0009F908F907F906F905F904F903F902F907F
:1009C0000895CF92DF92EF92FF920F93CF93DF9330
:1009D000EC016A017B0100E020E02FDE22E0B7019C
:1009E000A601CE012ADE23E0B701A601CE0125DE55
:1009F000B701A601CE015FDC1CAA1DAA1EAA1FAA70
:100A000018AE19AE1AAE1BAE288539854A855B85AE
:100A100060E070E0CB010E944EAD6CAF7DAF8EAF59
:100A20009FAFDF91CF910F91FF90EF90DF90CF902C
:100A300008958F929F92AF92BF92FF920F931F9350
:100A4000CF93DF93EC01F09082048FEF80938204C8
:100A50008090100290901102A0901202B0901302A8
:100A600010921002109211021092120210921302B0
:100A7000CE01A7DF0E944D5E02E512E02CAD3DAD38
:100A80004EAD5FADF80160857185828593850E94CA
:100A90004FADF80160877187828793871886198622
:100AA0001A861B861CAE1DAE1EAE1FAE0E942652BD
:100AB0008092100290921102A0921202B092130240
:100AC000F0928204DF91CF911F910F91FF90BF9020
:100AD000AF909F908F9008952F923F924F925F9288
:100AE0006F927F928F929F92AF92BF92CF92DF923E
:100AF000EF92FF920F931F93CF93DF9300D01F923B
:100B0000CDB7DEB75C01D090820410928204809150
:100B1000100290911102A0911202B09113028983E8
:100B20009A83AB83BC831092100210921102109230
:100B3000120210921302C50144DFE6E7F4E0D5018A
:100B40009C964D915D916D917C919F9740835183CF
:100B50006283738398964D915D916D917C919B9783
:100B6000448355836683778390964D915D916D9113
:100B70007C91939740875187628773878FEF80932B
:100B8000820410921002109211021092120210921E
:100B9000130282E5282E82E0382E20E030E040E487
:100BA00050E4F10160857185828593850E944FAD87
:100BB0004B015C0120E030E040E450E4D1011496A8
:100BC0006D917D918D919C9117970E944FAD2B0156
:100BD0003C0120E030E040E450E4F10160817181AB
:100BE000828193810E944FADAB01BC0192E0C92E7E
:100BF0008301720121E080E049DA20E030E040E446
:100C000050E4D10118966D917D918D919C911B9727
:100C10000E944EAD4B015C0120E030E040E450E426
:100C2000F10164817581868197810E944EAD2B010F
:100C30003C0120E030E040E450E4D1016D917D9131
:100C40008D919C910E944EADAB01BC01830172015C
:100C500021E080E01BDA89819A81AB81BC8180939D
:100C6000100290931102A0931202B0931302D0923B
:100C700082040F900F900F900F90DF91CF911F91F2
:100C80000F91FF90EF90DF90CF90BF90AF909F902B
:100C90008F907F906F905F904F903F902F9008952E
:100CA000CF92DF92EF92FF92CF93C09182042FEF09
:100CB00020938204C0901002D0901102E0901202A2
:100CC000F090130210921002109211021092120270
:100CD00010921302AEDEC0921002D0921102E09286
:100CE0001202F0921302C0938204CF91FF90EF9012
:100CF000DF90CF9008959C018CE0EBE1F3E0D90107
:100D000001900D928A95E1F798E0E7E2F3E0D901CE
:100D1000A05CBF4F01900D929A95E1F708954F9214
:100D20005F926F927F928F929F92AF92BF92CF927B
:100D3000DF92EF92FF920F931F93CF93DF93CDB784
:100D4000DEB7C854D1090FB6F894DEBF0FBECDBFD1
:100D5000CE010196D0DFD09082048FEF8093820481
:100D60004090100250901102609012027090130295
:100D7000109210021092110210921202109213029D
:100D800040E050E060EA70E4CE01019689DF40E087
:100D900050E060E87FE3CE0101969EDE40E050E047
:100DA00060E87FE3CE0101967BDF812C912C54011A
:100DB000CC24CA94850174012FEF40E050E066E135
:100DC00073E480E063D94092100250921102609265
:100DD000120270921302D0928204C85BDF4F0FB6EA
:100DE000F894DEBF0FBECDBFDF91CF911F910F9161
:100DF000FF90EF90DF90CF90BF90AF909F908F903B
:100E00007F906F905F904F9008959F92AF92BF92A6
:100E1000CF92DF92EF92FF920F931F93CF93DF93C6
:100E2000CDB7DEB7C854D1090FB6F894DEBF0FBEF8
:100E3000CDBF81E00E940516009147021092470243
:100E40009090300680E00E94BB1D41E061E081E0AF
:100E50000E94AE558111EEC0CE0101964CDF85E5B2
:100E60000E94E66D882341F12091400C3091410CA5
:100E70002115310509F1F9015F011191812F8F7D54
:100E800099F0153411F01536B9F7F501108260E0CC
:100E900070E08091400C9091410C0E94CBB16B01AD
:100EA0007C01F50110830EC060E070E0C9010E9472
:100EB000CBB16B017C0106C0C12CD12C80E8E82E9F
:100EC0008FE3F82E82E40E94E66D882331F0B701AB
:100ED000A601CE01019600DEADC084E50E94E66D5C
:100EE000882391F08091400C9091410C009731F053
:100EF0004AE050E060E070E00E9431B3B701A60123
:100F0000CE01019696DD96C086E50E94E66D8823A7
:100F100009F48FC0B701A601CE01019652DD8AE027
:100F20000E94C71B88EA9AE10E945D164D855E8586
:100F30006F85788980EA9AE10E94A8168AE00E946B
:100F4000C71B498D5A8D6B8D7C8D87E99AE10E9474
:100F5000A8168AE00E94C71B4D895E896F89788D2B
:100F60008DE89AE10E94A8168AE00E94C71B8AE0D9
:100F70000E94C71B84E89AE10E945D1649855A8544
:100F80006B857C8581E89AE10E94A8168AE00E9420
:100F9000C71B8AE00E94C71B86E79AE10E945D1684
:100FA0004DA55EA56FA578A98DE69AE10E94A816C9
:100FB0008AE00E94C71B49A55AA56BA57CA583E6BC
:100FC0009AE10E94A8168AE00E94C71B49A15AA173
:100FD0006BA17CA18BE59AE10E94A8168AE00E9491
:100FE000C71B8AE00E94C71B8DE39AE10E945D1631
:100FF0008AE00E94C71B84E50E94C71B6AE070E07C
:1010000080E090E00E94BA1C89E29AE10E945D169D
:1010100021964CAD5DAD6EAD7FAD219786E29AE134
:101020000E94A8168AE00E94C71B8AE00E94C71B84
:1010300001C075DE892D0E94BB1D0093470280E030
:101040000E940516C85BDF4F0FB6F894DEBF0FBED7
:10105000CDBFDF91CF911F910F91FF90EF90DF9067
:10106000CF90BF90AF909F9008951F93CF93DF9341
:10107000CDB7DEB72C970FB6F894DEBF0FBECDBF4D
:1010800083E50E94E66D8823B9F08091400C909131
:10109000410C892BC9F00E94706E97FD10C00E9410
:1010A000706E6F3F71058105910509F06CF40E9427
:1010B000706E611109C003C01091300606C080E057
:1010C0000E94BB1D10E001C011E08091520290917E
:1010D0005302A0915402B091550289839A83AB8345
:1010E000BC838091560290915702A0915802B09112
:1010F00059028D839E83AF83B88780915A02909165
:101100005B02A0915C02B0915D0289879A87AB87F0
:10111000BC8786E50E94E66D882331F06DED7AE1AB
:101120008CE096E00E941EA8812F0E94BB1D112317
:1011300051F080913006811106C00E946E168EEB30
:101140009AE10E945D160E946B1680EB9AE10E9464
:101150005D16809130060E94EA164CE050E062E590
:1011600072E0CE0101960E94F3B5892B59F02C96BE
:101170000FB6F894DEBF0FBECDBFDF91CF911F91A8
:101180000C94FE512C960FB6F894DEBF0FBECDBF67
:10119000DF91CF911F9108958F929F92AF92BF924E
:1011A000CF92DF92EF92FF92CF934B015C016901E6
:1011B0007A0122ED30E040EE50ECC701B6010E940A
:1011C0002BB087FD33C027E030E04EE353E4C70186
:1011D000B6010E9428AE18164CF123EA31E040E433
:1011E00050ECC501B4010E942BB087FD1FC027E061
:1011F00030E042E253E4C501B4010E9428AE181663
:10120000ACF027E030E041E253E4C501B4010E94B4
:1012100028AE18165CF0C1E027E030E041E253E46C
:10122000C701B6010E9428AE18160CF4C0E08C2F3E
:10123000CF91FF90EF90DF90CF90BF90AF909F90B5
:101240008F900895CF93DF93D82FC62F0E942D6ED5
:101250008823D1F08091400C9091410C892B11F49E
:1012600081E01AC00E94706E97FD15C00E94706EDA
:101270006F3F71058105910509F094F70E94706E2A
:1012800081E0611109C007C08D2F0E94E66D8111B8
:10129000E7CF8C2F01C080E0DF91CF9108952F928E
:1012A0003F924F925F926F927F928F929F92AF92F6
:1012B000BF92CF92DF92EF92FF920F931F93CF9343
:1012C000DF93CDB7DEB7CB51D1400FB6F894DEBF78
:1012D0000FBECDBF81E00E94051641E061E081E0D4
:1012E0000E94AE5581111AC080913006882329F0E2
:1012F00060E08FE4A7DF811111C0FE0131968CE31D
:10130000DF011D928A95E9F7309030068AE40E9449
:10131000E66D982E882329F00E94DA1D912C0C94FA
:10132000609360E070E086E50E943177C351DF4F43
:1013300099838883CD5ED040059718F080EC9CE1BE
:1013400036C160E084E47EDFC950DF4F8883C75F29
:10135000D040C351DF4F28813981CD5ED04023304A
:1013600031054CF460E084E56DDFC450DF4F8883C5
:10137000CC5FD04006C031E0C450DF4F3883CC5F33
:10138000D04062E070E088E50E943177182F62E07B
:1013900070E089E50E943177082F80E50E942D6E6C
:1013A000811103C0612F802F03C00E94706E862FB1
:1013B000623019F087E99CE1FAC0823019F08EE6BC
:1013C0009CE1F5C083E50E942D6E882319F00E94F0
:1013D000396E04C060E070E88BEB95E420E030E00B
:1013E00040E752E40E942FAE609348027093490296
:1013F00080934A0290934B0288E40E94E66D882312
:1014000091F10E94396E0E9497AE8B0177FF02C066
:101410000F5F1F4F15950795119501951109035BF6
:101420001F4F0E3F4FEF14072CF44DEFA42EBB249B
:10143000BA9401C058016501C60ED71E51EAC516FF
:10144000D1041CF031EAC32ED12C0A3FAFEF1A07AA
:1014500014F409EF1FEF7801E60EF71EB1EAEB1660
:10146000F104CCF135C08CE40E942D6E882331F05C
:101470000E94396E0E9497AE5B0104C02DEFA22E30
:10148000BB24BA9482E50E942D6E882331F00E941D
:10149000396E0E9497AE6B0103C091EAC92ED12C20
:1014A00086E40E942D6E882331F00E94396E0E94DE
:1014B00097AE8B0102C009EF1FEF82E40E942D6EF0
:1014C000882331F00E94396E0E9497AE7B0103C0E1
:1014D00081EAE82EF12CB801012E000C880B990B43
:1014E0000E94CAAEC250DF4F688379838A839B8390
:1014F000CE5FD040B5010B2C000C880B990B0E94DD
:10150000CAAECE5FDE4F688379838A839B83C250E5
:10151000D140C250DF4F288139814A815B81CE5F43
:10152000D0403ADE882309F440C0B7010F2C000CEC
:10153000880B990B0E94CAAE9B01AC01B6010D2C21
:10154000000C880B990BC85EDE4F2883C851D14030
:10155000C75EDE4F3883C951D140C65EDE4F488337
:10156000CA51D140C55EDE4F5883CB51D1400E9455
:10157000CAAEC85EDE4F2881C851D140C75EDE4F7B
:101580003881C951D140C65EDE4F4881CA51D14031
:10159000C55EDE4F5881CB51D140FEDDCA50DF4FD2
:1015A0008883C65FD040811106C082E59CE10E941D
:1015B0005D160C946093B6016A197B09072E000C26
:1015C000880B990B0E94CAAEC65FDE4F6883798391
:1015D0008A839B83CA50D140B701601B710B072ED1
:1015E000000C880B990B0E94CAAEC25FDE4F688365
:1015F00079838A839B83CE50D140C351DF4FE881EA
:10160000F981CD5ED040EF2B91F08CE39CE10E94FC
:101610005D16C950DF4FE881C75FD040EE2321F04F
:1016200082E39CE10E945D168AE00E94C71B0E9433
:101630004D5E80E00E94BB1D81E00E941A4F88230E
:1016400029F0832D0E94BB1D0C9460930E94FE53D1
:1016500060E085E4F7DD811107C0F2E0C350DF4FA1
:10166000F883CD5FD04006C021E0C350DF4F288310
:10167000CD5FD040C151DF4F19821882CF5ED0407C
:10168000C752DF4F188219821A821B82C95DD0406F
:10169000C850DF4F188219821A821B82C85FD0405F
:1016A000C751DF4F1882C95ED0404FEF5FEFC35282
:1016B000DF4F59834883CD5DD0405FEFCB50DF4F84
:1016C0005883C55FD0408FEFCD50DF4F8883C35F15
:1016D000D04091E0CB52DF4F9883C55DD040C352DC
:1016E000DF4F88819981CD5DD0400196880F991F89
:1016F000880F991F4DE350E04C0F5D1F480F591F95
:10170000CB51DF4F59834883C55ED040DC0114972D
:10171000C85FDE4FB983A883C850D1408CE0C35264
:10172000DF4F28813981CD5DD040829FF001839FBA
:10173000F00D1124CA5FDE4FF983E883C650D14013
:10174000CF51DF4F19821882C15ED040C151DF4FA7
:1017500088819981CF5ED040092E000CAA0BBB0B6B
:10176000CE5EDE4F88839983AA83BB83C251D1406A
:10177000C151DF4FA881B981CF5ED040AA0FBB1FF6
:10178000CA5EDE4FB983A883C651D140CB52DF4F2A
:101790005881C55DD040CD50DF4F8881C35FD040B8
:1017A000581709F497C2CE5EDE4F688179818A812D
:1017B0009B81C251D1400E94CAAE9B01AC01C65F61
:1017C000DE4F688179818A819B81CA50D1400E9415
:1017D00066B09B01AC01CE5FDE4F688179818A8162
:1017E0009B81C250D1400E944FAD4B015C01CB5256
:1017F000DF4FB881C55DD0406B2FBB0F770B880BD7
:10180000990B0E94CAAE9B01AC01C25FDE4F68819A
:1018100079818A819B81CE50D1400E9466B09B0124
:10182000AC01C250DF4F688179818A819B81CE5F94
:10183000D0400E944FAD6B017C0120E030E0A90157
:10184000C501B4010E9428AE87FD05C020E030E04C
:1018500040E05FE303C020E030E0A901C501B4012E
:101860000E944FAD0E9405AFC355DF4F6883798357
:101870008A839B83CD5AD04020E030E0A901C70184
:10188000B6010E9428AE87FD05C020E030E040E0B0
:101890005FE303C020E030E0A901C701B6010E9468
:1018A0004FAD0E9405AFC755DF4F688379838A83A8
:1018B0009B83C95AD040C352DF4FE881F981CD5D87
:1018C000D0403196C352DF4FF983E883CD5DD040DD
:1018D000CA5EDE4FE881F981C651D140CB52DF4F5D
:1018E0002881C55DD040E20FF11D27FDFA95EE0F6E
:1018F000FF1F41EA50E04C0F5D1FE40FF51FC3527C
:10190000DF4F88819981CD5DD0409183808301E054
:10191000C351DF4F2881CD5ED040C350DF4F488197
:10192000CD5FD040BE0167557F4FCE0183559F4F9D
:101930000E94BB4FC752DF4F688379838A839B83A2
:10194000C95DD0409B01AC010E9414B1882321F0F5
:10195000832D0E94BB1DD5C1C752DF4F288139811D
:101960004A815B81C95DD040C850DF4F6881798171
:101970008A819B81C85FD0400E944FADC850DF4F25
:10198000688379838A839B83C85FD040CF51DF4FC0
:10199000E881F981C15ED040C85FDE4FA881B9817E
:1019A000C850D140EA0FFB1F2DE630E02C0F3D1F41
:1019B000E20FF31FC752DF4F88819981AA81BB8153
:1019C000C95DD04084839583A683B783C355DF4F19
:1019D000488059806A807B80CD5AD040CB51DF4F00
:1019E000A881B981C55ED0404D925D926D927D9285
:1019F000CB51DF4FB983A883C55ED040CF51DF4FB5
:101A0000E881F981C15ED0403496CF51DF4FF98330
:101A1000E883C15ED040C755DF4F88809980AA8097
:101A2000BB80C95AD0401C968D929D92AD92BC92BB
:101A30001F9720E030E040E85FE35C962D933D93F4
:101A40004D935C935F97A301920169817A818B81A9
:101A50009C810E944FAD69837A838B839C83A5010F
:101A600094016D817E818F8198850E944FAD6D8339
:101A70007E838F839887C752DF4F288139814A81BF
:101A80005B81C95DD04069857A858B859C850E9484
:101A90004FAD69877A878B879C87A3019201C30129
:101AA000B2010E9466B09B01AC016D857E858F8579
:101AB00098890E944FAD6D877E878F87988BA5018F
:101AC0009401C501B4010E9466B09B01AC01698913
:101AD0007A898B899C890E944FAD698B7A8B8B8B1D
:101AE0009C8BC752DF4F288139814A815B81C95D58
:101AF000D040CA01B9010E9466B09B01AC016D895A
:101B00007E898F89988D0E944FAD6D8B7E8B8F8BD8
:101B1000988FA5019401C301B2010E9466B09B0198
:101B2000AC01698D7A8D8B8D9C8D0E944FAD698F34
:101B30007A8F8B8F9C8FC752DF4F288139814A81E2
:101B40005B81C95DD040C301B2010E9466B09B01B8
:101B5000AC016D8D7E8D8F8D98A10E944FAD6D8FE4
:101B60007E8F8F8F98A3C752DF4F288139814A819A
:101B70005B81C95DD040C501B4010E9466B09B0184
:101B8000AC0169A17AA18BA19CA10E944FAD69A370
:101B90007AA38BA39CA31DA10EA13FA028A420E0A3
:101BA00030E0A901C301B2010E942BB073016201B0
:101BB00087FF04C0F7FAF094F7F8F094212F302F44
:101BC000432D522DC701B6010E942BB0181624F0E8
:101BD000C12ED02EE32CF22CCDA2DEA2EFA2F8A6CD
:101BE00019A50AA53BA42CA420E030E0A901C50159
:101BF000B4010E942BB07501640187FF04C0F7FA9D
:101C0000F094F7F8F094212F302F432D522DC70177
